:020000040001F9
:10000000B83A0700D5000100F1000100690D0100B8
:1000100000000000000000000000000000000000E0
:10002000000000000000000000000000F5000100DA
:100030000000000000000000F7000100E90F0100CF
:1000400041130100AD0D0100050E01001D0E010060
:10005000ED0D010059130100050D0100110C010007
:10006000151001002D100100451001005D10010068
:1000700071130100991001007D0D0100950D010023
:10008000B10F0100950F0100E10B0100350E0100D9
:1000900023010100CD0F010027010100F90B010030
:1000A000250C0100410C01005D0C0100790C0100E0
:1000B000950C0100B10C0100CD0C0100E90C010010
:1000C0000348854600F04EFD00480047BD9E0100F4
:1000D000B83A070072B6194819491A4A0123002B89
:1000E00003D002600A60013BF9E762B61648004798
:1000F000FEE7FEE7FEE7FEE7FEE7FEE7FEE7FEE7D8
:10010000FEE7FEE7FEE7FEE7FEE7FEE7FEE7FEE7C7
:10011000FEE7FEE7FEE7FEE7FEE7FEE7FEE7FEE7B7
:10012000FEE7FEE7FEE7FEE7FEE7FEE7FEE7FEE7A7
:10013000FEE7FEE7FEE7FEE7FEE7000080E100E005
:1001400080E200E0FFFFFFFFC100010030B50B4679
:10015000014600202022012409E00D46D5409D42A1
:1001600005D31D469540491B254695404019154627
:10017000521E002DF1DC30BD70B50024254600284C
:1001800001DA01244042002901DA01254942FFF742
:10019000DDFFAC4200D04042002C00D0494270BD8F
:1001A00003460B439B0703D009E008C9121F08C090
:1001B000042AFAD203E00B780370401C491C521E3B
:1001C000F9D27047D2B201E00270401C491EFBD246
:1001D00070470022F6E710B513460A460446194652
:1001E000FFF7F0FF204610BDF8B502464A40D40F95
:1001F00042004B0052085B089A4202D2024608466F
:1002000011464A0023D0C30D4A00DDB2120EAD1ACA
:10021000202D35DA49020126490AF6058A19002CF3
:1002200000D0524220214F1B1146B9402A411018DC
:10023000C20D9A4221D0002C17D0012D08DCDA051E
:10024000801AD20F8019D207DBB200F06DFBF8BD27
:10025000DA05801A012340001B06C01880185A4294
:100260008018CA0F1043490007E04908C20711432C
:10027000DA05801A80194008801800F04DFBF8BD9F
:1002800061000122511A001BF7E70122D2075140F9
:10029000AAE70122D2075040A6E7024670B54A40BD
:1002A000D30FDB0740002DD04A002AD0010E140ED8
:1002B000000212020919400A520A8418E501044694
:1002C0005443000A120A2E045043A4194219200C68
:1002D000C543AA18120C0125AD03521C5219120471
:1002E0007F39240400D0521C104301D44000491E21
:1002F000C2B20C06C0092018401C4008802A02D057
:1003000003E0002070BD40084000002900DA002012
:10031000184370BD70B502464A40D50F40004A00F0
:10032000ED0740085208002814D0002A12D0C40D4E
:10033000D30D41020120C0055202490A520AE41AB3
:10034000091812187D34914201D3641C00E0490061
:10035000002C01DA002070BD0023914201D3891ADC
:100360000343400849000028F7D100290AD09142F0
:1003700002D10121C90705E0914201D2012101E02A
:100380000121C943E005C018401900F0C5FA70BD4D
:10039000420005D04200120E52428A4201DB002088
:1003A0007047C90508187047F0B507460846584019
:1003B00087B0C00F049048000E4659004008490815
:1003C000BC1A884105D2384631461E4617460B46B0
:1003D00002465800400810434CD0300D03904005B1
:1003E0005900400D490D0590401A0290402872DADC
:1003F00018030121000B090508430190049800929D
:10040000002805D0019952420020884100920190B5
:10041000029840210A1A0199009800F049FA05460D
:100420000C466B4607CB00F064FAC0197141039A81
:100430000E0D0023D71756401A467A40164344D073
:10044000049A002A2DD0029A012A039A15DC12057B
:10045000C01A914101263605001C7141D20F059E3C
:10046000D2070093019202962A46234600F0A2FA90
:1004700007B0F0BD38463146FAE71605224A0F4666
:10048000B218C01AB74101210905001C4F410018DC
:100490007F41114618187941E20F10436D196441EC
:1004A00013E0E2076D0815436408C2071443039A7A
:1004B00001261205C01A91413605001C7141CE0774
:1004C000400830434908C01851412A46234600F0ED
:1004D00064FACDE7FFE7049801224000C117121A21
:1004E00000238B4104983146C417381AA141EEE726
:1004F00030B40124E407634030BC55E730B4012434
:10050000E407614030BC4FE70000E0FFF0B51FB4E6
:1005100088B00B990998002448400999C00F4900F8
:1005200049080991C0070B990090490049080B91AF
:1005300009990898A64608431CD00B990A980843C5
:1005400018D0099801244000420D4800410D099837
:1005500024050003000B204309900B980003000BB7
:1005600020430B9050181C4940180022019014465B
:10057000104605E0002001460DB0F0BD032801DA69
:10058000034600E003239C46C11A0AAE0AE05F005E
:1005900008ADED5B4F00F75B7D430027AA187C4157
:1005A000491C5B1E6145F2DD410004AB5A52210437
:1005B000120C0A43240C401C0828DFDB019802902F
:1005C0000099704601910090059B049A079906983E
:1005D00000F0F0F9D0E700000DFCFFFFF0B50C468D
:1005E0005C4085B0E40FE40703944C0000266408E7
:1005F00059009446490802460296224321D0624699
:100600000A431ED06200570D4A000E032303550D06
:10061000012402462C492405781B1B0B360B40187D
:1006200023432643614600901C46501AB44103D32D
:100630000098401C009002E0921800985B4100284E
:1006400003DA0020014605B0F0BD002001210905B4
:100650000746864611E064461D46141BB54106D385
:100660006546521BB341744607430C43A646CD076B
:1006700040084908284392185B4105460D43EAD1DA
:100680001046184313D06046194650407140084345
:1006900006D06046101AB34106D20122002306E0BC
:1006A00000220123DB0702E00122D243531000980D
:1006B00074460105381C6141029C039D0019694183
:1006C00000F06BF9BFE70000FD030000C217C10F87
:1006D000504010B54018CA079623002100F024F9B5
:1006E00010BD10B500229623114600F01DF910BD73
:1006F0000EB505490291002100910A460B46019171
:1007000000F058F903B000BD33040000C20F4100EF
:1007100040020123400ADB05D207090EC0187F29D9
:1007200001DA00207047962903DC9623591AC84045
:1007300001E096398840002AF4D0404270474100D9
:1007400040020122400AD205090E80187F2901DAF1
:1007500000207047962903DC9622511AC840704742
:10076000963988407047000070B5CD0F4A000903E4
:100770000123090B1B0519430B4BED070024520DF8
:100780009A4201DA002070BD074B34339A4203DCF1
:100790009A1A00F09DF802E00449511888402C4351
:1007A000F1D0404270BD0000FF030000CDFBFFFF11
:1007B0004A0009030123090B1B051943094B10B516
:1007C000520D9A4201DA002010BD064B34339A4292
:1007D00003DC9A1A00F07CF810BD034951188840D8
:1007E00010BD0000FF030000CDFBFFFFC20FD207CA
:1007F000400040080BD0C10D0723DB01C91840029F
:100800000905400A1143C208400711437047002000
:100810000146704710B5002904DB0124E40740427B
:100820008C412146002B04DB1C460123DB0752428E
:10083000A3418B4200D1824210BD00000122D207A9
:10084000002800DB101A002900DB511A884270478B
:10085000F0B51FB40646002082B005464024019141
:1008600000901BE0019922460F46304600F030F818
:10087000049A059B801A994110D3104619462246C6
:1008800000F016F8361A8F41019722460120002108
:10089000009F00F00DF838184D4100902046641E6E
:1008A0000028DFDC019B00982946324607B0F0BDE6
:1008B00010B5202A04DB0146203A9140002010BDEB
:1008C000914020239C1A0346E3401943904010BDF9
:1008D00010B5202A04DB0846203AD040002110BD84
:1008E0000B46D340D0402024A21A91400843194619
:1008F00010BD10B5202A06DBCB170846203A104160
:10090000C1170B4306E00B461341D0402024A21A26
:1009100091400843194610BD002904DA401C4900E3
:1009200001D140084000704770B40024050C05D187
:100930001024000402D1002921D01124050E01D178
:1009400000020834050F01D10001241D850F01D1DB
:100950008000A41C002801DB4000641C002908D092
:1009600020252E1B0D46F540A14000D00121294332
:10097000084301061B1B000ADB1D02D5002070BCCA
:100980007047DB05181880180029F8DA401C490068
:10099000F5D170BC40084000704710B5002B08DA54
:1009A0000024401C614192185B411A4301D1400868
:1009B000400010BDF0B51FB482B005460C0003D056
:1009C000084600F003FD02E000F000FD2030024682
:1009D000009021462846FFF76BFF049B059A0446CA
:1009E0000F4618431143084314D0184610431BD038
:1009F000009840210A1A18460599FFF769FF054635
:100A00000E46009A05990498FFF752FF084305D057
:100A1000012004E02046394607B0F0BD0020C11790
:100A200005430E432C43374300990E986305401A43
:100A30007905E40A00220C43FD0A0A3002D50020A1
:100A40000146E9E70105101969410C9C0D9D00194B
:100A50006941FFF7A2FFDFE7FEB500231A461B1A24
:100A60008A4103DB0020014603B0F0BD4A000D03BC
:100A700001212D0B0905520D0D43D10702D100189C
:100A80006D41521E5110FF31FF31013100270446E4
:100A90003E46384600970191024601210020090593
:100AA000FFF716FFC3197141F818324684468E4687
:100AB0004A4161462846611A904104D36046241A8F
:100AC000954176461F46241900986D41401C0090C0
:100AD0003428E1DDF91930467041091BA84103D2E1
:100AE0000022D243134601E000221346019801057B
:100AF000381C7141FFF751FFB6E700004A000903B7
:100B00000123090B1B0519430A4B10B5520D9A42DC
:100B100002DA0020014610BD064B34339A4203DC52
:100B20009A1AFFF7D5FE10BD034BD218FFF7C0FE8F
:100B300010BD0000FF030000CDFBFFFF10B5002932
:100B400004DB0124E40740428C412146002B04DBF6
:100B50001C460123DB075242A341994200D1904237
:100B600010BD0000064C0125064E05E0E36807CCE9
:100B70002B430C3C98471034B442F7D3FFF7A4FA48
:100B80003CEB01006CEB010070B58C180578401C43
:100B90006B075B0F01D10378401C2A1106D1027844
:100BA000401C03E006780E70401C491C5B1EF9D106
:100BB0002B0705D40023521E0DD40B70491CFAE7F5
:100BC0000378401CCB1A921C03E01D780D70491C61
:100BD0005B1C521EF9D5A142D8D3002070BD000085
:100BE00004480068002803D002488030806800472D
:100BF000704700000001070004480068002803D087
:100C000002488030C06900477047000000010700BB
:100C100003480168002901D0C06D004770470000FB
:100C20000001070005480068002805D0034880300F
:100C3000006A002800D0004770470000000107004C
:100C400005480068002805D003488030406A002825
:100C500000D0004770470000000107000548006809
:100C6000002805D003488030806A002800D0004763
:100C7000704700000001070005480068002805D003
:100C800003488030C06A002800D000477047000049
:100C90000001070005480068002805D0034880309F
:100CA000006B002800D000477047000000010700DB
:100CB00005480068002805D003488030406B0028B4
:100CC00000D0004770470000000107000548006899
:100CD000002805D003488030806B002800D00047F2
:100CE000704700000001070005480068002805D093
:100CF00003488030C06B002800D0004770470000D8
:100D00000001070003480168002901D0806D0047F9
:100D1000704700000001070070B50D4600281DD087
:100D2000022806D10121142007F06CFF022004F0F4
:100D300037F800240FE00021142007F0DBFF0A2021
:100D400004F03AF80121142007F0D4FF092004F040
:100D500033F8641CE4B2AC42EDD370BD0021142022
:100D600007F050FF70BD000003480168002901D062
:100D7000C068004770470000000107000448016890
:100D8000002903D0806F002800D000477047000082
:100D90000001070004480168002903D0C06F002843
:100DA00000D00047704700000001070004480168B8
:100DB000002903D0406C002800D000477047000095
:100DC000000107000FB410B503AA0648029900F00D
:100DD000EBFA044904A000F0D7FA10BC08BC04B038
:100DE00018470000A00D07000A2573000448016899
:100DF000002903D0006D002800D000477047000094
:100E00000001070004480168002903D0806C002815
:100E100000D0004770470000000107000448016847
:100E2000002903D0C06C002800D0004770470000A4
:100E30000001070005480068002805D003488030FD
:100E4000C068002800D0004770470000000107007C
:100E500070B54A4D08234A4A0121286802F0C4FFB0
:100E600007F0B0FF0028FBD0022003F099FF454CAB
:100E70000CE00823424A0121286802F0B5FF07F080
:100E8000A1FF0028FBD0022003F08AFF207807F0A2
:100E90007FFE0028EDD03A4E30780009000110287E
:100EA0004AD0202848D0302846D00321364802F0C6
:100EB000ABFF07F087FF0028FBD0012003F070FF95
:100EC00031480621263002F09FFF07F07BFF002803
:100ED000FBD0012003F064FF2B480321C01C02F06B
:100EE00093FF07F06FFF0028FBD0012003F058FFAD
:100EF00025480321801D02F087FF07F063FF0028CB
:100F0000FBD0012003F04CFF08231D4A0121286873
:100F100002F06AFF07F056FF0028FBD0F0790028A6
:100F20000AD0C006030E164A0121286802F05CFFB1
:100F300007F048FF0028FBD0207807F029FE0028A2
:100F40001BD0114901200B3908710146002220787D
:100F500007F0D4FE0021207807F00EFE0321207850
:100F600007F020FE0949207807F060FE0121207873
:100F700007F002FE06490020087070BD4805070012
:100F8000FC0A07003D050700030407005D4401005B
:100F9000D601070005480068002805D003488030C6
:100FA0004068002800D0004770470000000107009B
:100FB00005480068002805D00348803000680028F4
:100FC00000D0004770470000000107000548006896
:100FD000002805D0034880304069002800D0004731
:100FE000704700000001070004480168002903D091
:100FF000C06B002800D000477047000000010700C8
:1010000001FEF7FE05016110324F203835383336C6
:10101000A7D2D1BC04480168002903D0006E002883
:1010200000D0004770470000000107000448016835
:10103000002903D0406E002800D000477047000010
:101040000001070004480168002903D0806E0028D1
:1010500000D0004770470000000107000448016805
:10106000002903D0C06E002800D000477047000060
:101070000001070010B504480168044800F05BF85F
:101080000D2005F059FE10BDE40A0700006800407D
:10109000704700207047000004480168002903D011
:1010A000406F002800D00047704700000001070093
:1010B00010B503461846FFF7ECFFC1B204488A009A
:1010C00081580424A143022421438150996010BD1A
:1010D000E00A0700F8B504460E461746002C1BD060
:1010E000002E19D0002F17D0E06880210843E0605F
:1010F00031013846FFF72AF8054631463846FFF7F2
:1011000025F80107090FE8B220602804000E60608E
:10111000803421640020F8BD0120F8BD10B50029FD
:1011200004D00121062003F055FF10BD0021062048
:1011300003F050FF10BDFEB505460C46A089A088FF
:10114000A868C0B28109890101916969C9B2009199
:101150000607360F686980070AD52846FFF7A8FFFB
:10116000E769002F04D0D12221462846236AB847D8
:10117000022E01D00C2E30D1019800280CD10FE0A6
:10118000E86F800718D52068007828602068401C28
:101190002060A088401EA080A0880028F0D10BE02D
:1011A000A088002808D02068007828602068401CAB
:1011B0002060A088401EA080A08800280DD168680B
:1011C000022188436860CA20A062E769002F04D02A
:1011D000CA2221462846236AB847042E30D10198F6
:1011E00000280CD10FE0A089002818D02868A16839
:1011F0000870A068401CA060A089401EA081E86F14
:101200000007F0D40BE0A089002808D02868A16866
:101210000870A068401CA060A089401EA081A08921
:1012200000280DD16868812188436860CB20E06286
:10123000E669002E04D0CB2221462846236AB04717
:1012400000988E2108420FD0686814218843686096
:10125000D120E062CF20A062E669002E04D0D12226
:1012600021462846236AB047FEBD07E0C36F9B07AF
:10127000FCD50B78491C0360521E92B2002AF5D1AE
:1012800000207047F8B505460C462846FFF700FFDA
:1012900001212846FFF742FF2846FFF7FAFEC7B2B2
:1012A000E86800090001E8608026207A217C80003F
:1012B000C9000843E16831430843E86028462268D2
:1012C0006168FFF707FF0620617E002902D1217DBA
:1012D000C90700D0072030218843217D8A06920F5C
:1012E00012010243C02082430806800F8001104390
:1012F000A8601249BA0088502869627E2021002A1D
:1013000003D008434021884300E08843A27E0221A5
:10131000002A01D0084300E08843227E1021002AE1
:1013200001D0084300E08843286101210D2005F029
:1013300065FDE868B043E860F8BD0000E00A07001A
:1013400004480168002903D0006C002800D0004741
:10135000704700000001070004480168002903D01D
:10136000406D002800D000477047000000010700D2
:1013700004480168002903D0006F002800D000470E
:1013800070470000000107000FB410B503A9044B1B
:10139000044A029800F092F910BC08BC04B0184747
:1013A0001B720100F40A070037B514460846064BC5
:1013B0006A46214600F082F904466946002000F0A2
:1013C00019FD20463EBD0000F51D01002021020C44
:1013D00001D010211046020A01D010460839020936
:1013E00001D01046091F820801D01046891E42080C
:1013F00001D0881E7047081A704730B47446641EC6
:101400002578641CAB4200D21D46635D5B00E31887
:1014100030BC1847002805DBC106C90E01208840F2
:10142000014908607047000080E200E0002805DB09
:10143000C106C90E012088400149086070470000BC
:1014400080E200E0002805DBC106C90E01208840CB
:10145000014908607047000080E200E0002809DBD5
:10146000C106C90E0120884003490860BFF34F8FB1
:10147000BFF36F8F7047000080E100E0002805DBBC
:10148000C106C90E0120884001490860704700006C
:1014900000E100E08307FF22DB0E9A408907090E76
:1014A0009940002808DB830809489B001B1818682E
:1014B00090430843186070470007000F08388308FE
:1014C00004489B001B18D86990430843D8617047B3
:1014D00000E400E000ED00E08307FF22DB0E9A400D
:1014E0008907090E9940002808DB830809489B00FA
:1014F0001818036893430B43036070470007000FFD
:101500000838830804489B001818C36993430B43A9
:10151000C361704700E400E000ED00E002E008C8AD
:10152000121F08C1002AFAD170477047002001E05D
:1015300001C1121F002AFBD1704700000149086059
:1015400070470000F80A0700F0B51FB486B009988C
:10155000089A030D0021024314D05148514A18182B
:10156000504305141198012810981AD0281A401CCD
:1015700000264D4F4D49009601910490002812DA43
:10158000444211E01198012449A3012801D1109887
:10159000C1430698119A84600360C26041600BB039
:1015A000F0BD4042E4E70446210500203F4A001C0C
:1015B00051410391029012E0E00707D032463B46CA
:1015C00001990098FEF7A2FF0191009032463B4638
:1015D00010461946FEF79AFF06460F466410002C87
:1015E000EAD10498039B0028029A0999089806DA20
:1015F000FEF78CFF019B009AFEF788FF05E0FEF7DF
:10160000EDFF019B009AFEF7E9FF04460E4600221B
:10161000284BFFF793FA03D80020C043014607E0A8
:101620000022254B20463146FEF7BEFEFFF766FA44
:10163000102409E0002C0ADB0A220023FFF708F936
:10164000079B30321A55641E02460A43F2D111221A
:10165000641C079B121B1C19119B012B03D0012337
:1016600008430ED10AE0084304D011201090002056
:10167000119077E71098151A6D1E0BE010988242B2
:1016800002DD00236D1C03E0824201DA00236D1E9F
:10169000002BEED0069811998260C16030C07EE7C1
:1016A00001FCFFFF104D0000000014400000F03F5F
:1016B000300000000000F0430000E03FFFB597B0AD
:1016C0000646002518E2252877D100242746FD4943
:1016D000049400E00443761C32780120203A9040C4
:1016E0000842F7D130782A280ED0022230780146FD
:1016F0003039092916D804990A235943303940183A
:101700001443761C0490F1E7189802C804911890CD
:10171000002904DA012040030443484204900220D7
:101720000443761C30782E2814D1042004437078AA
:10173000761C2A2809D11898761C80C8189009E0D0
:101740000A214F43303FC719761C307801463039A3
:101750000929F5D930786C2810D006DC4C281AD02D
:1017600068280ED06A2817D104E0742813D07A288C
:1017700012D110E00120400504430CE001210905CD
:1017800001E0032109050C437178814203D1012056
:1017900000052418761C761C3078119066280BD032
:1017A00013DC58287DD009DC00287BD04528F6D0F2
:1017B0004628F4D047281AD1A5E118E0632835D08F
:1017C000642870D0652812D19DE170286CD008DCA7
:1017D0006728F1D069287BD06E280DD06F2806D1FC
:1017E000BAE073282ED0752871D0782859D01A9A6B
:1017F000199990476D1C7EE16002400F022809D0C4
:1018000003280DD00428189801680DD00D60001D24
:10181000189070E11898EA1701680D604A60F6E7C1
:10182000189801680D80F2E70D70F0E718986A4685
:1018300001781172001D18900020507202A80090CB
:10184000012005E0189802C8189000200091C043BC
:1018500061070DD5002101E00199491C0191B942B0
:1018600012DA8142F8DB009A515C0029F4D10BE0D6
:10187000002101E00199491C01918142FADB019AA2
:101880000099895C0029F5D1019904981A9B471A9F
:1018900021463846199A00F097FA019940194518DF
:1018A0000BE04FE02CE113E04EE000980099007847
:1018B000491C00911A9A199990470198401E01906D
:1018C000401CF2D1214638461A9B199A10E137E0A4
:1018D0000A200021009001916002410F022907D0E7
:1018E000189A01CA1892C2179446032908D00AE030
:1018F0001898C01DC108C90005C91891944607E091
:1019000000B2C2179446042902D140B2C1178C46D6
:1019100000226146944506DA0A4600214042914180
:101920008C462D2102E0210504D52B216A46117336
:10193000012103E0E10701D02021F7E7029155E002
:101940000A200AE0102008E0102000900021042066
:1019500004430191082703E0082000210191009031
:101960006002410F022907D0189A01CA189200227A
:101970009446032908D008E01898C01DC108C90082
:1019800005C91891944603E080B2042900D1C0B281
:1019900000210291210729D51199702906D0009ABA
:1019A0001021019B4A401A4305D00EE040216A46AF
:1019B0001173012108E06146014306D030216A46D7
:1019C00011731199517302210291009A0821019B10
:1019D0004A401A430AD16146014301D1610705D546
:1019E00030216A46117301217F1E029111995829F5
:1019F00004D035A10E910DA90D910DE037A1F9E7A5
:101A00006146019B009AFEF723FF0E9B8C469B5C70
:101A10000D9A521E0D92137061460143F0D10D983C
:101A200005A9081A20300190600703D501200004A1
:101A3000844300E001270198874201DD381A00E065
:101A40000020019900904118029809180498401A42
:101A50000490E00306D421461A9B199A049800F0DA
:101A6000B3F94519002706E003A81A9AC05D199931
:101A700090476D1C7F1C02988742F5DBE0030CD574
:101A800021461A9B199A049800F09EF9451904E022
:101A90001A9A3020199990476D1C0099481E0090A1
:101AA0000029F5DC08E00D980D990078491C0D918E
:101AB0001A9A199990476D1C0199481E01900029A6
:101AC000F1DC63E109280100303132333435363737
:101AD000383961626364656600000000303132337A
:101AE000343536373839414243444546000000001A
:101AF00000F05AF94519761C3078002800D0E2E54C
:101B000028461BB0F0BD600700D406271898C01DFA
:101B1000C108C90048680A680831C30FDB0718917B
:101B2000190001D09CA108E0210501D59BA104E08A
:101B3000E10701D09AA100E09AA1430011985B0847
:101B4000109165280CD006DC452809D046281DD008
:101B5000472841D141E0662818D067283CD13CE0B5
:101B60000021112F01DB112000E0781C0191009071
:101B700008A911A8FFF7E8FC139905910021119A13
:101B800015927F1C12980197009150E00120C00728
:101B900003900120019008A9009711A8FFF7D4FC39
:101BA000139A149905920022119B00921298159392
:101BB000059A0192002901D0104602E0791C4018D4
:101BC0000190381A01D5019804E04042401E00906F
:101BD000781C0190C01B029043E0012F00DA01271E
:101BE0000021112F01DD112000E038460191009005
:101BF00008A911A8FFF7A8FC13990591119A0021D3
:101C0000129815920091019721070CD40599B942B9
:101C100001DB019900E00191012904DD159A491EBB
:101C2000515C302906D0B84201DA011D05DA0121E4
:101C3000029115E00199491EEDE7002805DC0099A5
:101C4000411800910199091A03E0019A411C91423F
:101C500000DD01910099401A401C02900120C0074C
:101C60000390200706D402990198814202DB0020EC
:101C7000C043029000206946C87707AF012103984E
:101C80000337C907884224D0022011902B201290DC
:101C9000039800280CDA404203902D20129007E0B0
:101CA0000A210398FEF752FA30317F1E03903970F3
:101CB0001199481E11900029F2DC03980028EFD1F9
:101CC000791E129808703078202108404530BF1ED8
:101CD000387006A8C01BC01D03901098007800281B
:101CE00000D00120019941180298C01709180398E3
:101CF00009180498401A401E0490E00306D42146B7
:101D00001A9B199A049800F05FF84519109800780A
:101D1000002803D01A9A199990476D1CE00324D526
:101D200021461A9B199A049800F04EF845191CE0B8
:101D30000098002807DB00990598884203DD159874
:101D4000405C199901E0199930201A9A904700983F
:101D50006D1C401C00900298401E0290002804D187
:101D60001A9A2E20199990476D1C0199481E0190CE
:101D70000029DDDC05E038781A9A7F1C1999904714
:101D80006D1C0399481E03900029F4DC21461A9B20
:101D9000199A0498ACE600002D0000002B0000000A
:101DA0002000000000000000F8B5044600251E4693
:101DB0001746880404D405E039462020B0476D1C3E
:101DC000641EF9D52846F8BDFFB50446002581B04C
:101DD0001E46C80301D5302700E02027880404D51B
:101DE00005E038460399B0476D1C641EF9D52846B6
:101DF00005B0F0BD0A68531C0B60107070470000FE
:101E0000F0B5FD4EABB00D46F06905F0CDFADA2D18
:101E10003CD00124DB2D45D0DC2D4FD00A2D57D0EE
:101E20000E2D7FD00F2D72D00027EE2D70D0032DF8
:101E30006FD0042D6ED0052D6DD05A2D6CD0872D0E
:101E40006BD0FE2D6AD07F2D69D0E92D68D0A12DF1
:101E500067D0A22D72D0D62D71D09A2D70D0C62DFC
:101E60006FD0C72D6ED0B52D6DD0B82D6CD0C82DCC
:101E70006BD0C92D6AD0F069EA2D68D005F094FACC
:101E800000902B46DD4ADEA1E0A0F0E3F06905F00A
:101E90008BFA012804D081222B46920000900AE39D
:101EA000A120FFE0F06905F07FFA012804D0852227
:101EB0002B4692000090F2E70094F4E0F06905F000
:101EC00073FA012870D089222B4692000090E6E731
:101ED000F06905F069FA9F21012805D0032805D093
:101EE0002B46D44A0090DAE70091DCE0707A0028B3
:101EF00001D09B202DE0009101910291032300224B
:101F00001C21F06905F01CFE7472B3E20AE025E0C2
:101F100027E030E039E048E051E0A5E0C1E0C9E069
:101F200028E139E1F06905F03FFA01287ED0032865
:101F30000ED0C04A2B4618320090B0E7F0E1B1E273
:101F4000C3E2D1E253E3C5E3D4E3E2E3F4E3F4E331
:101F500080200090019002900323EFE33471C020B1
:101F6000A0E0F06905F020FA01287DD0B14A2B46A7
:101F70003332009093E7F06905F016FA01289BD000
:101F8000AC4A2B464332009089E7F06905F00CFA21
:101F9000032804D0A74A2B46533200907FE7042041
:101FA000A12101940091D6E7F0E0F06905F0FCF979
:101FB000012874D02B222B46120100906FE7B07AD3
:101FC000002838D0BB21AC229B2021972891269253
:101FD00025972797239724901D9720921C91199756
:101FE00022911F971B971E9017971597189011977E
:101FF00012901A92149216911397F6200EAB0D9729
:1020000091C3FF20ED210C910B970A9003210690BC
:10201000079708917D2009940594292300220291B5
:1020200001970397009404901C2100E03BE1F069C4
:1020300005F086FD69E7259726972797289721972A
:1020400022972397249720971D971E971F971B97DA
:102050001C9719971A97169717971897159711970E
:1020600012971397149700E019E00F9710970D97A8
:102070000E970A970B970C970997032005970697D9
:1020800007970397019702940497009408902923D7
:1020900000221C21F06905F053FDB47235E700976A
:1020A00001E010200090012300222121F06905F0B9
:1020B00047FD2AE7F06905F077F9B9210A2808D029
:1020C00004284AD0032850D05A4A2B46C8320090E0
:1020D000E5E6307B002804D0012819D002282AD058
:1020E00013E703976E209B230497089133220297EE
:1020F00005970693099040210792042000910190D2
:102100000A2300221C21F06905F01AFD3473FCE655
:1021100006970797089709970597029703970497DB
:10212000009701970A2300221C21F06905F008FDA1
:1021300002203073E9E606970797089709970597F5
:10214000029703970497009701970A2300221C2106
:10215000F06905F0F5FC3773D7E66E2033229B2338
:102160000093019202910390D6E0FF20019702971D
:102170000090F1E6F06905F017F9012806D0022871
:1021800006D02C4A2B46E032009088E6042089E7EE
:10219000042001970090ABE2F06905F005F90A28E8
:1021A0000BD014287CD007287BD004287AD00128B3
:1021B00079D02B46204A009071E6707B002804D02D
:1021C00001283BD0022852D09FE6162321220D2160
:1021D0000E2006AD0FC50A23A4228E210C2002ADCD
:1021E0000FC5ED210B200191009000221C21F06908
:1021F00005F0A6FC747388E6D001070046050000D0
:102200005332315F64656D6F000000005B25735DC4
:10221000202825303464292072202578206E6720FC
:102220006E6565642072657475726E205B25645DF1
:102230000A000000470200006E030000532333220F
:102240005421582006AD0FC534204121FB220590B2
:102250000392049130200294019400900A230022FA
:102260001C21F06905F06CFC022070734DE63220F1
:1022700034214622079006920891099042234A226F
:102280003821372002AC0FC4332141200191009046
:102290000A2300221C21F06905F052FC777334E612
:1022A00002E026E033E039E031221192302134207F
:1022B00047230C9242250DAF10931391129029C71A
:1022C0004122332353250B930A92099505905423F9
:1022D00008905825079306950492F92000910194DF
:1022E00002940390142300221C21F06905F028FCBD
:1022F0000BE61420E0212F22049003920691059012
:1023000006220221A5206C4607C4072374E2872316
:102310000C22EF210B20FDE3042379E28120C1E6AA
:10232000F06905F041F80A2805D0092872D02B463B
:10233000F84A0090B3E5B07B00280FD01C2101289B
:102340001CD0022826D0032834D0042841D00528E8
:102350004FD006285FD007286DD084E038230422B0
:102360006021092006AC0FC480203022892105900D
:10237000112002970492039100905AE002200E224D
:102380000890029009920690049003910797059196
:1023900078200CE0CF210C200991079007210697A7
:1023A0000897AF220B2002AB059185C32020009730
:1023B000019052E00321069120220C2007AB85C337
:1023C000F022102118200290039705920491D92041
:1023D000EDE75424462338222A2006AD1DC50E22DF
:1023E00033230B2005910621039304920290009160
:1023F000DEE7022009907E227D2106AD16C57721F9
:102400007B20792370220391059069210493029225
:10241000622020E02FE01921FA22FC2007AB069170
:1024200007C30920BE224021009402900592039127
:102430000490019711E02A21F62208911A200992AE
:10244000B6237821079338220591069002900490D4
:10245000F82103921920019100900A2300221C21E7
:10246000F06905F06DFBB07B401CC0B2B07307286B
:1024700000D9B77313E2B773F4216B22742007916C
:1024800006922B213B230590342208970291049356
:10249000019200910390092300221C21F06905F0AC
:1024A0004FFBFCE1F06904F07FFF052804D0994A56
:1024B0002B460F320090FDE3EE2398223021452079
:1024C00001AC0FC408200090F5E3F06904F06CFF44
:1024D000042804D08F4A2B461F320090EAE343239E
:1024E0006B22EA212D2015E3F06904F05DFF0A2834
:1024F00008D0032877D0012877D0864A2B465C3253
:102500000090D7E3F07B002806D001281CD00228D9
:1025100034D003284DD0C2E1F521099193230E2236
:10252000052006AD0DC520221021059202900491D0
:1025300008200397009401900A2300221C21F069CF
:1025400005F0FEFAF473AAE1412307934522A42182
:10255000E4231120089206910293099010222E2163
:1025600003AC07C40E212A20019100900A23002207
:102570001C21F06905F0E4FA022018E0D520812141
:102580009123069108900993142117220792039131
:102590000491602205907D210292F4200191009027
:1025A0000A2300221C21F06905F0CAFA0320F07307
:1025B000DAE32820DB211E221923069307920891D3
:1025C000099005901F23C222D62102AC0EC4C1215E
:1025D0001D20009101900A2300221C21F06905F0C2
:1025E000AFFAF773C0E37FE0FFE755205AE5F069E3
:1025F00004F0DAFE0A2806D0032875D0454A2B4697
:1026000090320090A0E3307C002806D0012815D03D
:1026100002282DD0032843D0A6E33822F2230992C2
:10262000A221089308200C22072307900E20059270
:102630000691029003930491009028E01123172241
:102640003921632006AC0FC40E23D62274217220D8
:1026500002AC0FC40A21BC2001910B46009000225D
:102660001C21F06905F06CFA022030747CE36DE304
:102670008D2385221821772006AC0FC47D23F422F8
:102680001321452002AC0FC4D120032400940190F3
:102690000A2300221C21F06905F052FA347463E326
:1026A0002821DB2219230892099106931E20059107
:1026B00034220223C7210790E72403930492009158
:1026C000029401900A2300221C21F06905F038FAD7
:1026D000377449E3F06904F067FE022805D00D4A1B
:1026E0002B46A03200902FE327E1032114200DE0B8
:1026F000022399E0F06904F057FE022804D0472233
:102700002B46120100901FE3B221C02001910090DE
:10271000EEE701E0BF030000F06904F045FE0A287F
:102720000DD08A2107285CD004286BD0022876D0EF
:102730002B46FE4A009007E37CE0FEE2F7E2727C63
:102740005F205E21002A04D0012A1AD0022A30D04C
:102750000AE36022079006920891099005916E2085
:1027600045223923049032210293039220200191C3
:1027700000900A2300221C21F06905F0E1F974742D
:10278000F2E25D230991079350224A2108900692B4
:10279000029103914E2305924821049301910090E8
:1027A0000A2300221C21F06905F0CAF90220707486
:1027B000DAE25C212B226E2007AB069107C344238B
:1027C00052224221582002AC0FC45B2157200191B4
:1027D00000900A2300221C21F06905F0B1F97774FA
:1027E000C2E2C824232334222B2003AD1DC51420AC
:1027F000042302970091019000221C21F06905F04A
:102800009FF9B1E22B2014226C46039086C4042366
:1028100000221C21F06905F093F9A5E2FFE72321CE
:10282000662001230191009000222221F06905F029
:1028300087F999E2F06904F0B7FDC923AD210A28B0
:102840000DD08822272879D02B2874D0042873D063
:10285000032872D0B54A2B468332009074E2B07CD4
:102860003546002806D001281AD0022830D0032887
:1028700047D079E20F220692F3210D2007AE0BC656
:102880001421029100910191B523732203AE0DC66C
:102890000A2300221C21E86905F052F9AC7463E2B6
:1028A000122339220D21742006AC0FC410231B22E1
:1028B000DD21932002AC0FC40E2113200191009062
:1028C0000A2300221C21E86905F03AF9022016E0EB
:1028D00018220792099175205921089002917F24AE
:1028E0007422142003AE1DC66121242001910090A2
:1028F0000A2300221C21E86905F022F90320A874AC
:1029000032E2DB22282008921923069309902E2216
:10291000F6231E2103930492059007918624C72075
:102920006E4613C60A2300221C21E86905F008F947
:10293000AF7419E202E047E0EBE1F2E12691A62450
:10294000F823252023AD19C5A724209450207621F3
:10295000D7242023219122901E941F93E125F52155
:1029600019201BAF23C78425C1240421152017AFCC
:1029700033C7512516951224139415901293692488
:1029800023250F20109511940D921491D9233224F0
:102990000B250F900B950C940E93BC223423092425
:1029A0000A9282250794099308954123009002AF6B
:1029B00001900BC76624242214C7272300221C2160
:1029C000F06905F0BDF8CFE1F77A2721002F12D08A
:1029D000FE23012F5CD0022F7ED0032F7DD0042F49
:1029E0007CD0524A00902B4670325149019751A039
:1029F000FEF7E8F9B8E1F472F62068222A932892EB
:102A0000279129907023D2227721222023AD0FC550
:102A1000252222921E201F907D20DA211D90462320
:102A2000BE242191552220931E941C9218231B939F
:102A300075221992E423732018931A901324179483
:102A4000D9221124139415924420169043231493F1
:102A5000A3240E23452210940F9311921720422293
:102A60000E91129094240C920B230D940B936022E0
:102A7000C2210223099208930A910A242022622388
:102A80000794A22108240394049305920691AFE0D1
:102A90000224F472CC2027AD2A900EC5269023ADD7
:102AA0000EC52823EA2256211E201FAD0FC5BC22C9
:102AB0007521F5231E921C931D917122E42317208A
:102AC000132518931A92199117954321D92233236C
:102AD00011251B90139502E046E08DE0D3E014939E
:102AE000159216915523B3220E210FAF12900EC7E7
:102AF000A4210B230D91DC2572220B930E950C92D1
:102B00006223C721782208930A250A91AE230992ED
:102B10004C2100E001E1009005AF01902AC7092295
:102B200002AD15C5272300221C2119E0AC040000CA
:102B3000002201005B25735D2028253034642920A4
:102B400043392D2D2D2D2D20725B25785D205B25A1
:102B5000645D205B25645D6572720D0A00000000F3
:102B6000F06904F0EDFFFFE00320F072CC2027AC09
:102B70002A900EC4269023AC0EC42291E223562242
:102B80001E201FAC0DC4BD211E917D2415231822CB
:102B90001BAD1CC58523199373211A91F523159339
:102BA0001322F42447271894169781231792119320
:102BB000109212900C9153241125149404220C238A
:102BC00013950F24ED200B930D920F940E90DE21A0
:102BD000A2220B23EC20079308920A910990CE239E
:102BE000C821B2220A2006930492059103908EE038
:102BF00000900190029044E00420F072CC2027ADB8
:102C00002A900EC5269023AD0EC52523DE2236213F
:102C10001E201FAD0FC589201D900522BD211C92CD
:102C200018231E9175201B9399221A901992242320
:102C30001D221893159211234C20139314251690DE
:102C4000B323179510931191B425282293230D21B6
:102C5000149512920C930B910F2571220DAF34C76E
:102C6000F72360220A930992E3240C21EC224323E8
:102C700005901720069208940791009002AD0190EC
:102C80000BC527234FE70520F072CC2027AC2A90F4
:102C90000EC4269023AC0EC42323DE2226211E2040
:102CA0001FAC0FC4C0239922152118201BAC0FC4E0
:102CB0007B2101E048E051E0642218921A9114232C
:102CC00017931224C1205621139419905D22442396
:102CD0001691149315921D213824A42210231294C6
:102CE0000F93109211910E91E924F3230E220BAD54
:102CF0001CC516210A91D52307925324099311214B
:102D0000B32208940D230393049206910590172093
:102D10006EE7DB231E22192128206C460FC4FFF723
:102D2000FBFADB221E2119206C4607C40323002274
:102D30001C21F06904F004FF16E004F035FB0528BF
:102D400007D00B4A2B4600900A490BA0FEF73AF831
:102D50000AE0019702970397049700970523002242
:102D60001C21F06904F0ECFE01202BB0F0BD000046
:102D700041050000002201005B25735D20282530FD
:102D800034642920725B25785D205B25645D2065B5
:102D900072720D0A0000000000210A2005F032FFC7
:102DA0000021042005F02EFF0021142005F02AFF49
:102DB0000021132005F026FF404F01253D7000F053
:102DC00099FF07F081F83E4A3EA141A0FDF7FAFFC6
:102DD00006F0F0FF00210E20FEF75CFB01210F2022
:102DE000FEF758FB00F0DEFF3F48002606703F4C20
:102DF0000320A58206F0D2FE00233D4A0A210320CB
:102E000006F0DAFE2E4A2FA11C323AA0FDF7DAFFB7
:102E10006078002818D007F005F8206A05F09EFCBD
:102E2000322001F0BDFF292302220021052005F0F8
:102E300059FD6670657101F095F901F06FFC022291
:102E40003349012005F0FEFEE0790128A08A2FD049
:102E5000142805D9A682A5710021022005F04AFF99
:102E600000F05AFF01F070FBE06904F047FA002817
:102E7000FAD1A0780028CBD001210A2005F0C2FEAB
:102E8000206A05F0A1FC206A05F05CFBE06904F013
:102E9000CBFFE06904F0E4F9094A0AA169321DA0F8
:102EA000FDF790FFA670002006F074FE3D70AFE7BE
:102EB00021498842D4D9A682A571D1E75B040700D5
:102EC0007B1300005332315F64656D6F00000000BA
:102ED0005B25735D2028253034642920733231202E
:102EE00064656D6F310A00005C040700D0010700C3
:102EF00031AA01005B25735D202825303464292028
:102F000073746172742074696D6572330A00000015
:102F1000C92F01005B25735D2028253034642920EA
:102F200064697361626C6520766964656F207061A5
:102F30007468200A00000000B603000070B58EB06F
:102F40000020FF2206900790059208900A900B90AF
:102F500009920D920C90CB6819462031C8784C78B4
:102F600000020419174844621D7805724C7CC48223
:102F7000CB7C03834E7D468309A9002D1ED0141BF4
:102F80006400E4252C1BD31A5D00EE235D1B921B0D
:102F9000A4B25200C482ADB29A1A058392B242839F
:102FA000099505940D9214226846FDF7F9F805ADD0
:102FB0000FCD05F09FFB01200EB070BD0D9605945E
:102FC0000993F0E7D0010700FF223D3209A10CA0D0
:102FD000FDF7F8FE012006F0D9FD012006F0DAFD2C
:102FE000BFF34F8F11491048C860BFF34F8F00BF28
:102FF000FDE700005332315F64656D6F0000000033
:103000005B25735D20282530346429206469736151
:10301000626C652072657365742121212121212153
:103020002121212121210A000400FA0500ED00E000
:103030001CB5C96851230878497801910090032292
:103040000021392005F04EFC01201CBD10B52823BD
:1030500002220021052005F045FC5922120103A19E
:1030600005A0FDF7AFFE012010BD00005332315F17
:1030700064656D6F000000005B25735D20282530BE
:103080003464292064697370206F6666200A00002A
:1030900010B5034A03A106A0FDF794FE012010BD60
:1030A000AD0500005332315F64656D6F00000000B4
:1030B0005B25735D20282530346429206469737092
:1030C000206F6E200A00000010B5114CE06904F07A
:1030D0006BFE00210846FDF71FFE322001F060FE66
:1030E000102302220021052005F0FCFB142001F032
:1030F00057FE0021132005F0FDFD064A06A109A098
:10310000FDF760FE0120A0700020E070012010BDDE
:10311000D0010700A20500005332315F64656D6F76
:10312000000000005B25735D2028253034642920D1
:10313000656E74657220736C656570206D6F646573
:103140000A00000010B50E4A0EA111A0FDF73AFECC
:103150000120174C0246E07022230021052005F0D3
:10316000C1FB012001F01CFEE06904F07BFE13238B
:1031700001220021052005F0B5FB012010BD000053
:10318000B50500005332315F64656D6F00000000CB
:103190005B25735D202825303464292065786974A7
:1031A00020736C656570206D6F64650A0000000017
:1031B000D0010700C8680178012904D140780128AE
:1031C00001D102490870012070470000D0010700BA
:1031D00010B50321294800F017FE05F0F3FD002883
:1031E000FBD0012001F0DCFD24480321C01C00F0CD
:1031F0000BFE05F0E7FD0028FBD0012001F0D0FD1B
:103200001E480421123000F0FFFD05F0DBFD002810
:10321000FBD0012001F0C4FD18480421163000F055
:10322000F3FD05F0CFFD0028FBD0012001F0B8FD33
:1032300012480321801D00F0E7FD05F0C3FD0028C2
:10324000FBD0012001F0ACFD0C480321093000F057
:10325000DBFD05F0B7FD0028FBD0012001F0A0FD4B
:10326000064803210C3000F0CFFD05F0ABFD00282F
:10327000FBD0012001F094FD10BD00000F040700F9
:103280000020054A01461154401CC0B20628FAD35A
:10329000D1719171916070478C0C07001CB50AA127
:1032A00003C900240191009020016946401C487028
:1032B0000822002000F064FF062001F071FD641C6C
:1032C000E4B2052CF0D31CBD330100000000000067
:1032D00010B50E4C2079002815D0C8680278E07C23
:1032E000824210D0E2744B2120464901C069002A75
:1032F00000D0052204F072FDAD22E37CD20004A1CF
:1033000006A0FDF75FFD012010BD0000D001070001
:103310005332315F64656D6F000000005B25735DA3
:1033200020282530346429204672616D655F726102
:1033300074653A253032780D0A00000010B5054852
:103340004168002901D000208847122003F0F4FCD6
:1033500010BD0000B00A070010B5074C2068002817
:1033600006D001F03BFD002802D0216800208847EC
:10337000172003F0E1FC10BD9805070010B50548C3
:103380000168002901D040688847182003F0D4FC68
:1033900010BD00008C0F070010B50548816800299A
:1033A00001D0C0688847192003F0C6FC10BD00009A
:1033B0008C0F070010B505480169002901D040694C
:1033C00088471A2003F0B8FC10BD00008C0F0700DE
:1033D00010B505488169002901D0C06988471B20C4
:1033E00003F0AAFC10BD00008C0F070010B50548C3
:1033F000016A002901D0406A88471C2003F09CFC28
:1034000010BD00008C0F070010B50548816A002927
:1034100001D0C06A88471D2003F08EFC10BD00005B
:103420008C0F070010B50548016B002901D0406BD7
:1034300088471E2003F080FC10BD00008C0F0700A1
:1034400010B50548816B002901D0C06B88471F204B
:1034500003F072FC10BD00008C0F07009D2202A13A
:1034600004A0FDF7AFFCFEE76472765F636F6D6DDD
:103470006F6E00006572726F72205B25735D20288D
:10348000253034642920456E746572206861726449
:103490006661756C7420696E746572727570742ED5
:1034A0000D0A00000249014809680847004C004025
:1034B000A805070002490148096808470050004074
:1034C000A405070070B5184D2C68A8680440A00733
:1034D00002D507F067FA1FE060070DD503F02AF95F
:1034E0000146114E803E304602F02EFF002202219E
:1034F000304602F09CFF0FE0E00705D00B4A0CA11C
:103500000EA0FDF75FFC07E0200705D5074A08A1DC
:10351000121D16A0FDF756FC686820436860012064
:1035200003F00AFC70BD0000800800409605000012
:1035300068616C5F7673796E630000006572726F0C
:1035400072205B25735D20282530346429204C438C
:1035500044433A4C4344435F494E545F44425546CA
:103560005F554E444552554E210000006572726F02
:1035700072205B25735D20282530346429204C435C
:1035800044433A4C4344435F494E545F5352435F74
:1035900044504948414C545F494E545F4D534B2170
:1035A0000000000010B5204C0021204603F03AF83E
:1035B000002803D00021204603F008F8012120460E
:1035C00003F030F8002803D00121204602F0FEFF6E
:1035D0000221204603F026F8002803D002212046CD
:1035E00002F0F4FF0321204603F01CF8002803D06A
:1035F0000321204602F0EAFF0421204603F012F8DE
:10360000002803D00421204602F0E0FF05212046D7
:1036100003F008F8002803D00521204602F0D6FF69
:10362000042003F089FB10BD000C0040F8B53949B7
:10363000CC683948394F3A4D044213D0394A0020FA
:10364000506048600120506048602B68364A37A1BE
:1036500038A0FDF7B7FB3B6B334A34A1521C3FA0A7
:10366000FDF7B0FBA00706D52B6A2F4A2FA1521DEC
:1036700044A0FDF7A7FB4D4E600706D533682A4AE4
:103680002AA109324AA0FDF79DFB200706D5336A1F
:10369000254A26A10D3250A0FDF794FBE00606D581
:1036A0003B68214A21A1113255A0FDF78BFBE003B5
:1036B00006D52B691C4A1DA115325CA0FDF782FBC3
:1036C000A00306D52B6B184A18A1193260A0FDF78C
:1036D00079FB600306D52B68134A14A11D3215A08F
:1036E000FDF770FB200306D5336B0F4A0FA1213283
:1036F00060A0FDF767FB600208D508484030036909
:10370000094A0AA1263264A0FDF75CFB022003F0FF
:1037100013FBF8BD0028004001002000802A004073
:10372000002A004000290040A50200006473695F80
:10373000727800005B25735D2028253034642920D1
:103740004453495F52585F4552525F5048595F4653
:103750004154414C5B307825785D0A005B25735DF0
:1037600020282530346429204453495F52585F454E
:1037700052525F4552525F5250545B307825785D0B
:103780000A0000005B25735D202825303464292061
:103790004453495F52585F4552525F4453495F4614
:1037A0004154414C5B307825785D0A00402A004046
:1037B0005B25735D20282530346429204453495FFC
:1037C00052585F4552525F4444495F464154414C10
:1037D0005B307825785D0A005B25735D20282530F5
:1037E000346429204453495F52585F4552525F491F
:1037F00050495F464154414C5B307825785D0A0062
:103800005B25735D20282530346429204453495FAB
:1038100052585F4552525F4649464F5F46415441B8
:103820004C5B307825785D0A000000005B25735DF5
:1038300020282530346429204453495F52585F457D
:1038400052525F5048595B307825785D0A0000007D
:103850005B25735D20282530346429204453495F5B
:1038600052585F4552525F4453495B307825785D2A
:103870000A0000005B25735D202825303464292070
:103880004453495F52585F4552525F4950495B303B
:103890007825785D0A0000005B25735D20282530BF
:1038A000346429204453495F52585F4552525F5255
:1038B000585F54524947474552535B307825785DED
:1038C0000A00000070B50D48C36B0C484030046816
:1038D000416885680B4204D0094A0AA10BA0FDF794
:1038E00071FA2C4206D08F222346D20005A112A0E5
:1038F000FDF768FA032003F01FFA70BD8004004052
:10390000730400007461755F6C6F67006572726F9D
:1039100072205B25735D202825303464292054589B
:1039200020494E5420696E745F7374303A307825A4
:103930003038780A000000006572726F72205B25D3
:10394000735D2028253034642920545820494E5472
:1039500020696E745F7374313A3078253038780A94
:1039600000000000F8B5132003F0E6F900240D4D27
:103970000D4F0126E9693046A04001420DD069692A
:1039800001436961A969014207D07868002800D025
:1039900004703968002900D08847641C062CE9DBD4
:1039A000F8BD000000780040D00A070010B50848B4
:1039B0000168002901D007488847074801690122AA
:1039C0005204914301611120FDF73CFD10BD000040
:1039D000540A07000040004000880040F8B57C4EC3
:1039E000316800291CD07B4C70687A4A0027403C23
:1039F00001281AD0636ADDB2A84204D8022819D07F
:103A000003281FD085B231468B690868C0182B0087
:103A1000FDF7F3FC09A02329313B475565778B005F
:103A20000021F26908469047CEE0106A0870012034
:103A3000B0619AE00220B061106A0870106A3168C3
:103A4000487092E00320B061106A0870106A316813
:103A50004870106A3168887087E0136A037088695B
:103A6000401C886176E0136A0370136A43708869AA
:103A7000801C88616EE0136A0370136A4370136AD6
:103A800083708869C01C886164E0136A0370136ADC
:103A90004370136A8370136AC3708869001D88615C
:103AA00058E0136A0370136A4370136A8370136AD1
:103AB000C370136A03718869401D88614AE0136A04
:103AC0000370136A4370136A8370136AC370136AB6
:103AD0000371136A43718869801D88613AE0136A33
:103AE0000370136A4370136A8370136AC370136A96
:103AF0000371136A4371136A83718869C01D8861F9
:103B000028E0136A0370136A4370136A8370136AA0
:103B1000C370136A0371136A4371136A8371136A62
:103B2000C37188690830886114E0136A0370136AEE
:103B30004370136A8370136AC370136A0371136A44
:103B40004371136A8371136AC371136A03728869BC
:103B5000093088618B694868C01A002805D0636AFB
:103B6000DDB2854225D385B24EE7F26918490120BE
:103B70009047A06AC00713D0174800680006850F59
:103B800002211020FDF7A8FCA06AC007FCD1F26951
:103B90000F490220904729461020FDF79DFC03E0C5
:103BA000F2690B4902209047B761102003F0C4F876
:103BB000F8BD002DD8D1A06AC00700D023E7F26974
:103BC000034902209047B761102003F0B5F8F8BD13
:103BD000942A07004048004010E400E010B515208A
:103BE00003F0AAF8002003F07DF8034801680029DB
:103BF00001D04068884710BDD80A07000448016812
:103C0000491C01604168002901D000200847704725
:103C10008C05070010B5002003F030F910BD10B579
:103C2000012003F02BF910BD10B5022003F026F996
:103C300010BD10B5032003F021F910BD10B5FDF73C
:103C400019FA10BD10B505480168002901D00020FF
:103C50008847002003F070F810BD0000B80A070084
:103C600010B505480168002901D0002088470520CB
:103C700003F062F810BD0000B00A070010B50C2078
:103C800003F05AF80A480078002803D103F0A6FA96
:103C900003F08CFA03F09AFA002808D003F08EFAA9
:103CA0000348001D0168002901D04068884710BD05
:103CB000E80A070010B5024801F084FA10BD0000C0
:103CC0000054004010B50948C168C9B2CC070123AF
:103CD000074A002C00D0D370490700D5137103F0B8
:103CE00097FA062003F028F810BD000000000140FC
:103CF0007805070010B50721482005F09DF8044815
:103D000005F0DAF8C821034805F0CCF810BD000032
:103D1000753D0100C40B070010B507480178002964
:103D200008D000210170FFF753FA044A04A107A04C
:103D3000FDF748F810BD0000D0010700691300002E
:103D40005332315F64656D6F000000005B25735D69
:103D5000202825303464292063616C6962726174A3
:103D6000696F6E207375636365737366756C200A83
:103D7000000000001CB500200190002904D001AB18
:103D80006A46074800F044F8C821054800F0F0F9F9
:103D90000199002902D0009800F0EEF91CBD000046
:103DA000C40B070010B500220121182004F0A6FF63
:103DB00000220121192004F0A1FF00F037FB074881
:103DC0000021007804F01EFF0548007804F00AFF87
:103DD000044A0721492004F0A1FF10BD5A0407003E
:103DE0003D050700801A0600F8B505460024204668
:103DF00005E02E5DE700BE403043641CE4B28C4217
:103E0000F7D304F0C1FFF8BD10B504F0CDFF10BD2D
:103E1000F8B51546074601200622C74E1C46022962
:103E200015D033469B78032920D0012936D13F781D
:103E30000221902F6FD06FDC552F6ED072DC232FB4
:103E40006DD063DC212F6BD0222F6AD1ECE0397862
:103E5000E42907D1717B491C7173B7497B780B70DA
:103E60000021F1703C78702C19D01AE03878302895
:103E700001D10020F0703878852801D17978F1726D
:103E8000AE2806D17878A32803D10021184604F083
:103E900031FF3878922801D178783074F8BD79787C
:103EA000B1737D2C02D0742C22D023E07978F17389
:103EB000737C032B06D0012B0FD0022B11D0032BC8
:103EC00004D017E0012904D0032904D007290CD01D
:103ED00010E0F2730EE0072108E007290AD109215A
:103EE00004E0072906D1082100E01021F17301E068
:103EF00079787174EA2C01D17978B17139789B297C
:103F0000CCD179780229C9D1F070F8BD302F79D0A1
:103F1000522F42D19DE0B5E011E09FE002E08DE03C
:103F20007FE03AE0722F4BD004DC602F23D0612F6A
:103F300033D13DE0752F4FD0852F2ED191E0042352
:103F4000B12F3AD00CDCA42F73D004DC922F71D0A7
:103F5000A32F22D1AFE0A52F6DD0AF2F1DD1B3E09D
:103F6000E42F69D0F12F68D07349F52F097B6FD00A
:103F7000F62F12D1C4E00121184604F0BBFE70797F
:103F8000002805D0002070707071F0706B480CE054
:103F90007078002806D00020707067481C302860B8
:103FA000C82096E00020707065482860102090E0DE
:103FB00061482C302860B8208BE05F48123044E024
:103FC0005F48B27B23215D304901032A3DD0052A99
:103FD0003BD0132A39D0F8BDF07B4721C900012816
:103FE00011D0022811D0032811D0052811D006289D
:103FF00011D0072811D0FF21213108280FD0514AB4
:104000002A6023E01FE050481FE050481DE0504860
:104010001BE0504819E0504817E0504815E0504860
:1040200013E04749493953E04548233828600520C3
:104030004FE043E02BE044E049E04CE040481030E2
:1040400028600B2045E03E48423828602160F8BDDA
:1040500044E03B483E38286003203AE0384948397C
:1040600036E0F17A002907D01C20022907D0202948
:10407000EDD1334937312BE03149473928E0304918
:104080001B3125E02E48533028600A2021E0307C87
:10409000F02808D00A2809D01528D8D128483B385C
:1040A00028602360D3E726484038CEE724481E38EE
:1040B00028602260CBE722483738F1E720483338C0
:1040C000EEE71F482F38EBE71D482B38E8E71A4981
:1040D00029602060BBE71A482738E1E7002906D0AD
:1040E000012907D0022908D015494339F0E71449BE
:1040F0004639EDE712494539EAE711494439E7E71E
:1041000000290FD0012910D0022911D00C48801F9E
:104110002860491CC8B222603073032897D9002058
:10412000307394E706481838F2E705481238EFE78D
:1041300003480C38ECE70000580407001CE80100B5
:10414000CFD30100FCE601008CD80100C4DA0100E5
:10415000FCDC0100A4E3010034DF01006CE101009C
:10416000DCE501000149002088707047F803070072
:1041700010B504F097FE10BD10B504F041FE10BD5F
:10418000F0B50E46A64989B00025CD71F1792C46CF
:10419000102902D90021084601E0002011E0C200E8
:1041A000B25C12091201202A01D0102A03D1641C2A
:1041B0006D1CE4B2EDB2302A01D1641CE4B2401CA3
:1041C000C0B24A1C03929042E9D3002C01D0641E75
:1041D000E4B2002007460890ABE0F900705C0009EB
:1041E0000001202804D0102802D030284DD09EE0B5
:1041F0008919CB781807020D88781B0902430879C2
:10420000000118434B235B01181A05904878872159
:10421000000904901003C900FBF798FF814907903B
:10422000884201D90846079005984B2100034901AF
:10423000FBF78CFF7B49884200D9084604998B0024
:10424000089984330A0176498B54079B51181B093E
:1042500002094B708A70079A00071201000F02438F
:10426000CA7008200871487120208871CC71042020
:10427000087283204872641E022088720020C8726F
:1042800008734873E4B288734CE088190690C278CA
:1042900083781107090D1943037912091B01134390
:1042A000614AD21A059240780009049008038721D8
:1042B000C900FBF74BFF5B490790884201D90846CC
:1042C000079005984B2100034901FBF73FFF554933
:1042D000884200D908460499514B8A000899C43293
:1042E00009015A54079AC91812094A7002098A70BA
:1042F000079A00071201000F0243CA7008200871D4
:1043000048712020887106983A01C079C87104204C
:1043100008728320487200208872C872087348733C
:104320008873D118C8730898401CC0B208907F1CCD
:10433000FFB20398874200D24FE7394C1C3C002D56
:104340001ED0A07900281BD0277A627A0020C300F3
:104350009B191979DB7809011B090B43FF21F53102
:104360008B4208D2BD4202D9E3795B1CE371E37949
:10437000012B00D90122401CC0B20A28E7D3627287
:10438000E0780127002838D0002D3BD12448C2789E
:10439000417813090901C918E182807812070001E8
:1043A000120F8018A0822279921F362A1ED23278EC
:1043B0001209032A1AD1628B914201D9891A00E0AD
:1043C000511A6183218B884201D9401A00E0081AF2
:1043D0002083618BFF206930814207D2218B81428B
:1043E00004D267710021A07804F084FCE08A608325
:1043F000A08A20830020207101E0002D02D100203E
:104400006072E0712572E078002805D167706071F4
:104410000146A07804F06EFC042009B0F0BD000055
:1044200074040700FF0F0000E808000010B50A4CF4
:104430000121207804F0E6FBC82000F0BDFC00213B
:10444000207804F057FCC82000F0B6FC0121207849
:1044500004F050FC10BD00003C050700014901209C
:1044600048707047F803070010B5FEF717FFFEF716
:1044700007FF234C0121207804F03CFC052000F0CC
:104480008FFC0021207804F035FC0A2000F088FC25
:104490000121207804F02EFC052000F081FC03218E
:1044A0001848FFF7B1FC04F08DFC0028FBD00A206F
:1044B00000F076FC134803211230FFF7A5FC04F04E
:1044C00081FC0028FBD0052000F06AFC0D48032188
:1044D0000C38FFF799FC04F075FC0028FBD0052090
:1044E00000F05EFC074803210938FFF78DFC04F05B
:1044F00069FC0028FBD0052000F052FC10BD000034
:104500003C0507000C04070010B504F05BFC002814
:1045100012D00A4C0A496079097888420CD2207876
:10452000002803D005F0D0FA00202070054800785C
:10453000012801D1FCF78CFC10BD0000F803070036
:104540002CE80100D6010700F8B54C4D2879002869
:1045500005D0687800264A4F002808D102E0FFF70E
:10456000D3FFF8BD387804F013FB0028F9D1454C8F
:104570006E702823444A01212068FFF735FC04F0BF
:1045800021FC0028FBD0022000F00AFC3E48017804
:10459000F32903D04178FF290AD012E0FFF764FF26
:1045A000052000F0FDFB6522D20038A139A061E0B2
:1045B0008178FF2905D1C178FF2902D10179FF292E
:1045C0000BD0044608300090387804F0E1FA002857
:1045D0000CD02078F32836D03BE0FFF745FF0A20C7
:1045E00000F0DEFB334A29A133A043E0254808232D
:1045F0000068254A0121FFF7F7FB04F0E3FB0028E0
:10460000FBD0642000F0D8FBE07900280ED0C00673
:10461000030E1C4801210068009AFFF7E5FB04F037
:10462000D1FB0028FBD0642000F0C6FB2078F328E3
:10463000CAD1FFF719FF0A2000F0B2FB1D4A13A1EF
:10464000163226A016E06078022802D1A078002851
:104650000AD00120E8710B480B49826AA879FFF75C
:104660008FFDAE71EE70F8BDFFF7FEFE114A07A197
:10467000203222A0FCF7A6FBF8BD0000F8030700DB
:104680003D05070048050700FC0A07007461755FD7
:104690006C6F67005B25735D20282530346429200A
:1046A00054502073797374656D207265736574203E
:1046B000300A0000310300005B25735D202825309F
:1046C0003464292054502073797374656D207265A9
:1046D00073657420666620300A0000005B25735DF8
:1046E0002028253034642920545020737973746550
:1046F0006D20726573657420310A00005B25735D5F
:10470000202825303464292054502073797374652F
:104710006D20726573657420320A000070B5044C18
:10472000002525716571FFF7EFFE657070BD000013
:10473000F803070010B5074805F0D2F9012005F08D
:10474000CAF9E120400205F00FFA012005F01AFA3B
:1047500010BD000000B4C4040FB4F0B589B0E04C43
:10476000207B00280AD0DE22DEA1E1A0FCF72AFB94
:10477000002009B0F0BC08BC04B0184710A8017BA9
:10478000807B002901D1002802D00121217201E0A3
:104790000021217210A9227A497B07918721C90043
:1047A000002A7ED0012807D0032805D0109A0E9940
:1047B000914224D20E9A23E0109B0F9A9A4201D282
:1047C0000F9A00E0109A8A4206D80F9A10998A42EE
:1047D00001D20F9900E01099119B0E9A9A4201D2D2
:1047E0000E9B00E0119B05221202934225D8119BDB
:1047F0000E9A9A4201D20E9A1FE0119A1DE0109A69
:10480000192149018A4206D8109A0E99914201D283
:104810000E9900E01099119B0F9A9A4201D20F9BBA
:1048200000E0119B6D221201934206D8119B0F9A52
:104830009A4201D20F9A00E0119ACB179B0F591898
:1048400089088900D3179B0F9A18920892004B0091
:10485000CB18DD176D0FEB18DD080323ED005B07A8
:104860004B4301D0082300E00023EB181E4601252E
:1048700056432D05AE4204D8002802D107980028DF
:1048800003D00120607202E00BE0002060729448C7
:104890002038C160026143610021C1610562017677
:1048A000D1E00E9A1098824201D20E9800E0109842
:1048B0008721C900884201D90F4606E00E99109859
:1048C000814201D20E9F00E0109F11990F988842FB
:1048D00001D20F9800E01198904A904201D91046F9
:1048E00006E011990F98884201D20F9800E01198C4
:1048F00002907B4820384068A030407D032804D0D7
:10490000022849D00A2863D06DE00F98FBF7F0FE2B
:1049100006900546049005910E4603911198FBF709
:10492000E7FE2A463346FBF759FE06F099F80246A1
:104930000B4603990498FBF7E9FD05460E468720D0
:10494000C000874214D20E98B84211D90699059832
:10495000019000910E98FBF7CBFE2A463346FBF7F9
:10496000D5FD019B009AFBF739FEFBF721FF0746B7
:1049700011990F98884236D90022694B2846314652
:10498000FBF748FF02D22846314601E00020644987
:10499000FBF70EFF029026E08720C000874209D275
:1049A00010990E98884205D910990E98401A41081E
:1049B00010980F180F991198814214D911990F98D6
:1049C000401A40084118914200D3114602910AE072
:1049D00087270E98FF00B84200D80E9F0F9890428C
:1049E00000D80F9A0292F817800FC0198008800033
:1049F0000299CA17920F51188A0892004100411873
:104A0000CB175B0F5918CB080321DB004907414343
:104A100001D0082100E000215B181946012551430F
:104A20006D05A94202D80799002902D001216172BF
:104A300001E0002161722A492039C8600A614B6196
:104A40000020C8610876264A203A5068A030407F8E
:104A5000012842D110990E98884201D20E9900E0A7
:104A600010992D200001814206D810990E98884295
:104A700001D20E9800E01098119B0F99994201D233
:104A80000F9B00E0119B7921C9008B4206D8119B36
:104A90000F99994201D20F9900E01199C3179B0F0A
:104AA000181880088000CB179B0F59188B089B00A3
:104AB00041004118CD176D0F6918CD080321ED0095
:104AC0004907414301D0082100E000216918002571
:104AD0006572D060136151611576012049E60000CE
:104AE0002C11070068616C5F7673796E63000000BB
:104AF0005B25735D20282530346429207761726935
:104B00006E6720212066622073657474696E672069
:104B10006279206D616E75616C0A0000140A0000F4
:104B20000028A440F8B54A002B4B520DD6182B4A4A
:104B30000C460546142E2BDA002E12DA284BFBF712
:104B400033FC00221346FBF7F9FF40D2002C03DAB6
:104B50000124E40700253AE02046284337D0214CC1
:104B600014E0214F0B46F7403B402B4331D01C4B08
:104B7000FBF71AFC00221346FBF7E0FF27D2002CBC
:104B800003DD01200005F0400419BC4300251EE0B0
:104B9000332E1EDC33460027143BFF43DF403842F0
:104BA00017D00F4BFBF7AAFC00221346FBF7C6FFFA
:104BB0000DD2002C0ADD142E0CD03420811B0120D4
:104BC00088404019A84200D2641C0546BD432146D6
:104BD0002846F8BD641CF9E701FCFFFF9C750088BE
:104BE0003CE4377E0000F03FFFFF0F000FB4079951
:104BF000009888420BD108990198884207D10999F9
:104C00000298884203D10A990398884202D0002072
:104C100004B070470120FBE738B56424154D21E04E
:104C20000821284601F087FF002801D0012038BD67
:104C300028684007800F15D00F48406900902B6806
:104C40000E4A0FA111A0FCF7BDF8284601F009FF9C
:104C50000221284601F00AFF0421284601F006FF40
:104C6000002038BD2146641EE4B20029D8D10020BE
:104C700038BD000000200040002100405302000029
:104C800068616C5F7673796E630000006572726FA5
:104C900072205B25735D20282530346429206572DD
:104CA000205B25785D5B25785D200A0030B51349CF
:104CB000C87B0A7B904201D1002030BD887BFF2257
:104CC00015320F4B5043C01802461432C2608A7B23
:104CD000FF2515356A43D2180124FF320132D474FE
:104CE0000B7B8A7B5B1E9A4202D100228A7301E011
:104CF000521C8A73CA7B521CCA7330BD842A0700B7
:104D0000641A070004480F21017300214173817365
:104D1000C173012070470000842A07000E48C17B40
:104D2000002910D0417BFF23153359430B4B002240
:104D3000C918FF310131CA74037B417B5B1E994264
:104D400003D1427303E000207047491C4173C17BCB
:104D5000491EC17301207047842A0700641A0700A6
:104D60000648C17B002906D0407BFF21153148430E
:104D7000034940187047002070470000842A07004C
:104D8000641A07000549C0000A5C012A04D14018D2
:104D900040684168002900D1002070474411070095
:104DA00010B5044603E07D20C00000F005F8204661
:104DB000641E0028F7D110BD0021022800D27047E0
:104DC00005E0082100BF0A46491E002AFBD1024621
:104DD000401E002AF5D100BFF1E7000030B50120E8
:104DE0000A4D297802290DD30948C0698003840F30
:104DF0000120001BC0B201F0B3FF2878001903287E
:104E000001D0012030BD002030BD0000580A07004D
:104E1000008800400148006870470000C00A070091
:104E200010B50D4C204600F0DBFE0C4A68212046F0
:104E300000F0ECFE094A6021121D204600F0E6FE5B
:104E4000064A38210832204600F0E0FE00201121F9
:104E50000903C860012010BD00900040C00A07008F
:104E600010B51E4A1E4B112491682403994216D195
:104E7000017D00290CD12021095C002908D1817D08
:104E8000012905D0032903D0BD21095C002906D0E2
:104E9000FF200230E06013A0FCF776FAFEE75168CD
:104EA0000A0CFF2A0DD92D2302685B019A4208D310
:104EB0004068AF221201904203D30804000F0F286C
:104EC00001D0012010BD56220AA10EA0FBF77AFFE7
:104ED000FF200430E060002010BD0000C00A070081
:104EE0000368FFFF33363820686172646661756C51
:104EF00074210A006472765F636869705F696E6628
:104F00006F0000006572726F72205B25735D202850
:104F1000253034642920334B212068617264666136
:104F2000756C740A0000000011200003C16800299C
:104F300001D10149C16070475A5A000070B50A2872
:104F400001D9002070BD0F4D00242C6001467D204A
:104F5000C000FBF7FBF80146A868FBF7F7F80A4921
:104F6000401E88420BD80949486109480723C26995
:104F70001202120A4D042A43C2618C610B610120A6
:104F800070BD00008C050700FFFFFF0000E000E09F
:104F900004ED00E010B5FFF743FF10BD0249C86003
:104FA0000020C860704700000080004003494A6844
:104FB0005208520002434A607047000000800040DF
:104FC0008000034A1168042399430143116070472C
:104FD000008000400122064B8240002903D09868DF
:104FE000104398607047986890439860704700003D
:104FF000008000404005034A116893019943014332
:1050000011607047008000404002044A5168072345
:105010005B029943014351607047000000800040EB
:105020000005034A11685301994301431160704719
:1050300000800040C000034A51680823994301439F
:1050400051607047008000400002034A11689315C8
:105050009943014311607047008000400001034AFA
:1050600051683023994301435160704700800040EC
:10507000C001034A5168802399430143516070473E
:1050800000800040C002034A1168D31499430143D1
:1050900011607047008000400002034A5168931578
:1050A0009943014351607047008000400003034A68
:1050B00011689314994301431160704700800040C8
:1050C0008004034A1168D30099430143116070477B
:1050D000008000400004044A116801231B04994326
:1050E00001431160704700000080004001218140B1
:1050F0000348C2680A43C260C2688A43C2607047FC
:10510000008000408001034A5168402399430143D5
:1051100051607047008000408001034A1168C0233D
:105120009943014311607047008000408002034AA8
:1051300011681315994301431160704700800040C6
:1051400010B51207120F436889008A401343436069
:10515000072001F0F1FD10BD014680310A774B7741
:105160000021416001609100014A505070470000E9
:10517000700F07001422514308188168490849003C
:10518000816070471422514308188168012211433D
:105190008160704710B514225143081881680A22B3
:1051A000114381600121072001F028FE0149802080
:1051B000086010BD00E100E000688900C8400007F9
:1051C000000F7047F1B582B00026072001903AE049
:1051D0001F49B0000C58002C33D025468035297F5C
:1051E0000298FFF7E9FF0090009880070CD5297F0F
:1051F00002220298FFF7A4FF2768002F04D00223A1
:10520000012220466168B8470098400704D5297FED
:1052100004220298FFF794FF009800070CD5297F1D
:1052200008220298FFF78CFF2768002F04D008237C
:10523000002220466168B847297F01220298FFF7C3
:105240007FFF761CF6B201988642C1D3FEBD0000F6
:10525000700F070030B5039C1425694308180261DC
:105260004361C46030BD30B505460B46144619464F
:105270002846FFF77FFF14214B435819846130BD46
:10528000016042607047000030B505460C46294673
:105290000D48FFF7E8FF142045430B4810218A0210
:1052A0002818022C08D0012C05D183688B43836019
:1052B00081689143816030BD83680B43836081685E
:1052C0009143816030BD00000054004078B500215A
:1052D00000913A21425CD308D4011B194418667826
:1052E000B5096D015B196D462B705207920FB50021
:1052F00052196D466A7043546270891C5829E9DB63
:1053000078BD8030016A4908490001627047000099
:10531000FFB581B00D4617461E46134C204600F0DF
:105320005FFC6A463821204600F070FC0F49009867
:10533000884208D1FF20023011210903C8600CA067
:10534000FCF722F8FEE70E4CFA00521CB0000243B4
:10535000280402432020024301988030016AA143BF
:105360001143016205B0F0BD009000400368FFFFEB
:1053700064736320686172646661756C74210A00ED
:105380002D0007008030006A4003400F704710B5C1
:10539000602A01D2002010BD034600228C589C5088
:1053A000121D602AFADB8030016A0122D207114304
:1053B0000162012010BD0000FFB585B00E9F0F9D5A
:1053C0000E4614462846FBF78CF9384A014610462B
:1053D000FAF7A0FF03903846FBF783F901463348FC
:1053E000FAF798FF01460398FAF794FF3049FAF765
:1053F00054FF04902146059800F080F80290214661
:10540000059800F0A3F801902846FBF76AF9274DAC
:1054100001462846FAF77EFF04463846FBF761F955
:1054200001462846FAF776FF05463046FBF759F95C
:1054300006460898FBF755F907460299FAF72DFF3B
:105440001C49FAF7D1FE2146FAF727FF3146FAF751
:1054500061FF064638462946FAF71FFF0199FAF719
:1054600059FF074639463046FBF7E8F90FD239466F
:105470003046049CFAF709FF2946FAF74BFF21460C
:10548000FAF7B2FE8121C905FAF7AEFE04E08121E8
:10549000C9050498FAF7A8FEFBF7A8F90022064B05
:1054A000FAF782FFFBF784F909B0F0BD286B6E4E66
:1054B0000000A0410000C0400000E03F10B50424FF
:1054C000002809D0022001F037FC0121022001F060
:1054D00095FC0948046010BD022001F02DFC00215C
:1054E000022001F08BFC044880300460BFF34F8F32
:1054F000BFF36F8F10BD000000E100E000B5024671
:10550000002902D07F20C00500BD0C481300FBF726
:1055100074FF0B07080B07070D0F0807071107009B
:10552000F2E70120800700BD054800BD054800BD29
:10553000054800BDFF20800500BD00000000404080
:105540000000104014AE574000009040002901D0E8
:10555000044870470A2802D07F20C0057047012008
:10556000800770470000C0404069C007C00F704707
:105570004069000C70470122C11DF9310A604A6080
:105580004260704730B5039D8468E408E400491E1A
:105590000C4304210C43846091005A0011432943B9
:1055A000016130BD01238B400321090240180361D2
:1055B000426170474250704710B50124A40200199F
:1055C00001604260836010BD70B504460D46FFF770
:1055D00021FCC100302000290CDA002D06D0012D5D
:1055E00003D1A16881431031A16070BDA16801435E
:1055F000A16070BD002D06D0012DFAD1A1688143B4
:105600002031A16070BDA1688143A16070BD0323FA
:105610001B02C3185960FF30FF300230002A04D04B
:10562000416C0122114341647047416C49084900B3
:1056300041647047F7B5084614463949FAF786FDC4
:1056400001F038F90746022501F0E6F80646009811
:1056500001F0E4F9B87944214006020E009801F007
:10566000EBF9FF2E0BD04D222021009801F0E4F938
:105670007007C20E921C2121009801F0DDF98B23E6
:105680001B222221009801F0E1F9002C3FD0FFF706
:10569000C1FBC0001CD5E00704D0012255210098B1
:1056A00001F0CAF9A00704D501228521009801F074
:1056B000C3F9600704D501229521009801F0BCF9D7
:1056C000200721D501224521009801F0B5F91BE002
:1056D000E00704D001224521009801F0ADF9A007B0
:1056E00004D501225521009801F0A6F9600704D5E0
:1056F00001228521009801F09FF9200704D501229D
:105700009521009801F098F9E00600D50325EAB24A
:105710003521009801F090F9009801F085F9FEBD5F
:1057200040420F000022C11DF9310A604A60426008
:10573000704710B5029C92010A4319020A432104E2
:105740000A43C26610BD0FB452000A436946097B82
:1057500009020A436946497B49020A436946897B33
:1057600089020A436946C97BC9020A436946097C22
:1057700009030A436946497C49030A436946897C0F
:1057800089030A436946C97C09040A436946097DBD
:1057900049040A436946497D89040A436946897D6B
:1057A000C9040A436946C97D09060A43826604B0F2
:1057B000704701677047002904D0C16A0122114374
:1057C000C1627047C16A49084900C16270478030B0
:1057D00041648264704712040A4382617047C16069
:1057E000190211430161704707B56B461A7999791F
:1057F000520011435A79DB799200DB001A431143BE
:105800006B461A7A1201114341610EBD4166704721
:10581000406F70474163704702228030002903D0F7
:10582000416911434161704741699143416170474A
:105830008030002904D04169012211434161704741
:10584000416949084900416170471202491E0A43F3
:105850008030426270478030416A8907890F491C55
:10586000026BD20709D0012909D002290BD00329E4
:1058700011D0042918D00020704700207047006B19
:10588000C006C00F7047006B9021084201D0012074
:10589000704700207047006B29210901084201D0A0
:1058A0000120704700207047006BA92109010842C0
:1058B00001D0012070470020704700B580300B00F8
:1058C000FBF79BFD0504080C10141800006B400743
:1058D000C00F00BD006BC006C00F00BD006B00060E
:1058E000C00F00BD006B8005C00F00BD006B000540
:1058F000C00F00BD002000BDF3B583B008465021A5
:105900000A2250434F30FAF721FC441E601C5021FC
:1059100048430A21FAF71AFC0290029800F0CAFFE5
:105920000190E506ED0EE005070F8037029800F0C4
:1059300091FF044600F070FF0646039801F00AFB51
:105940000020FFF7C7FB0020FFF7BAFB039801F028
:10595000FCFA0198442180794006020E039801F078
:1059600015FB802302221421039801F018FB2C223E
:105970001521039801F00AFB90221621039801F0EB
:1059800005FB30221921039801F000FB09221721A1
:10599000039801F0FBFA3B462A461821039801F0D0
:1059A000FEFA2279C02002431221039801F0EEFA98
:1059B000A078C10060794000014380200143CAB251
:1059C0001021039801F0E2FAE2781121039801F026
:1059D000DDFAFF2E0CD0B006440F4D222021039893
:1059E00001F0D4FAA200921C2121039801F0CEFA12
:1059F0000021039801F0DDFA039801F0B9FA02984A
:105A000005B0F0BD10B5CC788B78240423438030EA
:105A100083610B7949791B0409060B431343C36166
:105A200010BD014601204860704770B504AC70CCD1
:105A300092000A43E1000A4329010A4371000A4324
:105A4000C262036370BD01229203002903D0816BFF
:105A5000114381637047816B914381637047826812
:105A6000120A12020A4382607047000010B508242F
:105A7000002806D0094804600121032001F0BEF986
:105A800010BD0021032001F0B9F904488030046002
:105A9000BFF34F8FBFF36F8F10BD000000E100E038
:105AA0008268FF231B029A4309020A4382607047FF
:105AB000C1630264436470470FB409990165059995
:105AC00081640699C16401994165029981650499CF
:105AD000C1650399016604B0704701460020486023
:105AE00070470FB40199029A090411438167039921
:105AF000C167803004990160059941600699816011
:105B00000799C16004B070470FB5826B920892008C
:105B10000A43826369460A7AFF210131002A03D0D1
:105B2000826B0A43826302E0826B8A438263694626
:105B30004A7A01214902002A03D0826B0A43826318
:105B400002E0826B8A43826369468A7A0121890274
:105B5000002A03D0826B0A43826302E0826B8A438D
:105B600082636946CA7A0121C902002A03D0826B86
:105B70000A43826302E0826B8A43826369460A7B3E
:105B800001210903002A03D0826B0A43826302E0E9
:105B9000826B8A43826369464A7B01214903002A5A
:105BA00003D0826B0A4382630FBD826B8A43826398
:105BB0000FBD1022002903D0816B11438163704710
:105BC000816B9143816370470122D203002903D086
:105BD000816B114381637047816B9143816370478F
:105BE00000B5034600201860184600F009F89868D0
:105BF000032109040843986098688007FCD100BD20
:105C000041680322120411434160704710B50346F6
:105C1000144658684906C009C001490E0843586037
:105C20000121184600F00BF898688003FCD5D8686D
:105C300020609868012149040843986010BD00293C
:105C400004D00168012211430160704701684908CE
:105C50004900016070470000044909680122824040
:105C6000114201D001207047002070474070004071
:105C70000149086070470000980507001838034B79
:105C8000C0001950C0184260704700008C0F070018
:105C900070B50446E006C00E01258540002908D0F5
:105CA000002C01DB0A4805600121204601F0A6F81E
:105CB00070BD0021204601F0A1F8002CF8DB04485B
:105CC00080300560BFF34F8FBFF36F8F70BD000052
:105CD00000E100E00122064B8240002903D0186A4F
:105CE000104318627047186A9043186270470000AA
:105CF00000700040024A136883430B4313607047EF
:105D000000700040024A536883430B43536070475E
:105D100000700040024A936883430B4393607047CE
:105D200000700040024AD36883430B43D36070473E
:105D3000007000400122064B8240002903D05868C1
:105D4000104358607047586890435860704700008F
:105D50004070004070B51E4601252C468C40491C01
:105D60008D4047490300FBF748FB080518132B3EFD
:105D700051647713002A03D008692043086102E0C8
:105D80000869A0430861002E03D008692843086110
:105D900070BD0869A843086170BD002A03D0486936
:105DA0002043486102E04869A0434861002E03D0C7
:105DB00048692843486170BD4869A843486170BD7F
:105DC000002A03D0C8692043C86102E0C869A04323
:105DD000C861002E03D0C8692843C86170BDC86976
:105DE000A843C86170BD002A03D0086A2043086236
:105DF00002E0086AA0430862002E03D0086A284324
:105E0000086270BD086AA843086270BD002A03D00A
:105E1000486A2043486202E0486AA0434862002E74
:105E200003D0486A2843486270BD486AA843486264
:105E300070BD002A03D0886A2043886202E0886A25
:105E4000A0438862002E03D0886A2843886270BD10
:105E5000886AA843886270BD002A03D0C86A2043BC
:105E6000C86202E0C86AA043C862002E03D0C86AB4
:105E70002843C86270BDC86AA843C86270BD0000EC
:105E8000407000408030017F01290AD00748084A4D
:105E9000012908D05268022B07D1002A05D0002121
:105EA00010470448F3E71268F5E7704700500040D8
:105EB0009C050700004C0040F0B58E4694462349EF
:105EC000884201D1012400E003241F2201468031D1
:105ED000CA6000270F611E4B996802221143996026
:105EE000142122464A431B4953189F601A4A1669D7
:105EF0008025AE431661A4000F22A2404A60174AD3
:105F000001211560FF2281329A606246012A03D086
:105F1000022A06D00420F0BD9A68114C22409A60F3
:105F200007E09A68102422439A609A68A402A24368
:105F30009A609A687446240322439A60103018616C
:105F40005F61DF6099610020F0BD0000004C0040FF
:105F500000800040005400400088004080E200E0E3
:105F6000EFBFFFFF8030002904D081680122114378
:105F7000816070478168490849008160704702224A
:105F80008030002903D081681143816070478168A7
:105F9000914381607047000010B515490300FBF77D
:105FA0002CFA0B07090B0D0F11131715191B1C00E9
:105FB000086812E0486810E088680EE0C8680CE0E5
:105FC00008690AE0486908E0886906E0086A04E0B0
:105FD000C86902E0486A00E0886A0648016901224F
:105FE000D203914301610F20FBF714FA10BD0000AA
:105FF00040500040008800400249CA6A0243CA6219
:10600000704700004050004070B50A4C616901259E
:10601000ED03A9436161084908632069A843206131
:106020000F20FBF7F7F960692843606103480560BA
:1060300070BD0000008800400050004000E100E01A
:106040000149086070470000A4050700F8B50B4639
:1060500015461C498D4201D2012100E002211A4A55
:106060009468961534439460184EF26A52085200B0
:10607000F2624A000A2B18D000210A431449134C3B
:106080000A43403C226060601048012740300762AC
:10609000104829460068FAF759F8801D4008094958
:1060A0008D4204D26061A06104E01021E5E7E06167
:1060B000206220620020E063A063F06A3843F0624F
:1060C000F8BD0000E0930400008000404050004014
:1060D0006102000094050700FFB581B017461D4618
:1060E000032408260020FFF787FF304600F076FEE5
:1060F000012211462046FFF7C7F80D4E3B460B4ADA
:10610000214630460095FFF7A5F80120FFF774FF00
:1061100021463046FFF736F804482B461038029ADD
:10612000019900F025F805B0F0BD000010500040C6
:1061300000540040F8B505460E460324082000F040
:1061400055FE012202212046FFF79EF82B46074DFF
:10615000054A214628460096FFF77CF82146284646
:10616000FFF710F8F8BD0000105000400054004048
:10617000F0B50024FF2501359B180DE0944206DAA6
:10618000E6000F46F740FEB20661641C04E0066FAD
:10619000B60701D50561641CA342EFD8F0BD00002D
:1061A00010B514490300FBF728F90B07090B0D0F75
:1061B00011131715191B1C00086812E0486810E03D
:1061C00088680EE0C8680CE008690AE0486908E0E1
:1061D000886906E0086A04E0C86902E0486A00E0ED
:1061E000886A054801690214914301610E20FBF79A
:1061F0001DF910BD404C00400088004070B5094CAE
:1062000061692514A9436161074908632069A843AE
:1062100020610E20FBF70AF960692843606103489A
:10622000056070BD00880040004C004000E100E0C7
:106230000549002803D0012803D000207047486B8F
:106240007047886B70470000404C0040014908606F
:1062500070470000A805070000B502460020FFF7C0
:10626000E7FF202803D203480261012000BD00207F
:1062700000BD0000004C004010B5104B104A114CFE
:1062800098420CD111600023012221460E48FEF7EE
:1062900063FF00220D490C48FEF7F2FF10BD51606C
:1062A0000948002303222146A030FEF755FF064887
:1062B00000220649A030FEF7E3FF10BD004C00406D
:1062C0009C05070000540040CC0F0700855E0100CC
:1062D00010B50E4A93688024234393600C4BDA6A0E
:1062E00052085200DA620A290ED00021A42211437A
:1062F000074A403A116090600020D0639063D86AEA
:1063000001210843D86210BD0821EFE7008000405A
:10631000404C004008B503460091034A0121034860
:10632000FEF798FF08BD0000104C004000540040EC
:1063300001238B40002A03D0016819430160704794
:1063400001689943016070478B880A681B041A43EF
:10635000FF30013042608A6882600B8ACA681B0481
:106360001A43C2604A6902618B8B8A691B041A4313
:106370004261096A816170470222002903D00168E5
:10638000114301607047016891430160704707B590
:106390006B461A799979520011435A79DB79920048
:1063A000DB001A4311436B461A7A1201114301664E
:1063B0000EBD0FB405990164069941640899816482
:1063C0000799C16401990165029941650499816544
:1063D0000399C16504B070470422002903D0016805
:1063E00011430160704701689143016070470822C2
:1063F000002903D00168114301607047016891438F
:106400000160704712040A43FF3001300260704798
:1064100003B56B465A791979520011439A79DB79A1
:106420009200DB001A431143803081600CBD10B52F
:106430008030446801238B401C434460002A03D011
:1064400081681943816010BD81689943816010BDE6
:1064500001225203002903D001681143016002E0C8
:1064600001689143016001680122920411430160B7
:10647000704712020A4319040A43426370470FB47B
:10648000029A0199120411434162049A0399120479
:106490001143816204B0704701225202002903D0E7
:1064A00001681143016002E00168914301600168E5
:1064B0000122920411430160704710B50022FF30A1
:1064C00001309300CC580462CB588362521C202ABE
:1064D000F7DB10BD12040A43FF300130026570473C
:1064E00010B503460C46104621686268091A184622
:1064F000FFF788FF20692189C008C908C90508433A
:1065000018616069C0085861207B002808D0A06924
:10651000C108A020C15018680121C90208431860B1
:106520001868012189040843186010BD09044160FE
:10653000704712050A430267016801229204114361
:10654000016070470122D204002907D0016811437D
:106550000160016852101143016070470168914366
:106560000160704710B50224002806D00948046075
:106570000121084600F042FC10BD0021012000F07E
:106580003DFC044880300460BFF34F8FBFF36F8F32
:1065900010BD000000E100E003239B058905D20542
:1065A000114302689A430A4302607047002908D0E9
:1065B0000168012211430160016852051143016025
:1065C000704701684908490001607047426801232B
:1065D0008B401A434260704710B51024002809D040
:1065E000042000F0A9FB0121042000F007FC094869
:1065F000046010BD042000F09FFB0021042000F087
:10660000FDFB044880300460BFF34F8FBFF36F8FF2
:1066100010BD000000E100E00168012252041143B6
:1066200001607047406801228A40104201D0012079
:1066300070470020704702680323DB039A43C903B5
:106640000A4302607047026830239A4309010A43F3
:10665000026070478269034B09041A400A43826151
:1066600070470000FFFF00F00268520852000A4322
:106670000260704702680123DB049A43C9040A439D
:106680000260704702680121C9020A430260026881
:106690008A430260704712030A43016A490B4903A7
:1066A000114301627047002A03D042680A434260E6
:1066B000704742688A43426070470000044B0904F7
:1066C00012071143026A9A430A43026270470000AC
:1066D0000000FF1F10B50B24A401490292011143D1
:1066E000DA0111430268A2430A43026010BD026846
:1066F00002239A4349000A430260704710B5084BD1
:106700009A4200D91A4603680424A34389000B4324
:1067100003608169090C09041143816110BD000007
:10672000FF030000C2691203120B09050A43C2618C
:106730007047000000487047300A0700002801D069
:106740000148704701487047B0070700B0050700CF
:10675000002801D00148704701487047B008070081
:10676000B006070000487047B009070010B50146A1
:1067700024220248F9F714FD10BD0000300A07007A
:10678000F0B5002A14D00023144DEE1DF936DA00BE
:106790008458AC501418646857197C608C58B450F5
:1067A00054186468921954605B1C202BEFDB13E0D3
:1067B00000230B4DEE1DF936DA008458AC50141846
:1067C000646857197C608C58B450541864689219E6
:1067D00054605B1C202BEFDB0120F0BDB0070700ED
:1067E000B00507001CB5074906C9019200910021B8
:1067F0006B468A009C588450491C0229F9DB012011
:106800001CBD000030E80100002802D00149002032
:1068100008707047BC0A070038B50C4C2078002877
:1068200011D1FEF7F7FA400008D56A466C210848F6
:10683000FFF7ECF900988006800E20702078002881
:1068400001D11B202070207838BD0000BC0A070051
:10685000009000401549884201D915487047FF2132
:106860002D3188420FD90021114A2A3A06234B4381
:10687000D35A834203D30620414388187047491CEA
:10688000C9B20829F2D30021094A921D06234B43BD
:10689000D35A834203D30620414388187047491CCA
:1068A000C9B20529F2D30248801D7047DC050000FB
:1068B0009AE9010010B51249884201D9114810BD6A
:1068C000FF21693188420AD932213130F9F73EFC83
:1068D0000838C0B20B49C000B039401810BD0021C3
:1068E000084A0832CB00D35A834202D3C80080182A
:1068F00010BD491CC9B21029F4D30248083010BD9C
:10690000DC050000E8E801000168490849000122AF
:10691000114391430160704701230A681B041A4325
:10692000120A12020A600168022291430160704754
:1069300038B504460D460093D2B22946204600F0F1
:106940001AF801236A462946204600F023F838BD8C
:1069500038B5044604980D4669460B704870D2B2AB
:106960002946204600F007F802236A4629462046B9
:1069700000F010F838BD10B503680224234303600B
:10698000E3031A430A600268A2430260086898435E
:10699000086010BD70B50024022508E00668AE430B
:1069A0000660165D0E6006682E430660641C9C42FD
:1069B000F4D370BD0649002804D00869400840009F
:1069C00008617047086901221043086170470000A0
:1069D000408400400449002802D00020086170472C
:1069E00002200861704700004084004008490028E8
:1069F00006D0086A0A1410430862064848627047C5
:106A000005484862086A0122D20390430862704731
:106A1000008400404004C0034001200310B5FF3053
:106A20001930FFF771FF10BD10B50146FF311D3160
:106A3000081FFFF771FF10BD10B513460A46014647
:106A4000FF311D31081FFFF773FF10BD08B500931C
:106A500013460A460146FF311D31081FFFF778FF34
:106A600008BD012181610721016070470160704705
:106A700010B5002814D0052000F05EF9122000F0B7
:106A80005BF90121052000F0B9F90121122000F085
:106A9000B5F90520FAF7F2FC1220FAF7EFFC10BD69
:106AA000052000F049F9122000F046F900210520E8
:106AB00000F0A4F90021122000F0A0F90520FAF757
:106AC000CDFC1220FAF7CAFC10BD0000034B1202E5
:106AD0000A43416C9943114341647047031F00000E
:106AE00000200A498A6812020BD508680006800F48
:106AF000002807D0012807D0054849684906C90F72
:106B0000C84070470348F8E70348F6E700800040B4
:106B100000A3E11100B4C40400C2EB0B406B70474A
:106B20004268006802400A4201D0012070470020FC
:106B30007047806B7047006801228A40104201D084
:106B40000120704700207047026C120C12040A43A7
:106B50000264704712040A430264704701490860E6
:106B600070470000B00A0700014948607047000004
:106B7000B00A070010B5029C92010A4319020A43A9
:106B800021060A43426110BDF0B5FF261C021F0614
:106B9000360215040B00FAF730FC08050F1B2531EF
:106BA0003B47510E016A090A090211430162016A59
:106BB000B14321430162F0BD016AFF2212049143F7
:106BC00029430162016A0902090A39430162F0BDE1
:106BD000416A090A090211434162416AB1432143F2
:106BE0004162F0BD416AFF22120491432943416290
:106BF000416A0902090A39434162F0BD816A090A02
:106C0000090211438162816AB14321438162F0BD6F
:106C1000816AFF221204914329438162816A090239
:106C2000090A39438162F0BDC16A090A09021143A8
:106C3000C162C16AB1432143C162F0BDC16AFF2292
:106C4000120491432943C162C16A0902090A394306
:106C5000C162F0BD10B5029C12020A4319040A4336
:106C600021060A43026310BD002A03D042680A438A
:106C70004260704742688A4342607047426C072313
:106C80001B049A4309040A434264704770B504AC7C
:106C900070CC52000A4399000A43E1000A432901DB
:106CA0000A4371010A43C16B890989011143C16318
:106CB00070BD12040A434263704712040A438263A0
:106CC000704700000649896A0907C90F002905D0E5
:106CD00003494031096A0160042070470020704771
:106CE0000040004070B5012676050E4C02250028B4
:106CF00009D00D4806600121152000F07FF8A0683A
:106D00002843A06070BDA068A843A06000211520A2
:106D100000F074F8044880300660BFF34F8FBFF373
:106D20006F8F70BD006C004000E100E00149002061
:106D3000486170470088004010B500280BDB064A08
:106D4000136901210C468440A3431361C006C00EA1
:106D500081400248016010BD0088004080E200E0F0
:106D60000004044AD16903231B0499430143D16100
:106D7000704700000088004000B5054908700228EF
:106D800001D30321081AC0B2FFF7EAFF00BD0000DB
:106D9000580A07000246183AD2B2182808DB9000B9
:106DA0000322824081400348836993430B438361FC
:106DB00070470000008800400246183AD2B21828F6
:106DC00008DB50000322824081400348C36993439B
:106DD0000B43C361704700000088004002494A6AC3
:106DE00082434A62704700000088004002494A6AB4
:106DF00002434A627047000000880040002807DB19
:106E00000122064B8240002903D058691043586183
:106E100070475869904358617047000000880040EF
:106E200010B50246104600F019F8083251B200229F
:106E3000C2600846FFF780FF10BD00B50A4600F0AB
:106E40000DF8002A04D0416801221143416000BDC1
:106E5000416849084900416000BD000014214843D1
:106E600001490858704700005C0A070000B5FFF7A9
:106E7000F5FF40680007400F00BD000070B50546F3
:106E80002846FFF7CDFF2846142148430B494418F4
:106E9000207C00280BD10021284600F021F8002199
:106EA000284600F041F80021284600F013F8A168B8
:106EB000002901D0E068884770BD00005C0A070027
:106EC00014235843024BC0188160C2607047000011
:106ED0005C0A070000B50A46FFF7C0FF026000BD6C
:106EE00070B50246083254B20830C006C00E012503
:106EF0008540002908D0002C01DB0A4805600121EB
:106F00002046FFF77BFF70BD00212046FFF776FF8C
:106F1000002CF8DB034880300560BFF34F8FBFF3D0
:106F20006F8F70BD00E100E000B50A46FFF796FFE5
:106F3000826000BD00B50A46FFF790FF510042682D
:106F40000E239A430A43426000BD10B5B430FFF7E8
:106F5000DBFC10BD8030016A490849000162016A0A
:106F6000022291430162416B012211434163704748
:106F70008030016A042211430162016A0122114337
:106F80000162016A022211430162704710B5134683
:106F90000A460146B831B430FFF7CAFC10BD08B547
:106FA000009313460A460146B831B430FFF7D0FCCF
:106FB00008BD10B50A460146B831B430FFF7DBFC16
:106FC00010BD01228A4002607047002904D0C168C8
:106FD00001221143C1607047C16849084900C1607E
:106FE0007047000010B50124002809D00020FFF7E9
:106FF000A3FE01210020FFF701FF0948046010BD36
:107000000020FFF799FE00210846FFF7F7FE04482D
:1070100080300460BFF34F8FBFF36F8F10BD00004F
:1070200000E100E0006801228A40104201D0012006
:10703000704700207047000070B5049E059D074C06
:107040004900120411435A041143B2041143EA04E3
:107050001143C268A2430A43C26070BD02000F0020
:107060000149086070470000B80A070001218160EB
:1070700070470FB4029A0199120311438161039979
:10708000C1610599416206998162C16804229143F8
:1070900008AA127892001143C1606A46117C002947
:1070A00003D0079AC9070A43026304B07047002A55
:1070B00003D042680A434260704742688A43426094
:1070C0007047026901239B039A4389030A430261C3
:1070D0007047FF3001300161704730B50B071B0F5F
:1070E0001407240F1025002900DA2B43002A00DAA8
:1070F0002C43190322051143FF300130C16030BD1C
:1071000030B50B071B0F1407240F1025002900DAD8
:107110002B43002A00DA2C43190322051143FF30C8
:107120000130816030BD0000044BC9009202114360
:10713000C2689A430A43C26070470000080C00000E
:1071400007221202801801607047026903231B03A3
:107150009A4309030A43026170470322120280180E
:10716000C161704703221202801801627047120445
:107170000A43D9070A4303210902401802607047F5
:107180000322120280184162704703221202801803
:107190008162704730B5C468F025AC431B011C43C5
:1071A000C46012030A43426130BD00000248016816
:1071B00004221143016070470044004002484168C6
:1071C0004908490041607047004400400248406857
:1071D000C007C00F704700000044004010B50124F4
:1071E0002403002806D00948046001210C20FFF781
:1071F00005FE10BD00210C20FFF700FE0348803083
:107200000460BFF34F8FBFF36F8F10BD00E100E04C
:10721000C16807221143C160704703B585B00122E0
:1072200005A901A802F036FD059807B000BD0000D1
:1072300010B50A4C207D01280DD02046C021A03871
:10724000F8F7C7FF01202075002120462038C162D1
:107250000163803810BD002010BD0000380D07000C
:1072600010B5244981423CD10846A030007D002859
:1072700037D002F05FF8042835D01F48FEF741F8F8
:107280000020FEF71BF90020FFF7F2FB0020FFF7BC
:10729000A9FE0020FFF7A0F900211820FDF79AFEB3
:1072A00000211920FDF796FE00211220FDF792FE25
:1072B00000211420FDF78EFE00211720FDF78AFE25
:1072C00002F04AF8022810D000211620FDF782FEB5
:1072D00075208004FDF762FE042002F0A7F901206A
:1072E00010BD002010BD012010BD65208004FDF7F9
:1072F00055FEF1E7980C07000024004070B50446E5
:107300001C48A04214D1A030007D002810D0FDF709
:1073100027FD014608000DD00869002804D0426806
:10732000002A01D020469047FDF7F8FC012070BDEF
:10733000002070BD1048026881150A4201D0012268
:1073400000E00022002A13D005220C4C02256369BC
:107350002B4201D0012300E00023002B03D1521E59
:10736000D2B2002AF3D1002A02D10122FFF77CFC1D
:10737000002070BD980C0700002000400021004054
:1073800010B50749814209D10846A030007D002888
:1073900004D00448FFF740F9012010BD002010BDC3
:1073A000980C0700000C004010B50749814208D135
:1073B0000846A030007D002803D00448FEF7D8F826
:1073C00010BD002010BD0000980C070000280040F0
:1073D00070B505462248A84230D1A030007D002873
:1073E0002CD0284600F040F8284601F0BBFF284684
:1073F00000F0D2F8284600F0D7F92C462034207847
:10740000184E00281CD0207C617C00024018217D91
:10741000627D09028918002815D0002913D0F8F7D9
:1074200095FE411E012300223046FDF771FF2946DB
:10743000802228313046FDF7AAFF04E0002070BD0D
:107440003046FDF75EFF284600F046FA284600F079
:107450000DF9012002F0EAF8FDF766FD012070BD8C
:10746000980C070000240040F8B5014600240D46A2
:1074700020352A78FF23364E2D33486A002A04D05F
:107480001A46B0421DD9022422E0C822314CA04243
:1074900001D9032405E0304CA04201D9022400E0C8
:1074A00001240F7F072F13D1497C002907D1B04257
:1074B00001D9032403E02949884200D902241A464D
:1074C00006E0264EB04203D9487C002806D00224AC
:1074D0009A4205D10020FDF729FE09E00124F7E7D3
:1074E000C82A31D0FF2265321DA121A0F9F76AFC1C
:1074F0000120FDF7C7FD0020FDF7BAFD012118208E
:10750000FDF768FD01211620FDF764FD0121122021
:10751000FDF760FD01211A20FDF75CFD01211B2014
:10752000FDF758FD01211420FDF754FD012117201E
:10753000FDF750FD01210D20FDF74CFD2978204677
:1075400000F0F8FB0120F8BD0120FDF7EFFDCFE7CB
:10755000008C864700105E5F00CA9A3B0008AF2F80
:1075600068616C5F6473695F72785F6374726C00EA
:107570006572726F72205B25735D2028253034643C
:1075800029206572726F7220636C6B5F7669646329
:1075900020434C4B210A0000F8B504462B48A0427A
:1075A0001ED1A030007D00281AD0FFF799FA0646B8
:1075B000274841683046F8F7C9FD0746002000908B
:1075C000244D0346617F01222846FDF7DBFFFAB216
:1075D000E17F2846FDF7E6FF607C002802D005E049
:1075E0000020F8BD3146204600F088FB628A28461C
:1075F000616AFEF71FF8217E2846FDF7E5FFAD2101
:10760000154A89002846FDF7D5FFA034207F812147
:107610008900002804D0114A2846FDF7CBFF03E07B
:107620000F4A2846FDF7C6FF31460E48F8F78EFD93
:1076300001460D48F8F78AFD014601222846FDF76C
:10764000E6FF0120FDF73AFF0120F8BD980C070086
:107650003004070000280040020600008F070707DB
:107660000101010100CA9A3B00E1F50530B589B07E
:1076700004464B48A04218D1A030007D002814D009
:10768000484D617C2846FEF7EFFF01A801F032FD6E
:10769000607C00280CD0207D002855D001230022DA
:1076A00019462846FFF716F854E0002009B030BD0F
:1076B000207C0300F9F7A1FE050406080A0A24004D
:1076C000002104E0012102E0022100E0032128461C
:1076D000FEF7B1FF207C002814D008A8007800280D
:1076E0001FD0002208212846FEF7D5FF00220821DE
:1076F0002846FEF7E3FF02212846FEF7A4FF29E013
:107700000020D3E701212846FEF79DFF0022042137
:107710002846FEF7C0FF002204212846FEF7CEFFD0
:1077200018E003212846FEF78EFF00220421284698
:10773000FEF7B1FF002204212846FEF7BFFF182103
:107740002846FEF7EFFF05E000231A4619462846B3
:10775000FEF7C0FF092200212846FEF7CFFF0121D6
:107760002846FEF7C4FF08A801782846FEF782FFE6
:10777000A07D01280FD003280DD028460299FEF7DE
:1077800069FF012211042846FEF78DFF0120FEF754
:1077900023FF01208AE728460199FEF75BFFF0E707
:1077A000980C0700000C0040F0B587B0044646482E
:1077B000A04216D1A030007D002812D00020002564
:1077C000002600210691059161684A080492890803
:1077D0000391217F04290BD0052905D0072905D065
:1077E00006E0002007B0F0BD012001E003200126E3
:1077F000274620373978012904D1617C002901D13D
:1078000001210591002300901A4619462F48FFF7E1
:1078100021FA607C00281BD10125207C012806D09C
:1078200002280AD003280ED004280CD010E004222D
:1078300002212648FFF74AF90AE0022201212348E3
:10784000FFF744F904E01A2203212048FFF73EF92C
:10785000207D012803D103211C48FFF70FFA069869
:10786000009502900196194D637C39782846059A57
:10787000FFF70CFA22680021521E2846FFF719FA7A
:1078800062680021521E2846FFF717FA2846039A1D
:107890000499FFF75FF901220D492846FFF7E4F943
:1078A0008034A06B002804D0012211052846FFF780
:1078B000DBF90120FFF7DCF806480078002801D04A
:1078C00001F026FE01208DE7980C07000020004003
:1078D00007C2240030040700F0B58FB00446864884
:1078E000A04210D1A030007D00280CD001200E90C5
:1078F000012601250D90002705A801F0FBFB207F44
:10790000072803D005E000200FB0F0BD08270020B5
:107910000E90A07D012810D003280ED02068059974
:10792000884200D9002660680699884200D900255F
:1079300008A8407C01280BD00CE0206806998842FA
:1079400000D90026606805998842F1D90025EFE743
:1079500000200D903B46694862682168FFF71AFCD9
:10796000607C002806D1082F04D10122114663480B
:10797000FFF7DAFB142208A96846F8F711FC05A9FD
:107980005E4F0EC93846FFF774FB0D9801903346E1
:107990000095002138460E9AFFF74EFBA17D384630
:1079A000FFF7D3FB002E01D0002D4DD1A07D544E0A
:1079B00001284DD003284BD020680599401E491E50
:1079C0000003F8F7C3FBF8F793FE00223346F8F7FD
:1079D000EBFCF8F7EDFE054660680699401E491E6F
:1079E0000003F8F7B3FBF8F783FE00223346F8F7FD
:1079F000DBFCF8F7DDFE0246002329463F48FFF78F
:107A0000B6FB08A8007CFEF799FE049008A8007C4D
:107A1000FEF79EFE074600250498EE008159374880
:107A2000FFF79BFB0498301841683448FFF79AFB36
:107A3000B9593248FFF7A4FBF01941682F48FFF706
:107A4000A4FB6D1C202DE7DB0E98002821D040E020
:107A500020680699401E491E0003F8F777FBF8F7E7
:107A600047FE00223346F8F79FFCF8F7A1FE0546D3
:107A700060680599401E491E0003F8F767FBF8F798
:107A800037FE00223346F8F78FFCF8F791FE0246E6
:107A9000B2E70726194DF643324608212846FFF77C
:107AA0002FFB082231462846FFF717FB03A8FEF7F5
:107AB00099FE28460399FFF70CFB28460499FFF727
:107AC00008FB28460399FFF704FB28460499FFF7B3
:107AD00000FB617D094C2046FFF7F3FA00212046A8
:107AE000FFF72EFB012204212046FFF7E0FA0120D8
:107AF000FFF778FA012007E7980C07000010004014
:107B00000000E03F70B50D4B834207D1A0331B7DD1
:107B1000002B03D0802A03D9002070BD002070BD47
:107B2000002304E0C418CD5C203425725B1C934212
:107B3000F8D32830FDF7CAFB012070BD980C070070
:107B40000FB4FEB50CA8029008A8037B11290AD037
:107B5000122908D0212906D0222904D01A2922D09E
:107B60001C2920D054E000260022022B09D9294AE2
:107B700029A12D48F9F726F90020FEBC08BC04B065
:107B80001847002006E0029C20CC0294C400A540C7
:107B90002A43401C9842F6DB1346009623480A9A73
:107BA000FEF7E8FF34E001200190002408A8007BE4
:107BB00080088446401C864622E00022A4450FD15E
:107BC00098071CD000209F07BF0F06E0029D40CD04
:107BD0000295C500AE403243401C8742F6DC0CE003
:107BE00002980568426812022A4305892D0415434C
:107BF000027B103012062A4302900C480261641C7A
:107C0000A645DADC0198009008480A9AFEF7B2FF10
:107C10000120B2E77F04000068616C5F6473695FF4
:107C200072785F6374726C00C0E90100002000404C
:107C300070B505460C46FEF753FF2146F8F786FA65
:107C4000C2B2E97F0348FDF7ADFC03484460012060
:107C500070BD00000028004030040700F0B589B076
:107C60000E4617461649814227D10846A030007DAE
:107C7000002822D00024E50071591248FFF76DFA60
:107C8000A81941680F48FFF76DFA79590D48FFF7B9
:107C900077FAE81941680B48FFF777FA641C202C43
:107CA000E9DB01A801F026FA08A802783946304637
:107CB000FEF766FD012009B0F0BD0020FBE70000E3
:107CC000980C07000010004010B50A4A82420BD100
:107CD000A032127D002A07D0407C002806D008463A
:107CE00001F0AEFC012010BD002010BD0248FEF7DF
:107CF0002BFFF7E7980C0700002000401CB5044656
:107D0000606AC008019000912020025D617F207FA1
:107D10002368FDF751FB0346A07F002805D0012111
:107D2000E27F0348FDF748FC1CBD0021F8E7000096
:107D30000028004070B502460E46012000240025B0
:107D4000002A1BD0012A1CD0022A02D0032A1CD0F0
:107D50000220FDF7E1F92046FDF7D4F92846FDF7AA
:107D600073F9002E13D00020FDF778F90120FDF7FC
:107D700061F901211920FDF72DF912E001240125F7
:107D8000E7E7022001240125E3E70220E1E70120E3
:107D9000FDF764F90020FDF74DF900211920FDF7EA
:107DA00019F9012070BD000010B50A4981420ED1B9
:107DB0000846A030007D002809D000210648FEF7C3
:107DC00096FC0121002001F049FC012010BD00209B
:107DD00010BD0000980C0700000C004010B50846CC
:107DE000114601F03BFC012010BD000010B50B490D
:107DF000814210D10846A030007D00280BD001211F
:107E00000748FFF7E2F80748FDF7B5FB022001F04D
:107E10000DFC012010BD002010BD0000980C0700D3
:107E2000001000400028004010B50B49814210D1DD
:107E30000846A030007D00280BD000210748FFF73E
:107E4000C4F80748FDF76EFC032001F0EFFB0120AA
:107E500010BD002010BD0000980C0700001000406D
:107E60000028004010B50649814207D1A031097DA4
:107E7000002903D001F046F9012010BD002010BDFB
:107E8000980C0700F0B59DB004460D46A66A6778C9
:107E9000E07814902869F8F724FC0221C943F8F728
:107EA00077FA1590E9681C911598F8F733FA139052
:107EB0003846F8F716FC1B901399F8F7EEF9129074
:107EC0002F6830463946F8F757F97843002900D132
:107ED0000027C019F8F7FAFB024668681A900146B5
:107EE00019901046F8F7D9F9F8F710FC0746304614
:107EF000F8F7F7FB179018901299F8F7CEF916904B
:107F0000F8F774FCFCF70EFEF8F72EFCC01B11907E
:107F10001698109019991798F8F7BFF907467F211E
:107F2000C9051098F8F760F93946F8F7AEF9FF215E
:107F3000C905C84203D30020C0431DB0F0BD11984D
:107F4000002847D01498022844D001200F903046D2
:107F5000F8F7BCFB1A99F8F7A0F92A49F8F744F9A1
:107F600007467F20C0051C99F8F797F905901B98E4
:107F7000049015991898F8F790F90499F8F78DF985
:107F80000599F8F7C7F93946F8F77FF9F8F7BEFB16
:107F90000E90AF6A202106A8F8F71BF9286A0A900C
:107FA000E8690B90A0680690E0680790E06A089086
:107FB0002069099014480A99814208D80B99814296
:107FC00005D81248874202DCC1108E4206DD00202F
:107FD000C043B2E700200F900E90DAE70C4C314618
:107FE00020460E9B0F9AFDF763FD142209A96846EF
:107FF0000597F8F7D5F806A90EC92046FDF75CFDF0
:1080000000209AE700004041FF010000FF3F000010
:108010000004004010B50C462030417C084800297F
:10802000006C06D0A060074860600220206000203D
:1080300010BD7F21C905F8F7D7F8A060F3E700006D
:10804000580D070000004040F0B599B006460C46B8
:1080500000273720855DF06A1890B06AF8F741FB79
:108060001790304640301590007916907078F8F7E8
:1080700038FB1490012D49D0149802906568179828
:108080002946F8F70AF90299F8F744F9F8F7AEFB30
:10809000FCF748FDF8F78CFB089014980290706983
:1080A000F8F71FFB2946F8F7F8F80299F8F732F9C4
:1080B000F8F79CFBFCF736FDF8F77AFB0A9014986A
:1080C0000290B069F8F70DFB2946F8F7E6F8029937
:1080D000F8F720F9F8F78AFBFCF724FDF8F768FBBE
:1080E0000990F168B068326941181898101808189A
:1080F0000F9003200390169800286FD009990A98D2
:10810000411808980818DD3007908FE00120B06012
:10811000F06030611898C01C0F90149D179861682A
:10812000F8F7BBF82946F8F7F5F8F8F75FFBFCF726
:10813000F9FCF8F73DFB08900320039016980028FF
:1081400002D0089DCE3502E0089DFF3557350F98C7
:108150006843F8F7C6FAA168F8F79FF8DC49F8F722
:10816000D9F8F8F743FBFCF7DDFCF8F721FB0646EE
:108170002AE00C96F000FEF79DFB07461598007963
:10818000002807D03879797942180399089840185F
:10819000151807E03879B9784218039908984018FB
:1081A00015186D1D0F9928464843F8F79AFAA168EB
:1081B000F8F773F8C649F8F7ADF8F8F717FBFCF7CE
:1081C000B1FCF8F7F5FA06460C98B042D1D10C98FC
:1081D000BB280CD98F22D200BEA100E01EE0C1A0B6
:1081E0000C9BF8F7EFFD0020C04319B0F0BD0F99CC
:1081F00028464843F8F775FA0290C6493046484386
:10820000F8F76FFA0299F8F785F8A060F00020619E
:1082100027636661A5620F98E06257E109990A98A1
:10822000411808980818FF30573007900F990798A1
:108230004843F8F756FAA168F8F72FF8A449F8F779
:1082400069F8F8F7D3FAFCF76DFCF8F7B1FA0025F6
:1082500034E00546C000FEF72DFB0746159800796F
:1082600000280DD039790A980A18089909984018F9
:10827000797910184118039808180F3007900CE00E
:1082800039790A980A18089909984018B978101885
:10829000411803980818401D07900F990798484304
:1082A000F8F71FFAA168F7F7F8FF8949F8F732F8ED
:1082B000F8F79CFAFCF736FCF8F77AFA8542C8D151
:1082C0000220069005200590B06A049004980930B9
:1082D0000E900898C01EF8F704FA139004992846E7
:1082E000484312900899C91EF7F730FFF8F700FAD3
:1082F000FCF718FCF8F738FA3221F7F73DFF322186
:1083000041430B910798F8F7ECF902900E986843F7
:10831000F8F7E7F90299F7F7FDFFF8F767FAFCF7C6
:1083200001FCF8F745FA0B9988420BD93221F7F78F
:1083300023FF024632204243002900D000E0002003
:1083400010180B900B98C82802D9FF202D300B90E5
:10835000139802900B98F8F7C4F9119001901298B5
:10836000F8F7BFF90199F7F7D5FF0299F7F78DFFF5
:10837000F8F73CFAFCF7D6FBF8F7F6F9002835DDFC
:10838000089A07998A1A0399511A091F88422BDC07
:108390000D950B98A0617079109000281ED0707810
:1083A000F8F79FF9019000901098F8F79AF9616832
:1083B000F7F773FF0099F7F717FF7F21C905F7F764
:1083C00064FF0199F7F7A6FF02902846F8F789F9AC
:1083D0000299F7F709FFF8F7B2F90546BB2D2ED938
:1083E00065610020C04300E76D1C11E00498F8F7B8
:1083F00078F9054611991398F7F74FFF2946F7F7D3
:1084000089FFF8F7F3F9FCF78DFBF8F7D1F905468A
:108410000F98F8F766F9A168F7F73FFF07463D495F
:1084200028464843F8F75DF93946F7F773FFF8F740
:1084300086F90790E800FEF73DFA07464EE70D98EB
:10844000854217D00D950D9DE800FEF733FA0746DB
:108450000F98F8F746F9A168F7F71FFF05462D4971
:108460000D984843F8F73DF92946F7F753FFF8F719
:1084700066F907900F9907984843F8F732F90546CF
:1084800024490D984843F8F72CF92946F7F742FF9D
:10849000A06070780D994843F8F723F96168F7F701
:1084A00039FF069971610599B161E0600D98C000CE
:1084B000206127630D986061089860620998E06107
:1084C0000A9820620798A0620F98E06200208CE66C
:1084D0000024744968616C5F6473695F74785F63DA
:1084E00074726C006572726F72205B25735D202858
:1084F0002530346429206C616E65206279746520B2
:10850000636C6B206F76657220666C6F773A2564BA
:108510000A00000040420F0010B5084C20780128E6
:1085200009D048212046F7F754FE01202070044866
:108530002064204610BD002010BD0000580D07002B
:108540000000704210B5104981421BD10878002804
:1085500018D000211320FCF73DFD00211A20FCF764
:1085600039FD00211B20FCF735FD00211520FCF70B
:1085700031FD0520C004FCF711FD042001F092F844
:10858000012010BD002010BD580D070010B586B0A9
:108590000F4800796946087348738873C873087474
:1085A00048748874C874087548758875C8750599C5
:1085B0000498084C01910090002211462046039B2C
:1085C000FDF7C1F801212046FDF724F906B010BDE2
:1085D000580D0700000400401CB50023064C002283
:1085E0000093114620460193FDF7ADF8034920465C
:1085F0000978FDF70FF91CBD00040040380407009E
:1086000070B58EB00646342101A8F7F7E2FD2B487D
:10861000B04214D10078002811D0304600F052F852
:10862000304600F01DFF01A93046FFF7F3FC01A919
:108630003046FFF709FD3446403401250CE00020A8
:108640000EB070BD2079002801D00020F8E7257118
:1086500001A93046FFF7F8FC0698BB28F2D801A91B
:10866000304600F0E1F9164C05992046FDF744F933
:10867000059001A9304601F047F9304601F024F990
:10868000304600F0A9F901A9304600F083F900282E
:1086900001D00020D4E7304600F0D6F9304600F093
:1086A000B3F92046FDF7D7F80028FAD02046FDF7A9
:1086B000B8F9012000F0F6FF0120C1E7580D0700CE
:1086C0000004004010B501211320FCF783FC0121B8
:1086D0001A20FCF77FFC01211B20FCF77BFC012109
:1086E0001520FCF777FC10BD10B50146072000F0FF
:1086F00001FB10BD0FB410B502A8FEF737F8012238
:1087000002210348FDF793FE10BC08BC04B01847D3
:108710000008004010B513460A4601460148FDF71F
:10872000A8FE10BD0008004010B501460148FDF745
:10873000B3FE10BD0008004000B585B00190029165
:10874000039204930498009001A90EC90248FDF712
:1087500096FE05B000BD00000008004070B504465C
:108760001648A0421ED1007800281BD0144D0121CC
:108770002846FDF720F801212846FDF759F8114D4C
:1087800001212846FDF7DEFE2034607C01280BD055
:10879000012211462846FDF7FFFE022000F082FF6D
:1087A000012070BD002070BD01212846FDF750FE5C
:1087B00001212846FDF7FAFEEFE70000580D0700FB
:1087C000000400400008004010B50D49814214D15A
:1087D0000878002811D000210A48FDF7E7FE0020A4
:1087E000FDF7C0FE0020FDF741F90748FDF775F9D8
:1087F000032000F057FF012010BD002010BD000035
:10880000580D07000008004000040040FFB583B089
:1088100004461E460291132C18D0232C16D0052C8A
:1088200014D0152C12D0292C01D0392C1BD12C4F4F
:108830003846FCF7EDFF4007FAD50598800801900F
:1088400005988007800F009000252BE005980028F0
:1088500012D0012809D0022805D173783278204639
:10886000029900F067F907B0F0BD32780023204686
:10887000029900F05FF9F6E700231A4620460299B4
:1088800000F058F9EFE700210022AB009818305CA7
:10889000D700B8400143521C042AF7DB1048FCF70C
:1088A00088FF6D1C01988542EDD3009800280FD0F9
:1088B00000210020AB0005E01A18B25CC500AA40F8
:1088C0001143401C009A9042F6D30548FCF771FF13
:1088D00000232046059A029900F02CF9C3E7000016
:1088E000000400400FB4FEB506460F460BA80190E9
:1088F0000020132E11D0232E0FD0052E0DD0152EB3
:108900000BD0292E01D0392E1ED10025204C204617
:10891000FCF77EFF4007FAD52FE0009008A8027A06
:10892000022A11D800206B4605E001990C78091D38
:1089300001911C54401C9042F7DB68464378027852
:108940003946304600F0F6F8FEBC08BC04B01847C3
:10895000ECB200212D1D08E0019804C80190A00789
:10896000C00E82401143641CE4B2AC4201DA9C4266
:10897000F2D30748FCF71DFF254608A8037A9D425D
:10898000E6DB027A00233946304600F0D3F8DBE715
:1089900000040040F8B504460E4637200C4D015D3A
:1089A00029700C4F3846FCF735FF2878002805D091
:1089B0003846A16AFCF72AFF0020F8BD3146204660
:1089C00000F08CF80028F7D00020C043F8BD00006C
:1089D00038040700000400401CB50A4C81780023CD
:1089E00005222046FCF7FBFE002168460171204667
:1089F000019AFCF7F9FE1C2200212046FCF7EBFE51
:108A00001CBD00000004004010B50020FDF72EF84A
:108A10003F22D20100210348FCF7D9FE0120FDF7D7
:108A200025F810BD0004004070B50C46054D417896
:108A300028222846FCF709FF00222846216BFCF774
:108A4000E1FF70BD0004004030B58BB00546012049
:108A5000214C0090019002460146029000232046DE
:108A6000FCF7E3FF0A212046FCF7F9FF202120460E
:108A7000FDF716F8002104910591069107910891E0
:108A800009910A910091019102910B460A462046F4
:108A90000391FDF726F82879002811D000212046FF
:108AA000FCF789FE00212046FCF7C2FE40352879FC
:108AB00000280ED000212046FCF7AEFE0BB030BDE2
:108AC00001212046FCF777FE01212046FCF7B0FE8D
:108AD000ECE70121EFE70000000400407CB504460C
:108AE0000D4601216846017041708170C1700171AD
:108AF00041710F4EE1783046019B009AFDF704F872
:108B000000213046FCF79FFF00213046FDF75CF85E
:108B100000213046FDF74DF829462046FFF7B2F90F
:108B2000002802D00020C0437CBD00207CBD000096
:108B300000040040FFB581B006460F461D460C4CB0
:108B40002046FCF765FEC007FAD000953A4631464C
:108B50002046039BFCF7EDFD0649C979002905D0A5
:108B600001212046FCF7A9FE0028F9D005B0F0BD90
:108B700000040040980D070010B5044A80008218D8
:108B800002201056FDF784F810BD0000B4D2010099
:108B900010B5FDF761F8002801D0012010BD0020BC
:108BA00010BD0000F8B505460F460D48A9000C1889
:108BB0000226A65700212846FDF78CF86178284642
:108BC00000F068F8E1783046FEF7E4F839463046C0
:108BD000FEF7F2F802202056FEF7AEF8F8BD0000CE
:108BE000B4D2010010B5044600212046FDF772F80A
:108BF0000349A00040184178204600F04BF810BD12
:108C0000B4D2010010B504462046FDF793F80121C7
:108C10002046FDF75FF80449A0004018417820463F
:108C200000F038F810BD0000B4D2010010B5044ABD
:108C300080008218022010560022FDF71FF810BD98
:108C4000B4D2010070B5044608461546FDF710F889
:108C50002846FEF791F80125ED05002C09D00C48B7
:108C600005601720FEF768F801211720FEF7C6F807
:108C700070BD00211720FEF7C1F81720FEF75CF841
:108C8000034880300560BFF34F8FBFF36F8F70BD17
:108C900000E100E010B5164A8000125C0720242A8B
:108CA0000AD308D0252A06D0243A5300D21890407F
:108CB0009140FDF737F810BD182A07D3183A530032
:108CC000D21890409140FDF725F810BD0C2A07D32B
:108CD0000C3A5300D21890409140FDF713F810BDA4
:108CE0005300D21890409140FDF704F810BD0000E9
:108CF000B4D2010010B5FDF71DF810BD10B50C463B
:108D000041004118044813460818817840782246EB
:108D1000FDF720F810BD00002CD3010070B505460A
:108D20000E461548824200D20246144CA24200D898
:108D3000144601211820FFF7ADFF01211920FFF78C
:108D4000A9FF224631462846FDF780F90C48FDF779
:108D500077F901204002FDF757F90A4C0222002161
:108D60002046FDF7A9F801212046FDF7FBF8012177
:108D70002046FDF704F970BDA086010040420F00B7
:108D8000D18D01000050004070B5002B07D0054D7B
:108D900000242C70C9B2FDF79FF9204670BD032056
:108DA00070BD00003904070010B5002906D0044A40
:108DB00000241470FDF7BEF9204610BD032010BD3D
:108DC00039040700014800787047000039040700A3
:108DD00010B50548406B800502D504490120087094
:108DE0000020FDF7D9F810BD0050004039040700FD
:108DF000002902D101490120487070473C04070056
:108E000070B506460C46002C0ED0094900254D7061
:108E10000120087001210748FCF7ACF921463046D3
:108E2000FDF778FA284670BD0020C04370BD0000F1
:108E30003C0407000054004070B504460D46032171
:108E40001620FFF727FF03211720FFF723FF2946EE
:108E50002046FDF73DFA0E48FDF7F8F90D48FDF7FD
:108E6000CDF90D4C022200212046FDF725F80B49D3
:108E70002046FDF701FA0220FDF7B8FF0121204648
:108E8000FDF77DF801210648FCF784F970BD00006C
:108E9000C58E010024120000004C0040F18D01003D
:108EA00000540040034A00239370506091600020FA
:108EB000704700003C0407000149C860704700008B
:108EC0003C040700F8B5044600204A494D6B4A4E61
:108ED00069071CD57068002814D0B068002807D036
:108EE000226971680A70491C7160401EB06000E020
:108EF00020693069401C30610120FDF799F9002894
:108F0000EBD103E0F26801203169904701203B4F2B
:108F1000A9062BD50420FDF743F9F268002031693A
:108F20009047386AB061B86A002805D030780028C8
:108F300008D00020307013E02F481430B862304859
:108F400038620EE07069002823D001213846FCF712
:108F500011F9B86A396A7269891A20394018B862F9
:108F6000606D01213846FCF70DF90120A90529D5CE
:108F7000386A70611F48803004680820FDF710F9D6
:108F800070692049002808D0B269101A203808609A
:108F90000FE00020FDF760F9F8BDA00402D4B0692D
:108FA000086006E02001C00E00281FD0B269101A28
:108FB0000860F268022031699047307CB070002070
:108FC000306101200028E7D10A48403041688168BB
:108FD000C16841698169C169416A806A0A490A694F
:108FE000081482430A6109490860F8BDB069203855
:108FF0000860DEE7004C00403C04070000540040DD
:1090000060EA0000AC0507000088004080E200E054
:1090100070B50446607C002817D0224D01212846F7
:10902000FDF722FB092200212846FDF767FB0121FD
:109030002846FDF75CFB207D00280DD0012300228F
:1090400019462846FDF746FB0CE0174A17A11AA05F
:10905000F7F7B8FE002070BD00231A4619462846CF
:10906000FDF738FB2248017A2846FDF703FB20492B
:10907000A07D203901280FD003280DD0096928468A
:10908000FDF7E8FA012211042846FDF70CFB012048
:10909000FDF7A2FA012070BDC9682846FDF7DAFA8B
:1090A000F0E70000000C0040BD06000068616C5F46
:1090B0007673796E630000005B25735D2028253090
:1090C000346429206E6F7420737570706F72742011
:1090D000766964656F206D6F6465207265736F6C6F
:1090E0007574696F6E206368616E6765210A0000A0
:1090F0002C11070010B520220149F7F751F810BDD7
:1091000018110700F0B587B00024674DEE682F698D
:109110008369426901690293019200910FC8FBF7CC
:109120001BFBE868B04202D12869B84200D0012494
:109130005E4E00213046FDF748FF3046FDF796FFB2
:10914000002C6ED0AC786868FEF742F900215848D0
:10915000FDF7CDFA6868A968406848626868A96840
:1091600000680862022C06D0A868FFF749FA686810
:10917000FEF73CFE94E000240026A9682B8ECA6806
:109180009B189BB20693002500230593CB6A9A187F
:10919000CB6BD7188B68096959185118B94200D29E
:1091A0007F1A41484068FEF721FE0121C904414869
:1091B000FDF75CFC012109053E48FDF757FC3A4AE2
:1091C0009168106BC96840183B49496B8842FBD1D4
:1091D00035484068FEF7D4F818E03848844210D18A
:1091E0001E2E1FD0304B9968186BC9684018324941
:1091F0004A6B9042FCD15868FEF7C2F80024761CF6
:10920000B6B2641CA4B20120FBF7D6FD2948006861
:10921000C002E2D5284C606B04901E2E1BD2254E56
:1092200016E037E0264A27A129A0F7F7CBFDF1E7A2
:10923000606B05900598B8420AD1002D08D11E48F0
:1092400040380068800402D43148FCF746FC012510
:1092500030680003ECD50D20C004FBF79FFE124CD4
:10926000A068FFF7CDF96068FFF7D2FEA068FFF7AE
:1092700075FA002D14D1A0680499C06B059A6B464D
:1092800086C30F4A03902B320EA12248069BF7F7A4
:1092900099FD05E06868FEF79BF86868FEF7A6FD93
:1092A000012007B0F0BD00000C11070000100040C5
:1092B000000C00400020004040080040983A0000A8
:1092C0001B07000068616C5F7673796E63000000B5
:1092D0005B25735D20282530346429207761726E08
:1092E000696E6721206E6F742064617461207265FD
:1092F0006365697665642061667465722072657362
:109300006F6C7574696F6E206368616E67650A00C3
:10931000000400404CEA010070B5054C6578A67861
:1093200038212046F6F755FF6570A670012070BD04
:109330000C11070001484078704700000C1107002D
:109340000449086B002803D14868C06840080863D6
:10935000704700000C11070001488078704700003A
:109360000C110700F0B58DB005462846FBF778FDD7
:10937000334C6068A84214D06560A16800291CD0F5
:1093800020311C2203A8F6F70BFF2869AA69696936
:109390006B4607C328460FC8FBF728FC002803D0FC
:1093A00014E000200DB0F0BD2869AA6969696B4618
:1093B00007C30FCDFBF7D0F908E0AA6929696869EE
:1093C0000292009101900FCDFBF7C6F91DA003C8D2
:1093D0000C910B9000201A4E01270BA938360A5C1D
:1093E000D200B754401C0628F9D363688033986ACA
:1093F000002813D0002109E01258D200B7549A6A0D
:1094000015181058C00080194560491C08460C25E5
:1094100068439A6A051D5559002DEDD10020207032
:109420000B490A48C8600B48FDF798FB0A48FDF74E
:109430009BFB0A48FDF714FEFBF764FC0120B1E733
:109440000C1107002A3A3C2C2B3B00004419070062
:10945000501A070091A7010035A80100A9AA010030
:1094600030B58BB029498A68002A02D000200BB0A1
:1094700030BD88604C6801462031002C3BD01C2256
:1094800003A8F6F78DFE2069A26961696B4607C3E0
:109490000C202018017825790B46417809020B43EE
:1094A0008178C07809040B43000603430820201884
:1094B00001780A46417809020A438178C078090494
:1094C0000A432946657900062D022943A5790243FE
:1094D0002D04E07929430006257801432846657864
:1094E0002D022843A578E4782D0428432406204340
:1094F000FBF77CFB08E0016B836B426B6C460EC490
:1095000020300FC8FBF728F90120B0E70C11070045
:109510007FB5002100910191029103910121002862
:109520001DD00120324E6D46431EC200DC00B25CED
:10953000345DA24208D0012A01D0685400E06B5487
:109540000F2904D0491CC9B2401CFF28ECDDC21F02
:10955000F93A40D0274A28A12AA0F7F733FC6846F9
:10956000314C4378027800212046FDF70DFB684618
:10957000C378827801212046FDF706FB68464379CF
:10958000027902212046FDF7FFFA6846C379827905
:1095900003212046FDF7F8FA6846437A027A04214F
:1095A0002046FDF7F1FA6846C37A827A0521204603
:1095B000FDF7EAFA6846437B027B06212046FDF769
:1095C000E3FA6846C37B827B07212046FDF7DCFA7D
:1095D000012004B070BDFF200E2902D304E06854BE
:1095E000491C1029FBDBBAE76946C873B7E70000DE
:1095F00044110700B507000068616C5F7673796EEF
:10960000630000005B25735D202825303464292029
:109610006175746F2066696C746572207761726E13
:10962000696E67200A0000000020004010B5034961
:109630004870042801D1FFF76FFE10BD0C11070020
:1096400010B5054C62685168D2685043F6F77EFD4C
:109650002063012010BD00000C11070070B50C46FE
:109660000E4D002806D06A685168D2685043F6F75C
:109670006DFD286309482030417DA1420CD044751E
:10968000A878022801D101F0EBFA6878022803D10A
:1096900001210348FDF799FC012070BD0C11070062
:1096A0000010004070B504460C4D042C02D0022C72
:1096B00003D010E0FFF730FE0DE02878012808D134
:1096C000A8682030407C012803D100210448FCF721
:1096D000BFFE01F0C5FAAC7070BD00000C110700B0
:1096E0000008004070B50024FDF724F80146054D40
:1096F0002846FCF729FE224607212846FCF718FEDB
:1097000070BD0000000800407CB50D462030417C53
:10971000C47D0E4E3046FCF72FFE21463046FCF746
:109720005BFE00213046FCF762FE10213046FCF75C
:10973000FDFE0021684601713046019AFCF727FEC4
:10974000002229463046FCF7CBFE7CBD00080040D5
:1097500010B5012208210248FCF7EAFD10BD000007
:1097600000080040F0B585B00646B46AF56A08689E
:109770004F68497F01290AD0012103914036844274
:1097800002D1B179002905D00021029104E0002125
:109790000391F3E701210291BD4202D171790029C1
:1097A00002D00021019101E00121019102990029DB
:1097B00004D00199002901D001246AE0B179049113
:1097C00000292ED00499401E611A621E491E504382
:1097D000F6F7BCFC0003611EF6F7B8FCF6F788FF4D
:1097E0000022374BF6F7E0FDF6F7E2FF00907679BE
:1097F000002E25D0A91B781E6A1E491E5043F6F77D
:10980000A5FC0003691EF6F7A1FCF6F771FF002224
:109810002B4BF6F7C9FDF6F7CBFF0746002E21D1FB
:109820001DE0401E0003611EF6F790FCF6F760FF96
:109830000022234BF6F7B8FDF6F7BAFF0090D6E703
:109840007F1E3803691EF6F781FCF6F751FF0022F0
:109850001B4BF6F7A9FDF6F7ABFF0746DEE70498CA
:10986000002809D004980021231AAA1B0846FEF7F5
:1098700063FF0120FEF758FF124C3A46204600993C
:10988000FCF728FEFCF76EFF01462046FCF715FEAC
:1098900000240C4D0A212846039AFCF749FD0421B7
:1098A0002846029AFCF744FD05212846019AFCF758
:1098B0003FFD224606212846FCF73AFD05B0F0BDE3
:1098C0000000E03F0008004010B588B0044668463C
:1098D000FFF710FC69462046FFF744FF2046FFF7DC
:1098E00001FF2046FFF734FF01220C210548FCF759
:1098F0001FFD69462046FFF707FF204600F0C4F829
:1099000008B010BD00080040F0B599B004460D46FF
:1099100020210EA8F6F75DFC60691890A0691790E9
:10992000A06A1690AF693846F6F7DBFE0646C82FE8
:1099300006D90020FBF768FB0020FBF771FB09E06C
:10994000C82F5AD0962F5FD00220FBF75DFB012075
:10995000FBF766FB0020FBF74DFBE86AF6F7C1FE5C
:10996000A968F6F79AFC074645493046F6F795FC94
:109970003946F6F7CFFCF6F739FFFBF7D3F8F6F7E1
:1099800017FF1899411A1798091A1698081A189962
:10999000129117991391169914911590E06A1090ED
:1099A000A0680E90E0680F9020691190142211A910
:1099B0006846F6F7F5FB0EA90EC93248FCF7F9FC2C
:1099C00006A8FFF797FB079906984843F6F789FE24
:1099D000A968F6F762FC2A49F6F79CFCF6F706FF41
:1099E000FBF7A0F8F6F7E4FEF6F77BFE05463146F6
:1099F000F6F724FF0FD228460EE00020FBF704FB09
:109A00000120FBF70DFBA5E70220FBF7FDFA002084
:109A1000FBF706FB9EE73046F6F778FE6421F6F783
:109A2000ABFB044664214C4328463146F6F706FF5B
:109A300000D22E463046F6F769FE6421F6F79CFB0D
:109A4000002901D0642000E000202018642809D0FB
:109A5000C8280ED00020FBF71FFB0020FBF726FBD9
:109A600019B0F0BD0120FBF717FB0120FBF71EFB2F
:109A7000F6E70020FBF710FB0120FBF717FBEFE7F1
:109A8000002474490008004038B5FFF759FC05462A
:109A900000240020FCF766FD22460A4C2946204699
:109AA000FCF747FD01206A4610700021517091704B
:109AB000D17020460099FCF7ABFC0120FCF752FD69
:109AC00038BD00000008004008B56846FDF7FAF808
:109AD0000428FAD008BD10B5FBF730FA10BD00001D
:109AE00010B504460120FCF781FF174804601748B1
:109AF000844205D10120FBF763FA0020FBF756FAF8
:109B000000F0D0F8FDF712F9FBF744FA01210F201D
:109B1000FBF760FA0020FCF75DFF0D488169052224
:109B20005202114381610C480A4901600B494160AE
:109B30000B4981600B4AC2600A4A403A02610A0A34
:109B400042618161C16110BD9405070000E1F50526
:109B5000008400404080008000E400E080008040FD
:109B600080808080808040801FB5009003206946FF
:109B7000487100208871087102900390684600F0D7
:109B800043F81FBD10B5FCF73FFE10BD10B5FCF744
:109B900021FF10BD10B5FCF70DFF10BD10B5044638
:109BA00020460930C0B20121FBF714FA00212046FB
:109BB000FDF7C0F910BD000070B50C461146054612
:109BC0001A462846FDF77CF92846FDF74FF97D2116
:109BD000401CC90041430B480068F6F7B7FA6043E0
:109BE00001462846FDF7A0F900212846FDF772F945
:109BF00001212846FDF774F901212846FDF71DF9DA
:109C000070BD00009405070010B588B0044600211F
:109C10001120FFF73FF800211220FFF73BF81C212D
:109C200001A8F6F7D6FA184800680190206802905B
:109C300060790490A07969460875207908730698C0
:109C400001210843069006980221084306900698D1
:109C50000421084306900698302188430690069810
:109C6000C0218843069000206946487788770877A6
:109C700001A90648F7F706FB1ECC054840301EC078
:109C8000002008B010BD00009405070000680040E7
:109C9000200F070010B50248F7F7E7FA002010BDC3
:109CA000006800402249012008602248C863224819
:109CB0004864224888642248C8642248C86522480B
:109CC0008865224888672248C8670846214A80304C
:109CD0000260214A4260214A4A65214A8260214A43
:109CE0000A64214A0A65214A0A66214A4A66214ACB
:109CF0008A66214ACA66214A0A67214A4A67214A76
:109D0000C260214A4261214AC261214A0262214A5B
:109D10004262214A8262214AC262214A0263214A86
:109D20004263214A8263214AC2632148C860704766
:109D300000010700FD3B0100C53401002D36010084
:109D4000C5380100B53C0100C53C0100A534010047
:109D5000B5340100DD390100AD390100613C01007D
:109D60003D330100453C0100A5350100153C0100D3
:109D70001F3C0100293C0100333C01007D3C0100F7
:109D80003D3C010065390100DD3B01005933010014
:109D90007D33010099330100B5330100D133010057
:109DA000ED33010009340100253401004134010084
:109DB0005D34010070B5194C206A002802D1FEF70D
:109DC000ABFB206200218170042141700223C3702B
:109DD0000121017108258560C56045614622026147
:109DE0005A2282616322C2618722D2004B256D0113
:109DF00002624562C5628262024620321374517467
:109E00006422C263064A0264E2691175FEF7F8FB38
:109E1000002211461046FEF77DFC70BDD001070000
:109E200000007042FEB50120FEF75EFC0A20FAF742
:109E3000B7FF0020FEF758FC0A20FAF7B1FF012017
:109E4000FEF752FC0A20FAF7ABFFFEF79FFB194F13
:109E5000194D00242B199E785978285D3246DB1C59
:109E6000FEF7D4FCA4193220E41CFAF7A5FFBC428B
:109E7000F0D30520FAF794FF01211320FEF7C2FE6C
:109E80005020FAF78DFF2A210220F6F745FFC8205F
:109E9000FAF786FF0020009001460190512303222B
:109EA0002920FEF71FFD0220FAF77AFFFEF794FB48
:109EB000FEBD0000CC23000068AE0100FAF73AFCBA
:109EC000F8F76AFFFEE7000030B5A1B000210320DB
:109ED000FEF7E0FE254DE869002802D1FDF7A8F95C
:109EE000E86187204B21EC69C000490103C461602F
:109EF00020600220207201206072042121756175AA
:109F0000A0750022E27520761949E1612146194BBE
:109F100078318B62184BCB62184B0B630E23AD214B
:109F20000B55A27362732073802215496846083C62
:109F3000F6F736F9802269462046FDF7E3FDE86929
:109F4000FDF746FA0F49E869FDF7BEFE0E4AE869DB
:109F5000D11FF939FDF782FEE869FDF747FF0B498C
:109F6000E869FDF765FE21B030BD0000D0010700B3
:109F7000004E7253FCAD0100011E0100919F0100D3
:109F800034D2010098080000F8020700002D3101CA
:109F90007CB5164D1446E8691E460168A14202D1FF
:109FA0004168B14219D0014650C0012220310A70E7
:109FB0002D21090108388C4202D9296A4E620C62AF
:109FC000FDF750FFE8692346203000780190084AE9
:109FD00008A100960AA0F6F7F5FEB122D20005A16D
:109FE00015A0F6F7EFFE01207CBD0000D0010700B0
:109FF000860500005332315F64656D6F000000001C
:10A000005B25735D20282530346429207265736FC9
:10A010006C7574696F6E2075706461746520775B10
:10A0200025645D20685B25645D20636F6D707265DB
:10A0300073735B25645D0A005B25735D2028253002
:10A0400034642920505053205570646174650A00AF
:10A05000F3B587B005460027A148089940680E0C63
:10A060008030C36A0898000A002B05D0062D18D04E
:10A07000142D16D0242D14D0052D1BD0132D19D03E
:10A08000062D17D0142D15D0152D45D0232D43D0D6
:10A09000242D41D0392D73D0292D71D0002009B045
:10A0A000F0BDC1B20022242D00D1F2B2E8B298472F
:10A0B0000020F4E7C6B23046FAF764FE04462000FA
:10A0C0001DD0207A002801D086480BE0FAF7EEFD7B
:10A0D000002805D182484068FDF710F9FAF7E6FD3F
:10A0E000002805D000218160056046600461D6E744
:10A0F0007D4A7EA180A0F6F765FE0020CFE7062D01
:10A1000001D0142D06D10D223346920177A185A0EE
:10A11000F6F758FE0020C2E7C7B23846FAF732FE1B
:10A120000446200020D0207A002801D06D480BE0A2
:10A13000FAF7BCFD002805D169484068FDF7DEF854
:10A14000FAF7B4FD002807D001218160056047605F
:10A15000C1680E700461A2E7634A64A1353266A04B
:10A16000F6F730FE00209AE7242D06D15E4A3B46E2
:10A1700044325EA16BA0F6F725FE00208FE7FFE7D3
:10A1800008980002060C002E0AD0761E301D8008AA
:10A190000490FAF741FD00280BD06D4807690FE0E5
:10A1A000514A52A15B326BA0089BF6F70BFE0020D0
:10A1B00075E77322D2004DA171A0089BF6F702FE4D
:10A1C000F8B206900698FAF7DDFD0590059800288C
:10A1D00064D0FF2E62D80598007A002801D0414C47
:10A1E0000BE0FAF763FD0446200006D13C484068C6
:10A1F000FDF784F8FAF75AFD0446002C48D0A66013
:10A2000025600698606005982061032E00D903261A
:10A21000002006E0411CCA003946D140E2681154D2
:10A22000401CB042F6D301251DE0FAF7F5FC0028EA
:10A230001ED047480769A800A16884460E1A701C02
:10A24000042801D9042600E0761C002008E0C200A2
:10A250003946D140E2686346D318421E9954401CE7
:10A26000B042F4D36D1C04988542DED3204616E735
:10A270004E48406936490968069A00921A4A019187
:10A280000290A13219A14AA0089BF6F79BFDEDE7C9
:10A29000154A16A1A93253A0F6F794FD0124104DDA
:10A2A0002B4E2035594F0BE0FAF7B6FC00280CD0A6
:10A2B0003169287D002802D03846FBF77AFA641C01
:10A2C00004988442F0D30020E9E606980090FD222D
:10A2D000920006A14EA0089BF6F774FDF3E700007C
:10A2E0000C110700501A07003203000068616C5F10
:10A2F0007673796E630000006572726F72205B2561
:10A30000735D2028253034642920616C6C6F6320D4
:10A310006461746120627566666572206572726F31
:10A32000720A00006572726F72205B25735D2028CF
:10A3300025303464292072656164205B307825788B
:10A340005D206E6F20726573706F6E7365210A00F9
:10A35000002000406572726F72205B25735D2028BB
:10A360002530346429207061636B657420686561F1
:10A37000646572206572726F725B25785D0A0000F9
:10A380006572726F72205B25735D202825303464FE
:10A3900029205B307825785D6765742064637320BD
:10A3A00074696D656F75740A00000000002100403B
:10A3B0006572726F72205B25735D202825303464CE
:10A3C00029205B307825785D5B307825785D2074B6
:10A3D000696D65206F7574205B25785D5B25785D00
:10A3E000200A00005B25735D202825303464292075
:10A3F000616C6C6F63206461746120627566666570
:10A4000072206572726F720A000000000004004042
:10A410006572726F72205B25735D2028253034646D
:10A4200029205B307825785D6463735B307825780C
:10A430005D2067657420646174612074696D656F67
:10A4400075740A00F8B50E464A4D696800297DD03A
:10A450002022525C002A79D028317FD00024464F38
:10A46000002815D03846FCF759FB010C091A491C85
:10A470000804000EC9B26A682032137C834202D1FC
:10A48000537C8B4204D010746868203041740124DE
:10A49000002E15D03846FCF74CFB010C091A491C5C
:10A4A0000804000EC9B26A682032937B834202D14D
:10A4B000D37B8B4204D0907368682030C173012431
:10A4C000002C4BD069682031087C4A7C000280183F
:10A4D0000A7D497D12025118F5F738FE441E274EB9
:10A4E0003046FAF74FFFA0420AD0002C38D00020A7
:10A4F000FAF7AAFD0020FAF7B1FD0120FAF79AFD5C
:10A5000003239B021E494A6918469043FBD11B490D
:10A510008031086A07221204904322041043086223
:10A5200068682030437B027B1B021A43837BC47B19
:10A530001B04240623431A437260437C027C1B02E3
:10A540001A43837CC07C1B04000600E006E0034342
:10A550001A43B260086A0A06104308620120F8BD77
:10A560000120FAF771FD0020FAF778FD0020FAF7D4
:10A5700061FDC5E70C1107000020004000240040E9
:10A580000021004010B51F4C14E02069C2B20A2A15
:10A5900016D001461046FFF75BFD0146080008D0C3
:10A5A0000869027A002A04D0174A436852681046A4
:10A5B000984700200028E8D10A20144A02231BE013
:10A5C00000F026F8F5E75169194201D0012100E0B9
:10A5D000002100290ED121684907890F0CD020469F
:10A5E000FCF73FFA02212046FCF740FA04212046FE
:10A5F000FCF73CFA012010BD0146401EC0B2002904
:10A60000E1D1C2E7002000400C110700002100400A
:10A61000F0B5A1B00446802101A8F5F7DAFD2002CB
:10A62000040C3E4E802C0BD923463D4A3DA14048A8
:10A63000F6F7C8FB3046FCF714FA002021B0F0BD55
:10A64000E01C8708002501AE08E0FAF7E5FA0028CB
:10A6500012D032480069A90070506D1CBD42F4D37D
:10A66000344D686800280FD0582C02D901A8FAF799
:10A670002DFE002200201BE0294A2AA110322EA024
:10A68000F6F7A0FB0020D9E7254A26A1193234A00D
:10A69000F6F798FB0020D1E7014628316B680E469B
:10A6A0005F5C01A9095C8F4201D099550122401CD1
:10A6B000A042F1D368682030017C437C0902CF18A6
:10A6C000817BC37B0902C9180091002A1AD0017D41
:10A6D000407D090209183846F5F738FD461E2A481C
:10A6E000FAF742FF6968203108703146274E01238E
:10A6F00000223046FAF70CFE696880222831304685
:10A70000FAF745FE68688030056B002D04D0E1B291
:10A710003A4601A8009BA84701208FE7002000408F
:10A720008602000068616C5F7673796E63000000DA
:10A73000F0EA01000C1107006572726F72205B2550
:10A74000735D2028253034642920505053206765DC
:10A75000742064617461206661696C0A0000000005
:10A760006572726F72205B25735D2028253034641A
:10A7700029207669642073796E63206E6F74206976
:10A780006E697420210A0000002800400024004067
:10A79000F8B5274E7068C00512D508213046FCF781
:10A7A000CAF9002806D00020FFF7ECFE0121304650
:10A7B000FCF75CF9FF21002201313046FCF754FA26
:10A7C00000213046FCF7B7F9002806D00120FFF73A
:10A7D000D9FE01213046FCF749F9012189033046B1
:10A7E000FCF79EF9002801D0012400E00024012795
:10A7F000FF0339463046FCF793F9002801D00125C4
:10A8000000E000252046284310D029462046FFF7C7
:10A8100019FE002C04D0012189033046FCF726F9EB
:10A82000002D03D039463046FCF720F9F8BD000072
:10A8300000200040FEB5374E374D31462846FCF724
:10A840006FF9364C002810D06069296801903448AF
:10A850000091036B334A34A136A0F6F7B3FA00F047
:10A8600097F931462846FCF701F90126760531466D
:10A870002846FCF755F9002806D03C48FBF702FFB4
:10A8800031462846FCF7F2F801273F0539462846AD
:10A89000FCF746F9364E00280AD039462846FCF720
:10A8A000E5F870688030816B002901D0002088476E
:10A8B0002F4606213846FCF733F900280FD03846DA
:10A8C000FCF7CFF806213846FCF7D0F86069009015
:10A8D0003B68144A14A13C3226A0F6F773FA2F48BD
:10A8E0004568002D14D07068A030007F012801D980
:10A8F00000F04EF960693968094A126B0092094A02
:10A90000019102902B46483207A12548F6F75AFAE2
:10A91000FEBD0000000204000020004000210040B5
:10A92000802A0040FA04000068616C5F7673796EDB
:10A93000630000006572726F72205B25735D2028D2
:10A940002530346429207278206669666F2065722C
:10A95000725B307825785D2073305B307825785DC8
:10A960002073315B307825785D0A0000000C0040D0
:10A970000C1107005B25735D2028253034642920E5
:10A98000706B742062756666657220657272205BFA
:10A9900025785D5B25785D0A00000000C02400403A
:10A9A000A0EA0100F0B51C4B596B186B14308142C2
:10A9B00031D81A4801684213114301601848407D9C
:10A9C000022828D9174C184A2168887880008018F6
:10A9D000CE78164A1049D5014039002E0CD0134EBE
:10A9E0008036B668B60703D4D66876087600D66097
:10A9F0000A68AA430A6006E0D66801273E43D6608B
:10AA00000A682A430A6002881A630A6801239B04C1
:10AA10001A430A602060F0BD40080040000C00406E
:10AA20002C110700AC0A0700441A07000010004070
:10AA300010B50023074A0A210320FFF7BDF8064995
:10AA40000878401C08700549888A002801D0401CFD
:10AA5000888210BD31AA01005C040700D001070004
:10AA6000F8B506460C46F5F7F7FF051E0F4600D071
:10AA70000120014349000B484908411AC90F0DD074
:10AA8000002E01D0012100E000210C4361004908A3
:10AA9000401AC00F02D10120F6F750FD2846394672
:10AAA000F8BD00000000F07F7CB5304C022120464C
:10AAB000FCF7B8FA00282DD02D480178002920D1C4
:10AAC00001210170817802291BD101462031497D85
:10AAD000284B022911D919680A0327490AD5806829
:10AAE000C5688268C06A5219401E1218486B9042AD
:10AAF000FCD102E0486B0028FCD100211846FBF78E
:10AB0000A7FC02212046FCF75CFA00220421204623
:10AB1000FCF7CDFA00212046FCF784FA002803D088
:10AB200000212046FCF74DFA01212046FCF77AFA75
:10AB3000002803D001212046FCF743FA03212046D8
:10AB4000FCF770FA00280FD0084980318A684868FD
:10AB5000019200900B68094A09A10C48F6F732F9F6
:10AB600003212046FCF72DFA7CBD000000100040B8
:10AB70000C1107000008004040080040820500005A
:10AB800068616C5F7673796E6300000008EA01000B
:10AB9000F0B58BB02C484068A030007F022804D963
:10ABA0002A48002141602A4841602A4C6668276A89
:10ABB000606A0A90A06A0990E06A0890206B07908A
:10ABC000E06B0690234D4035286805906868049036
:10ABD000606B0390A06B02901F48006A01901720E1
:10ABE000FAF784FA1820FAF781FA1C48FCF73EFAC3
:10ABF000666027620A9860620998A0620898E0621D
:10AC0000079820630698E0630598286004986860B8
:10AC1000039860630298A0630F49019808620A4C88
:10AC20000D486168802228318038FAF7B0FB6068EF
:10AC3000A030007F022804D9044801214160044863
:10AC4000416001200BB0F0BD0C110700002900404D
:10AC500000280040002000408024004000100040F8
:10AC6000FEB53F4F38683902084338603D4D3E4AD3
:10AC7000687D2C46203C002816D000211046FBF7AA
:10AC800036FD6A7D012A64D9A068C3688168C91845
:10AC90000369C06A18180D18216B6C1A334E042A08
:10ACA00011D0052A49D131E001211046FBF71FFDE3
:10ACB000002201213846FBF7BAFB00223846216BFF
:10ACC000FBF737FCFEBD03212846F5F73FFA01905C
:10ACD000A04205D2264A27A129A0F6F773F86424DA
:10ACE00068000321F5F732FA001B81B2318001239D
:10ACF000B3700022F2700198001BB0800220B07186
:10AD0000F371281B3081B272F27216E0680800906D
:10AD1000A04206D2164A17A1143228A0F6F752F81C
:10AD200064240098001B81B231800120B070F07063
:10AD3000281BB0800020B071F0712F4806600022FF
:10AD40003846FBF7F6FB012211463846FBF76FFB4E
:10AD5000FEBD002201213846FBF769FBFEBD000065
:10AD6000000800402C110700000C0040441A0700A6
:10AD70006904000068616C5F7673796E630000009F
:10AD80006572726F72205B25735D202825303464F4
:10AD90002920736F667420393020687A207465200A
:10ADA00070617261206572726F7221207573652007
:10ADB00064656661756C740A000000006572726FEC
:10ADC00072205B25735D2028253034642920736F41
:10ADD00066742031323020687A2074652070617288
:10ADE00061206572726F72212075736520646566DB
:10ADF00061756C740A000000AC0A070029000000AD
:10AE00009130010001000000280000004D300100D9
:10AE100001000000DF0000003D2F010000000000E5
:10AE2000510000003130010000000000600000000F
:10AE3000D13201000100000010000000C930010003
:10AE40000100000011000000453101000100000078
:10AE500004000000B5310100010000000000000006
:10AE6000000000000000000005000111390006F09C
:10AE700055AA520800390009BA01AF001409AC0004
:10AE8000013900026F08390009BA01AF0014001C33
:10AE900000003900026F10390008BA01AF00140336
:10AEA0004C00390009BB01AF0014001C00413900FF
:10AEB000026F06390004B52B1C323900026F0B39C2
:10AEC0000004B5332B233900026F10390006B51C7E
:10AED0001C1C1C1C390003B586023900026F0239A4
:10AEE000000EB62F2F2F2F2F2F2F2F2F2F2F2F2F3B
:10AEF00039000EB700FEDCBA98765432100000001C
:10AF0000053900026F0D390007B70000000000008E
:10AF10003900026F1339000DB717899AABBCCDDE2B
:10AF2000EFFFFFFFFF3900026F1F390019B747FF1E
:10AF300088109921AA32BB43CC54DD65EE76B0FF70
:10AF4000FFFFFFFFFFFF390005B218630808390053
:10AF5000026F09390002B2403900026F0F3900094F
:10AF6000B2302081462146200039000DB300080090
:10AF70001800180031003100623900026F0C3900EE
:10AF80000DB3006200C000C0014601460147390010
:10AF9000026F1839000DB301470333033307FF076E
:10AFA000FF0FFF3900026F24390009B3015508CCA7
:10AFB00008CC0FFF3900026F2C39000FB30060007E
:10AFC00060006000600060006000603900026F3A5D
:10AFD00039000DB300600060006000600060006038
:10AFE0003900026F4639000DB30060006000600058
:10AFF000600060006039000FB40060006000600015
:10B00000600060006000603900026F0E39000DB40E
:10B010000060006000600060006000603900026F46
:10B020001A39000DB400600060006000600060002C
:10B03000603900026F3039000FB4006000600060BA
:10B0400000600060006000603900026F3E39000D52
:10B05000B4006000600060006000600060390002C1
:10B060006F4A39000DB4006000600060006000604D
:10B0700000603900026F2639000BB40990003000DF
:10B080003000300030390003B90096390003BD04A8
:10B09000B0390004C046F3C13900026F083900021C
:10B0A000C0403900026F09390003C0208139000215
:10B0B0006F02390002C1243900026F02390009C150
:10B0C00024570057005700573900026F0A39000310
:10B0D000C100573900026F01390002C30039000274
:10B0E0006F08390002C300390002C510390002C8D8
:10B0F0000D390002C984390005CA120082BC39002A
:10B1000002CB883900026F02390003EC801039004D
:10B1100002B900390005BE0E0B14133900026F0589
:10B12000390002BE8A3900026F29390002D900397C
:10B1300000026F01390002D9803900026F0739001F
:10B1400003B207FF3900026F17390003B207FF3956
:10B150000006F055AA5208003900026F2A39000291
:10B16000D943390006F055AA52080139000BB50041
:10B17000B000B000B000B000B039000BB60148001C
:10B18000C000C0014800C0390003B0040439000306
:10B19000B31313390007B71B1B1B1B1B1B39000301
:10B1A000B10808390003B41313390007B8464646FE
:10B1B00046464639001DB9001F0000001F00001F51
:10B1C00000001F0000000000001F1F1F1F1F0000C5
:10B1D000000000390005BA1010101039000DC2002F
:10B1E000B0014800B0014800B00148390002BB037B
:10B1F0003900026F05390014BB1B1B1B1B1B1B1BDB
:10B200001B1B1B2020202020202020203900026F23
:10B2100018390014BB1B1B1B1B1B1B1B1B1B1B20E0
:10B2200020202020202020203900026F2B390014FC
:10B23000BB1B1B1B1B1B1B1B1B1B1B2020202020A5
:10B24000202020203900026F3E390014BB1B1B1B3D
:10B250001B1B1B1B1B1B1B20202020202020202011
:10B26000390003C48003390003CD0581390002C7CA
:10B2700001390002CF5C390006CE0000010004391C
:10B2800000026F01390004D20000113900026F067C
:10B29000390002D2053900026F0F390002D200399D
:10B2A00000026F09390002D2003900026F10390024
:10B2B00002D80C390002D1073900026F02390002AE
:10B2C000D1063900026F05390002D106390003D6D4
:10B2D0000020390006F055AA520802390019B900B9
:10B2E00004000C0014001C002C003C004C005C000E
:10B2F0007C009C00BC00DC390019BA00FC013C0158
:10B300007C01BC01FC027C02FC037C03BC03DC036B
:10B31000FC03FF390002BC11390011BD9600690021
:10B3200000960069BB4444BBEE1111EE390002C126
:10B3300002390009C2910019009100190039000377
:10B34000C000003900026F02390002BF1339000645
:10B35000F055AA520802390002CC30390002BF2948
:10B36000390013B0000000EA013001BD022B029A3F
:10B3700002EF033503C1390013B10422048704E14D
:10B38000052F05C9064E06C50734079C39000FB2C4
:10B3900007FF086208C8092D09920A740A77390064
:10B3A00013B3000000AF00EA016001CD022E027E5F
:10B3B00002BF0342390013B4039803EE0444048E21
:10B3C0000512058005EC065006AD39000FB5070AD9
:10B3D000076307B9080E086209110914390013B68A
:10B3E000000000C4011C01CD026102E5034B03A172
:10B3F000043F390013B704AB0517057A05D1066D74
:10B4000006F3077407EB085B39000FB808CB093B5C
:10B4100009B00A240A970B870B89390002BF283923
:10B420000013B00000011D015901BC022402830277
:10B43000D703010379390013B103EB045404A904C1
:10B44000F7057E05F9067106DB074039000FB207E4
:10B450009B07F3085108AB090809E509E739001310
:10B46000B3000000F20136016A01BD0214025E025F
:10B470008A02FA390013B4035D03B90404044D04CD
:10B48000CA0534059A05F5064F39000FB506A3061F
:10B49000F30748079407E608A108A7390013B60088
:10B4A000000110015C01C0024002BA0322035B03E9
:10B4B000E8390013B7046404DE0535058E0620065E
:10B4C0009E071C078907F539000FB8085708B90906
:10B4D00021098609F10AF90AFE390002BF2739005D
:10B4E00013B00000012E012F018101CF0207024895
:10B4F000028602E6390013B1033E037903C4040C4B
:10B50000048A04F3055105A205F439000FB206437D
:10B51000068E06D40717075607CD07D0390013B398
:10B5200000000108012A014B017601A601DE021785
:10B53000026E390013B402BE02FA033B037A03E938
:10B54000044A049D04E9052F39000FB5057305B3BE
:10B5500005EF062A066306D106D3390013B60000AC
:10B56000013A0142018401D4021D026F02BE033779
:10B57000390013B703A203E9043D048C0515058ABD
:10B5800005EB0645069839000FB806EB073A078227
:10B5900007C9080D088F0892390002BF2639001329
:10B5A000B00000012901340150018601BA01E40212
:10B5B0000A025D390013B102A602E603200351031B
:10B5C000B20408045C04A904EE39000FB2052C058E
:10B5D00067059C05D20608066D0670390013B30096
:10B5E0000000FE011C013A014E016A018801A80118
:10B5F000F2390013B40234026E02A202D10328030E
:10B600007703C00405044539000FB5047D04B20476
:10B61000E40512054005970599390013B6000001AD
:10B62000360144015D018901C001F00220028C391C
:10B630000013B702E70337037D03B8042804890425
:10B64000E30537058439000FB805C50603063F0634
:10B650007606AD0718071A390002BF25390013B066
:10B660000000012801340150018601BB01E4020AF7
:10B67000025C390013B102A502E5031F035003B1B8
:10B680000407045B04A804ED39000FB2052B05661E
:10B69000059B05D30607066C066E390013B3000040
:10B6A00000FE011C013A014E016A018801A801F265
:10B6B000390013B40233026D02A102D003270376CE
:10B6C00003BF0404044439000FB5047C04B104E34F
:10B6D0000512053F05960598390013B6000001359F
:10B6E0000144015D018901C001F00220028C390092
:10B6F00013B702E60336037C03B70427048804E289
:10B700000536058339000FB805C40602063E0677E4
:10B7100006AC07170719390002BF24390013B0001F
:10B72000000124013601460166019101BC01DB02E2
:10B7300018390013B10259029302C702F8034B03F0
:10B740009F03E60429046439000FB2049F04D60560
:10B75000090539056705BD05BF390013B3000000B1
:10B76000F20115012F01420154016A018101B5392D
:10B770000013B401EF02230252027E02CB03140332
:10B7800055039203C739000FB503FC042F045E0470
:10B790008904B204FF0501390013B600000131012C
:10B7A000450150016F019401C101E50233390013D5
:10B7B000B7028802D10311034D03B10411046204DE
:10B7C000AC04EC39000FB8052C056A05A105D306B9
:10B7D0000306610663390002BF23390013B000007D
:10B7E00001210131013F014F0167018601A601DA04
:10B7F000390013B1020702370264028F02DB031C17
:10B80000035C039903CD39000FB204000430045ED9
:10B81000048A04B304FF0501390013B3000000F3E8
:10B820000108012301340142014F015F0180390009
:10B8300013B401A601D001F9021F026402A002D9CB
:10B84000030F033E39000FB5036C039803C003E7F1
:10B85000040E04550456390013B60000012E013FB2
:10B86000014B0159016F018B01AA01E4390013B7A3
:10B87000021E025C029602CC0329037903C4040A67
:10B88000044539000FB8047E04B404E505150543EA
:10B8900005960598390002BF22390013B000000157
:10B8A0001F012D013B013F014F0160017501A339CB
:10B8B0000013B101C901ED02100232027202AD02A1
:10B8C000E30315034639000FB2036F039D03C3035F
:10B8D000E9040D04500451390013B3000000F001D5
:10B8E000000117012C0134013E0148015D390013AC
:10B8F000B40176019001AD01CC0206023A026C025D
:10B900009802C439000FB502EA0312033403570347
:10B910007703B403B5390013B60000012B013A01D7
:10B9200048014A01590169017B01A7390013B70198
:10B93000D201FC0229025602A802F10333036F036D
:10B94000AA39000FB803DA040F043A0464048D0422
:10B95000D604D8390002BF21390013B00000011EFF
:10B9600001270138013C013E014A015701733900AA
:10B9700013B1019401B301CE01EA0220024D02800D
:10B9800002A602D139000FB202F5031B033B03618B
:10B99000037D03B703B9390013B3000000ED00FACB
:10B9A000010E011C012B013201380147390013B48B
:10B9B00001560167017A018E01BA01E402110233D6
:10B9C000025939000FB5027B029D02BA02DA02F475
:10B9D000032A032B390013B60000012A0134014564
:10B9E00001480149015501600179390013B70199F6
:10B9F00001B901D801F9023D027802B802E8031C3E
:10BA000039000FB803490376039D03C803E9042DE9
:10BA1000042E390002BF20390013B00000011F01BD
:10BA200022012C012D012E012F0130014939001373
:10BA3000B10159016A017D019101B601D701F902F5
:10BA40001C023939000FB202540270028E02A502A4
:10BA5000C002EB02EC390013B3000000E200F20177
:10BA6000020112011F0122012A0132390013B4011F
:10BA7000390142014B015501690181019A01B60169
:10BA8000D139000FB501E90204021C0231024A0259
:10BA9000720273390013B600000129012E013D0125
:10BAA000400141014201430154390013B7016201D1
:10BAB000710183019601BD01E3020E0237025E3976
:10BAC000000FB8028002A502C902E60309033D0384
:10BAD0003E390002BF39390013B0000001FD0244B5
:10BAE000028C02C30331038D042804A7390013B16B
:10BAF0000513057305C5061706A407230793080257
:10BB0000086439000FB208C109780A220A760A9D32
:10BB10000ACC0ACC390013B3000001E0021E024532
:10BB2000027702DC033303C10431390013B40492F9
:10BB300004E7052F057705F2066206C3072307769B
:10BB400039000FB507C3085B08E5092609440967F2
:10BB50000967390013B6000001E60241028E02D4E3
:10BB6000036103D5048A0516390013B7058C05F463
:10BB7000064C06A3073907C2083C08B4092039005F
:10BB80000FB809860A510B140B720BA00BCC0BCC0F
:10BB9000390002BF38390013B00000027302A1025D
:10BBA000CF02F70345038D040E047D390013B10461
:10BBB000DE0534058005C9064A06BD072607850748
:10BBC000E139000FB2083508D2096509AD09D0097D
:10BBD000F509F5390013B300000281029B02AB02A4
:10BBE000C402F6033203A30404390013B4045A0454
:10BBF000A704EA052B059B0600065C06AE06FD3988
:10BC0000000FB5074507CA08440880089E08B90810
:10BC1000B9390013B60000027002A402D003010378
:10BC20006303C0045F04DF390013B7054B05A905A2
:10BC3000FB064B06D5075007C10828088C39000FB2
:10BC4000B808E709950A3B0A8C0AB70ADD0ADD390C
:10BC50000002BF37390013B0000001C4028A02A8F5
:10BC600002C702FC032F039003E4390013B104342C
:10BC7000047D04BC04F9056405C6061C066C06B800
:10BC800039000FB206FD077E07F7082E0849086342
:10BC90000866390013B3000001CD028E029E02A98E
:10BCA00002C702E80334037F390013B403C4040459
:10BCB000043C047204D20528057305B905FB39005C
:10BCC0000FB5063806A80710073F0756076D076F20
:10BCD000390013B6000001C1028902AB02C8030794
:10BCE000034803C3042C390013B7048A04DF052674
:10BCF000056905DD064706A306FA074A39000FB8AD
:10BD00000795082108A408DF08FD091A091D390054
:10BD100002BF36390013B00000024D0268028302F0
:10BD20009F02C702EE03300372390013B103AD0363
:10BD3000E7041A044C04A204F7053E058405C03943
:10BD4000000FB205FC066706C806F6070E072307B4
:10BD500023390013B30000028B02920299029E0263
:10BD6000A802B702E40318390013B4034C0380039C
:10BD7000AE03DA0425047004AF04ED052239000F88
:10BD8000B5055605B4060906310645065806583964
:10BD90000013B60000026B0280029602A802C902DC
:10BDA000F10345039B390013B703E8042F046C0427
:10BDB000A80508056705B40600064139000FB80656
:10BDC0008206F4075C078E07A607BE07BE3900028D
:10BDD000BF35390013B00000024D026002740287C3
:10BDE00002B302D903250369390013B103A603E0A6
:10BDF00004150449049F04F4053C058205BE39007E
:10BE00000FB205FA066506C806F7070D07200720DA
:10BE1000390013B300000281028B0296029C02AA31
:10BE200002B602E40317390013B4034A037A03A9E4
:10BE300003D60421046C04AC04EA051F39000FB5D5
:10BE4000055405B306080630064306560656390063
:10BE500013B600000268027C029102A202C802EC42
:10BE60000347039B390013B703E4042B046904A6BA
:10BE70000506056505B305FF064039000FB80680C5
:10BE800006F3075C078D07A507BC07BC390002BF96
:10BE900034390013B0000002720283029502A70237
:10BEA000C802EA03300374390013B103B203E80493
:10BEB0001B044C04A504F5053B058005BB39000FA8
:10BEC000B205F6066006C006EF0704071807183922
:10BED0000013B3000002A602B102BD02C502D102E6
:10BEE000DC02FC032C390013B4035D038B03B8039D
:10BEF000E40431047604B404F1052539000FB505D6
:10BF00005805B40608063006410655065539001393
:10BF1000B60000028D02A102B602C802E7030603C2
:10BF20005203A6390013B703F10433046F04A905C3
:10BF30000C056505B205FD063D39000FB8067C0607
:10BF4000EE07550787079D07B407B4390002BF33D2
:10BF5000390013B0000002AE02BD02CD02DD02FDC9
:10BF6000031C035A0391390013B103C503FA0423D8
:10BF7000045304A504EF0532057305AD39000FB273
:10BF800005E5064B06A806D606EC06FD06FD3900BB
:10BF900013B300000306030D0315031D032703302D
:10BFA00003490364390013B4038803B003D203F8D0
:10BFB0000439047904B304EC051E39000FB5054EAD
:10BFC00005A605F6061C062E063F063F390013B6E9
:10BFD000000002ED02FA03080316032E0345038452
:10BFE00003BF390013B703FF043E047204A905061A
:10BFF000055A05A405ED062C39000FB8066906D8C8
:10C00000073B076B078207970797390002BF323952
:10C010000013B000000310031A0324032E0342038D
:10C0200057038503B1390013B103E4040A042F0454
:10C030005704A204E40522055F059639000FB205F6
:10C04000CA062A068306AE06C306D506D5390013EE
:10C05000B3000003590361036903710381038C0377
:10C060009E03AE390013B403C503DE03F6041104C6
:10C070004E047E04B204E4051339000FB5053F05F4
:10C080009005DC05FF061006210621390013B600D5
:10C0900000033F034B03570363037B039003BB037E
:10C0A000E5390013B7041B0449047504A205010512
:10C0B00048058F05D4061039000FB8064A06B307A5
:10C0C0001407410756076B076B390002BF3139006F
:10C0D00013B00000035D0365036D037503850395CD
:10C0E00003B603D6390013B103F404180439045A13
:10C0F000049A04D20509053F057139000FB2059E67
:10C1000005F706490670068206950695390013B3B1
:10C11000000003BC03C103C603CB03D503DF03EC5C
:10C1200003F7390013B40404041504260438046228
:10C13000048804B304DC050439000FB50529057033
:10C1400005B305D505E405F205F2390013B6000084
:10C15000039F03A703AF03B703C803D903F6041172
:10C16000390013B704310459047D04A204EE052EEE
:10C17000056C05A905E439000FB80616067A06D441
:10C1800006FE071207260726390002BF30390013C2
:10C19000B0000003B303B803BD03C203CC03D6034E
:10C1A000EA03FF390013B104140427043C045204C9
:10C1B0007D04A804D204FB052039000FB205470511
:10C1C0008C05CD05F00600060E060E390013B300EF
:10C1D00000041A041D04200423042A0431043E042C
:10C1E00047390013B40450045704600469047D0403
:10C1F0009104AB04C704E239000FB504FC05310516
:10C2000063057C058705940594390013B600000486
:10C21000000405040A040F041904230436044739F2
:10C220000013B7045B046C0481049704C704F4058D
:10C23000250555058139000FB805AE0600064A06EA
:10C240006F068006920692390006F055AA5208023F
:10C25000390002BF42390013B00000049E04D90522
:10C2600014054F059D05DD064806AE390013B107DC
:10C2700003075707A007E6086208D509360994099D
:10C28000E339000FB20A350AC40B430B810B9F0B35
:10C29000BA0BBA390013B3000004BB04BB04BB04DF
:10C2A000BB04D9051605950605390013B4066106C9
:10C2B000B306F9073A07A90812086908BE09073941
:10C2C000000FB5094F09CE0A3F0A750A8E0AA60A61
:10C2D000A6390013B60000047B04A504CF04F205C0
:10C2E0004605A5064E06D9390013B7074F07B7080C
:10C2F00010086208EB096D09D50A3B0A9039000F56
:10C30000B80AE80B800C070C480C670C850C8539C3
:10C310000002BF41390013B00000038504C404F1DA
:10C32000051E056A05A405FF0650390013B1069ED7
:10C3300006E10721076007CD082F088A08E0092ACF
:10C3400039000FB2097209F00A660A9C0AB70AD1CD
:10C350000AD3390013B30000039B04BB04BB04BB26
:10C3600004C504E0053E059E390013B405F3063C00
:10C37000067F06BC0723077B07CE081C085E390032
:10C380000FB5089F0912097A09AB09C309DA09DC5C
:10C39000390013B60000036A049604B604D5050FED
:10C3A000055005DA0659390013B706C3072007758B
:10C3B00007C2084508B20918097809C839000FB83A
:10C3C0000A160A9E0B1C0B560B730B8E0B90390032
:10C3D00002BF40390013B00000017F047D04B004A7
:10C3E000C304EA05100558058A390013B105B705DD
:10C3F000E006030625066906AB06E3071A0750396F
:10C40000000FB2078007DC082E0856086A087C086F
:10C410007E390013B300000188049904BB04BB04F7
:10C42000BB04BB04BE04D2390013B404F2051A05E0
:10C4300043056C05B90602063E067706AC39000FC7
:10C44000B506DB0731077A079E07B007C107C33976
:10C450000013B600000174045B0488049604B10460
:10C46000CC04FC0532390013B7056D05AA05E106B9
:10C4700017067B06D50722076B07AF39000FB807F1
:10C48000E9085708B108DE08F40909090B39000268
:10C49000CE01390002CC00390006F055AA5208023C
:10C4A000390019B90004000C001C002C003C004CA1
:10C4B000005C007C009C00BC00DC00FC390019BA68
:10C4C000013C017C01BC01FC023C027C02BC02FC80
:10C4D000033C037C03FC03FF390006F055AA520815
:10C4E000033900026F1E390007B0FFFFF0FFFFF0B5
:10C4F0003900026F24390007B0FFFFF0FFFFF03969
:10C5000000026F2A390007B0FFFFF0FFFFF039008B
:10C51000026F30390007B0FFFFF0FFFFF039000273
:10C520006F36390007B0FFFFF0FFFFF0390006B2A9
:10C5300000101006013900026F0539000DB200101D
:10C54000100010100010100010103900026F113987
:10C550000009B206010601060106013900026F1941
:10C56000390002B20039000AB401010101010101E0
:10C570000101390010B6B00000000000000000000A
:10C5800000000000003900026F0F390004B61F00E0
:10C590000A3900026F1A390004B60F000A39000286
:10C5A0006F25390004B60F000A3900026F303900D8
:10C5B00004B60F000A390011BB11000F5E000F5EB8
:10C5C000000F5E000F5E000F5E390011BC221010DC
:10C5D0003D00103D00103D00103D00103D390006AB
:10C5E000F055AA520804390002C214390002B102FF
:10C5F000390002B2403900026F01390004B2000074
:10C60000003900026F04390004B209E34039000226
:10C610006F07390004B209E4003900026F0A3900DB
:10C6200004B209E340390002CB86390006D000008D
:10C630000010013900026F01390006CB05101F3EC2
:10C640007C3900026F0639000BCB000800620147FD
:10C6500007FF0FFF3900026F00390006D240201893
:10C66000120A3900026F05390006D24020180C0B5F
:10C670003900026F0A390006D24020180F0B39002A
:10C68000026F0F390006D2401014100E3900026FED
:10C6900014390006D22F202010123900026F1939E8
:10C6A0000006D2803015100D3900026F1E390006C9
:10C6B000D280302810083900026F23390006D2805A
:10C6C00020180A0A3900026F28390006D268201A99
:10C6D00010123900026F2D390006D2602020101A86
:10C6E0003900026F32390006D2401018100A3900A2
:10C6F000026F37390006D2401018100A3900026F55
:10C700003C390006D240101810083900026F413938
:10C710000006D2401018100D3900026F463900068D
:10C72000D22F202010103900026F00390006D440AB
:10C7300030180A093900026F05390006D440282252
:10C740000A083900026F0A390006D440201010068A
:10C750003900026F0F390006D43020101004390060
:10C76000026F14390006D430201010043900026F13
:10C7700019390006D4804818100D3900026F1E398F
:10C780000006D48040300D103900026F23390006B6
:10C79000D4803020140D3900026F28390006D4A847
:10C7A0002820100A3900026F2D390006D460282095
:10C7B00010083900026F32390006D44030180A0AD6
:10C7C0003900026F37390006D44028200A083900A2
:10C7D000026F3C390006D440201010063900026F69
:10C7E00041390006D420201010043900026F463968
:10C7F0000006D43020101004390006F055AA520863
:10C8000005390003C70701390004B00721003900CA
:10C8100003B38580390003B58581390005B78400ED
:10C820000081390005B884000081390005B9850010
:10C830000081390004D0000310390005E0820000B7
:10C8400002390004D1000110390005E18200000224
:10C85000390003EC0D013900026F02390013EC00BE
:10C8600000000000000000000000000000000000C8
:10C87000003900026F06390003EC00FF390002CADC
:10C8800033390004CB333333390002D82239000264
:10C89000D901390006F055AA520806390006B0132E
:10C8A00032123204390006B132310E32313900060B
:10C8B000B23200323132390002B30F390006B613FA
:10C8C00032123204390006B732310E3231390006E5
:10C8D000B83200323132390002B90F390002D001CA
:10C8E000390006F055AA520807390006B08440788E
:10C8F0007000390007B11C0C000C1C00390002B29A
:10C90000203900026F36390002B2323900026F3F1F
:10C91000390002B2043900026F09390002B220392D
:10C9200000026F48390002B2323900026F513900FB
:10C9300002B2043900026F12390002B2F03900026B
:10C940006F5A390002B2033900026F63390002B234
:10C950009B3900026F1B390002B2203900026F6C54
:10C96000390002B2323900026F75390002B204395F
:10C9700000026F24390002B2203900026F7E3900B4
:10C9800002B2323900026F87390002B20439000264
:10C990006F2D390002B2CC3900026F90390002B21B
:10C9A000033900026F99390002B23A390002B4C06B
:10C9B000390003B70000390006C0010100005539F5
:10C9C00000026F00390016C1300F0AF91E40DB90DB
:10C9D0003FF3D3C47FE96E2C00036044A439000206
:10C9E0006F15390010C100180000A63533301D66E0
:10C9F0000FCB7200003900026F24390008C100100B
:10CA000030001735003900026F00390016C2380FA8
:10CA100002710211FB823FFB9C6AFFFE3D86000013
:10CA20005FE6F93900026F15390010C200003600C8
:10CA300017A333D009CB0F93E900003900026F240C
:10CA4000390008C290102A901335003900026F0097
:10CA5000390016C33C000AF9228426EC3FEB6D2016
:10CA6000000A17C080000000003900026F1539006D
:10CA700010C390142A90A65F331000000CCB9200D4
:10CA8000003900026F24390008C394242A942B35FE
:10CA9000003900026F00390016C43C0002400169F1
:10CAA00003903FFACB54C0000000000000000039A2
:10CAB00000026F15390010C48000BB90132933E0C9
:10CAC00000000C921300003900026F24390008C4E2
:10CAD000042030042735003900026F00390016C5E4
:10CAE0002A0F0AF92284D91400080EDC00204A58C3
:10CAF000FFF7D5E1643900026F15390010C5939135
:10CB00002A94235F331FE1C60035920000390002EA
:10CB10006F24390008C50000000000000039000241
:10CB20006F00390016C62A0F02110169FC96000435
:10CB3000BEAAC00040DE7FFFA2EF693900026F1578
:10CB4000390010C68424BC94372933DFF7E9006D1F
:10CB50001300003900026F24390008C600000000ED
:10CB60000000003900026F00390016C726000AF9DC
:10CB70001E402470000000007FD5380C000000002B
:10CB8000003900026F15390010C7039100041F35EA
:10CB90003330000003357200003900026F24390081
:10CBA00008C7000000000000003900026F003900D3
:10CBB00016C82E0002710211047E0003F348FFFD27
:10CBC000D63400000000003900026F15390010C88B
:10CBD0000420360437A333D00000036DE900003988
:10CBE00000026F24390008C800000000000000396E
:10CBF00000026F00390016C9210027D927D900008B
:10CC00003FE08EC63FE08EC6800633D5F139000284
:10CC10006F15390010C9001613007B7833D027D95F
:10CC20000F9B9B00003900026F24390008C90000E7
:10CC300000000000003900026F00390016CA27000A
:10CC400027D927D90000000000003FE08EC68000F1
:10CC50000000003900026F15390010CA007C130073
:10CC6000E17833D0000003659B00003900026F2497
:10CC7000390008CA000000000000003900026F00FF
:10CC8000390016CB2D0027D927D900003FE08EC6EA
:10CC90008000000000000000003900026F1539001C
:10CCA00010CB001679007BDE337000000C9B650012
:10CCB000003900026F24390008CB0000000000009A
:10CCC000003900026F00390016CC2B0027D927D974
:10CCD000000000000000800000007FF9CC2A0F391E
:10CCE00000026F15390010CC007C7900E1DE337F43
:10CCF000D82700656500003900026F24390008CC90
:10CD0000000000000000003900026F00390016CD5D
:10CD10002100038403C100003FFF26083FFF1EC41B
:10CD200000000D32843900026F15390010CD01FC6E
:10CD300017021B35339003A20FE2E1000039000215
:10CD40006F24390008CD0000000000000039000207
:10CD50006F00390016CE2D00038403C100003FFF91
:10CD600026080000000080000000003900026F1556
:10CD7000390010CE01FC36021B54334000000CE297
:10CD80001F00003900026F24390008CE00000000A7
:10CD90000000003900026F00390016CF270003841D
:10CDA00003490000000000003FFF3AE400000000DB
:10CDB000003900026F15390010CF021C17023935F7
:10CDC00033800000031EE300003900026F243900A5
:10CDD00008CF000000000000003900026F00390099
:10CDE00016D02B000384034900000000000000005F
:10CDF0000000FFFFF4735C3900026F15390010D09A
:10CE0000021C36023954335FFC9A001E1D000039A3
:10CE100000026F24390008D0000000000000003933
:10CE200000026F00390016D1000000000000000071
:10CE300000000000000000000000000000390002B7
:10CE40006F15390010D10000000000000000000044
:10CE500000000000003900026F24390008D10000F2
:10CE600000000000003900026F00390016D20000F7
:10CE700000000000000000000000000000000000B2
:10CE80000000003900026F15390010D200000000C8
:10CE900000000000000000000000003900026F24C4
:10CEA000390008D2000000000000003900026F00C5
:10CEB000390016D300000000000000000000000050
:10CEC0000000000000000000003900026F1539006A
:10CED00010D300000000000000000000000000006F
:10CEE000003900026F24390008D300000000000060
:10CEF000003900026F00390016D400000000000065
:10CF000000000000000000000000000000000039E8
:10CF100000026F15390010D400000000000000006E
:10CF2000000000000000003900026F24390008D41E
:10CF3000000000000000003900026F00390016D523
:10CF400000000000000000000000000000000000E1
:10CF500000000000003900026F15390010D50000F4
:10CF60000000000000000000000000000039000286
:10CF70006F24390008D500000000000000390002CD
:10CF80006F00390016D6000000000000000000000D
:10CF900000000000000000000000003900026F15D2
:10CFA000390010D600000000000000000000000062
:10CFB0000000003900026F24390008D6000000008C
:10CFC0000000003900026F00390016D70000000091
:10CFD0000000000000000000000000000000000051
:10CFE000003900026F15390010D700000000000062
:10CFF0000000000000000000003900026F2439002A
:10D0000008D7000000000000003900026F0039005E
:10D0100016D8000000000000000000000000000022
:10D02000000000000000003900026F15390010D820
:10D0300000000000000000000000000000000039B7
:10D0400000026F24390008D80000000000000039F9
:10D050000006F055AA520807390006C00101000079
:10D06000553900026F00390016C921002971297154
:10D0700000003FDEA7123FDEA7128006B563E1394C
:10D0800000026F15390010C981B50D821C7433E0A0
:10D0900029710F999900003900026F24390008C9DD
:10D0A000000000000000003900026F00390016CABD
:10D0B0002700297127D90000000000003FDFEF6240
:10D0C00080000000003900026F15390010CA821D6F
:10D0D0000D82827433D0000003679B000039000288
:10D0E0006F24390008CA0000000000000039000267
:10D0F0006F00390016CB2D0028A4297100003FDFF6
:10D100004C088000000000000000003900026F158C
:10D11000390010CB81B575821CDB337000000C9A8E
:10D120006700003900026F24390008CB00000000BE
:10D130000000003900026F00390016CC2B0028A433
:10D1400027D9000000000000800000007FF9AC90AB
:10D15000FC3900026F15390010CC821D758282DB0C
:10D16000338FD7C200666500003900026F24390092
:10D1700008CC00000000000000390002D94039004E
:10D18000053B001409AC390002030039000290028B
:10D19000390013918928000CC200031C017E000F86
:10D1A00008BB043D10F03900012C3900055107FF80
:10D1B0000FFF390005FFAA55A5803900026F1D3900
:10D1C0000002F2053900025320390001353900050B
:10D1D0002A000004373900052B0000095F390002DE
:10D1E0002F013900022604390006F055AA52080022
:10D1F000390002C0653900053B00100020390002EB
:10D2000090003900012C390003510300390006F069
:10D2100055AA520800390003B594423900026F053F
:10D22000390005B57F2B12333900026F0B3900042A
:10D23000B52B1A331100008930800960043800785A
:10D24000021C021C0200020E00200BAF0007000CA3
:10D2500000CF00D9180010F0030C2000060B0B3390
:10D260000E1C2A38465462697077797B7D7E0102F4
:10D270000100094009BE19FC19FA19F81A381A7880
:10D280001AB62AF62B342B743B7463F400000000AA
:10D29000000000000000000000000000000000008E
:10D2A000000000000000000000000000000000007E
:10D2B00000000000020218000302190006021A0012
:10D2C00007021B0008021C000E021D000F021E00B8
:10D2D00010021800110218011202190113021A019A
:10D2E00018021B0119021C011A021D011B021E015A
:10D2F00024021F01250218022602190227021A021F
:10D3000028021B0229021C0205021D02000218004D
:10D31000010218000C0218000D0218002A02180061
:10D320002B0218002C0218002D021800000010011A
:10D330000018020110030118040800050310060379
:10D34000180708000804080904100A04180B05004F
:10D350000C05080D05100E05180F06001006081123
:10D360000610120618130700140708150108160006
:10D37000001700081803001903081A08001B08000A
:10D380001C08001D08008020FFFF13000661008AB2
:10D3900025AC79A1101224002818010028180102D8
:10D3A0002818013000020100070700A253453792F8
:10D3B00000C7008400C700FAF4FB09FB09252323FA
:10D3C000E1218600010001000000020000000009C8
:10D3D000001000000000000000000000000000102D
:10D3E0000010000438096010230001270104030223
:10D3F00009010338090100000000000000000000DE
:10D40000000000000100012802040100032FFFFFBB
:10D41000FFFFFFFFFFFFFFFFFFFFFFFFFFFFFFFF1C
:10D4200001004E393836000400062001FFEC000CE4
:10D43000FFFFFFFE000000010000FFFE0000FFFFF5
:10D44000FFFE0000FFFE0001FFFF000300030005D8
:10D4500000010007FFFAFFFCFFFEFFFF00000001D4
:10D4600000010002000200000000000100020002B2
:10D47000FFFBFFE2000C00010000000100000001C2
:10D480000004000300010002000300050004000581
:10D4900000080009000F00080001FFF8FFF8FFFC7A
:10D4A000FFFDFFFF00000002000000020001000479
:10D4B000000100020003FFFEFFF5000AFFFBFFFB77
:10D4C000FFFEFFFDFFFFFFFF00040002000300045A
:10D4D000000400060007000B000D00100009FFF714
:10D4E000FFFCFFF4FFF8FFFDFFFE0001000000025B
:10D4F000000100030002000300040003FFFFFFF926
:10D500000001FFF9FFFCFFFF0001FFFFFFFF00002C
:10D5100000020001000500060008000B000C0013CB
:10D5200000090003FFFEFFFCFFF4FFF7FFFDFFFE15
:10D5300000000002000000030002000600070002D5
:10D5400000010004FFCA0006FFFF0001FFFF000109
:10D550000003000000040005000400070007000CA1
:10D56000000D001300100002FFFF0009FFFDFFF98E
:10D57000FFF5FFFBFFFCFFFE0001000000030002BF
:10D5800000030004000400060006FFDE0008FFFDA3
:10D59000FFFDFFFDFFFF0000000400030005000683
:10D5A0000007000B0009001000150005FFFAFFFF3F
:10D5B000000B0001FFFFFFF3FFF6FFFCFFFDFFFF85
:10D5C000000400010003000300090005000500023B
:10D5D000FFDA0003FFFBFFFBFFFDFFFE000400007E
:10D5E00000020003000500030009000D0012000DF9
:10D5F000FFFDFFF7FFFC0008000E0000FFF8FFF141
:10D60000FFF6FFFBFFFBFFFF000200010005000625
:10D61000000700070006FFC00004FFFEFFFD000139
:10D62000000000030003000600050007000B000DCA
:10D63000001300120003FFF7FFFA00000007000EBE
:10D6400000080001FFF2FFF7FFF9FFFDFFFE0001F8
:10D6500000000005000400090007FFFBFFED0003C8
:10D66000FFFBFFFBFFFE00010003000000030007BB
:10D6700000080007000F00120006FFF6FFF7FFFD8D
:10D6800000030006000A00100003FFFEFFF4FFF98C
:10D69000FFFCFFFEFFFF000100040006000600067D
:10D6A000FFF7FFEA0001FFFBFFFCFFFCFFFF0003A9
:10D6B000000200040007000A000E00130008FFFD2E
:10D6C000FFF3FFF9FFFFFFFF00050009000F00094E
:10D6D0000004FFF4FFF4FFF8FFFEFFFD000100046B
:10D6E0000007000400080005FFEA0005FFFEFFFC3C
:10D6F000FFFD00010003000200040007000B001101
:10D70000000D0003FFF3FFF3FFFDFFFE0001000625
:10D710000006000B0011FFFF0003FFF0FFF7FFFD05
:10D72000FFFD000200020003000400040003FFDC10
:10D730000001FFFDFFFDFFFEFFFD000100000006F0
:10D740000009000E00130007FFFBFFF2FFF9FFFBCB
:10D7500000000000000400060008000D000E00009C
:10D76000FFF7FFF4FFFAFFFDFFFDFFFF00030003DB
:10D7700000060005FFE20003FFFFFFFDFFFCFFFFC7
:10D78000000400020006000A0011000C0002FFF174
:10D79000FFF7FFFDFFFF000000080004000700087E
:10D7A0000009000C0003FFFDFFF3FFF8FFFD00017F
:10D7B00000050003000100020003FFF00004FFFF6A
:10D7C000FFFEFFFEFFFF000300050004000A001239
:10D7D0000006FFFDFFF7FFFAFFFEFFFF000000005D
:10D7E0000002000300040009000A000B0000FFFA19
:10D7F000FFF6FFFCFFFFFFFF000500010002000134
:10D80000FFEE0008FFFCFFFDFFFE00020002000328
:10D810000007000B00090002FFF8FFFBFFFE0000FD
:10D8200000010002000000020001000500040004E5
:10D83000000D0000FFFEFFF8FFFEFFFD00000001ED
:10D840000003000300010001000CFFFDFFFFFFFECD
:10D85000FFFF000100010001000600010002FFFCC3
:10D86000FFFE0001FFFE00010001000000010002B8
:10D8700000010004000300050002FFFFFFFBFFFDA5
:10D88000FFFE0000000100010001FFFD4654525957
:10D8900001069401D9F5F6F5F6F7F7F9FBFBFDFE65
:10D8A0000001030607080202020204030507070835
:10D8B000080806060707E417FBFBFAFBFCFDFEFF62
:10D8C000000102040507090B0B0A0A0B0B0E0C0ED4
:10D8D0001111121211100F10122B19FBFBFBFCFD82
:10D8E000FEFF000002030506080A0B0C0B0B0B0DD4
:10D8F000100D101213141313121112133018FCFC14
:10D90000FCFDFEFFFF000103040607090B0C0D0CD4
:10D910000B0D0F11101314151515141414151532C1
:10D9200019FCFCFCFDFEFF000102040506070A0CC1
:10D930000D0D0D0C0F1012101415161617151515C8
:10D940001616331BFDFDFDFEFF0001020304050753
:10D95000080A0C0D0E0E0E101213121516171717BB
:10D960001616161716351DFDFDFDFF0000010303F9
:10D97000050607080A0C0D0E0F0E121214141517C7
:10D980001718181817171818371EFCFDFDFEFF0092
:10D9900001020304050707090C0D0E0F0E121214E5
:10D9A0001215171718181816171814201EFCFDFC4E
:10D9B000FDFF0000020204040607090C0C0D0E0E08
:10D9C00011121412151617171717161717141F1BF5
:10D9D000FCFCFCFDFEFFFF010203040607090B0C23
:10D9E0000D0E0E11111312141616171717161617FF
:10D9F000173619FCFCFCFCFEFFFF000102040507C2
:10DA0000090B0B0D0D0D101113101315161616160C
:10DA1000151616173417FBFCFBFBFCFDFEFF00027E
:10DA200003050608090A0B0D0D0F1011101214152D
:10DA3000151515141516163316FBFBFBFBFBFCFD29
:10DA4000FF00020304050709090A0C0B0E0E110F53
:10DA5000121314141414131415153217FAFAF9F9D1
:10DA6000FAFBFCFE0001020304060708090C0A0B7E
:10DA70000C0F0D0F1213121313121113143113F88C
:10DA8000F8F8F8F9FAFBFDFEFF00020204060607AB
:10DA90000A090A0A0C0B0D1010111110100E1012A9
:10DAA0002DC9F0F0F0F0F1F1F3F5F6F7F7F9FAFC23
:10DAB000FDFDFE0706060708080A0C0C0D0E0F0EEA
:10DAC0000D0F11ED0000000000000000000000003C
:10DAD0000000000000000000000000000000000046
:10DAE0000000000000000000000000000000000036
:10DAF0000000000000000000000000000000000026
:10DB00000000000000000000000000000000000015
:10DCF00000000000000000000000000046544D330A
:10DD000001039601E40101FD0101FF010501050187
:10DD10000105030509070103FFFDFFFF01030103DF
:10DD200001050101FDFDD0260909050507050307C9
:10DD300005090503090E070E09090909090B05075D
:10DD40000E090B0909050905092B2A07070707070B
:10DD5000030707030B0703090E070E0B0B070B093D
:10DD60000B0707100E10070B05070709312A0709D3
:10DD7000070709050509050905050909090909092B
:10DD800009090909050910090B090D050905052FE0
:10DD900028090909070905050905090505090909EA
:10DDA0000E09090909090D0509100E1009090509CF
:10DDB00005092F2C090E090909050709050D090593
:10DDC0000B09090E0B0D090D090B050910090B09AB
:10DDD0000B070907052F2A070E07070E050509057A
:10DDE000090905090E090E09090909090905070E9E
:10DDF000090B0509050905092F2F090E09090E054B
:10DE00000509050D05050909090E09090909090989
:10DE100005090E090B070905090501122F09090952
:10DE20000909050907050D07050909070909090970
:10DE300009050D05090E090B0909030905FF122C37
:10DE4000090B09090B07070B070D07070B0B070B3E
:10DE50000B0B090B070B070710090B09090309072F
:10DE6000072D2A070E07070E050509050B05050BEB
:10DE700009070909090909090905070E070905091B
:10DE8000030705052F28090E09090E050509050DCB
:10DE90000905090E090E09090909090D05091209E3
:10DEA0000B0709050905092D280E10090E0E070795
:10DEB0000B070D0707090E070E0B0B0B0B090B07C2
:10DEC00007100E0B090B070907092D2A090E09096E
:10DED0000E050709050B09050B0E090909090909B2
:10DEE000090B0507100E0B0909050907092F28075B
:10DEF0000E07070903070B050B07050B0B09070B9B
:10DF00000B090B090B0707100709070D0707090B7A
:10DF10002DDC0103010103FDFF01FF01FFFF0103F0
:10DF20000103030D090B090D0709120E100B0D0952
:10DF30000B0D0DE4465452590105AA01D7F5F5F32E
:10DF4000F3F5F5F7F8FAFCFCFF00020407080104FA
:10DF50000404020304040608070705070608E2177D
:10DF6000FAFBFAF9FAFAFEFEFF0103040508090BB1
:10DF70000B0A0B0C0C0B0D0E0E11121111101011BF
:10DF8000112F18F9F8F9F8F9F9FBFCFE0001040665
:10DF9000080B090A090C0C0C0A0F0E1013141310AD
:10DFA000120F10103215F7F6F6F7F7F8FAFAFBFE33
:10DFB000FE00020405070706070808080A0B0A0DF9
:10DFC0000E0E0D0C0D0D0D2E19FAF9FAFAFCFCFED1
:10DFD000FF0002030506080B0C0C0C0D0E0F0D10B4
:10DFE00012111415141413131413351BFDFCFBFC30
:10DFF000FEFD01010103050607090B0C0D0D0E0FB7
:10E00000100E1112121515151514141515371DFCC7
:10E01000FCFBFDFEFD00010104050607090A0D0ECB
:10E020000E0E10100F1213121616161615151616C0
:10E03000381FFDFCFCFDFEFE010203040607070A73
:10E040000C0D0E10101111111314131617171716AB
:10E05000171715251DFAF9FAF9FCFBFEFEFF01035F
:10E06000040407090A0B0C0D0E0E0E1011101314E8
:10E07000141413131511221CFAFAFAFAFCFBFEFE13
:10E080000001030405080A0B0C0D0E0F100E1112EF
:10E090001115151515141516163818FAFAFAF9FA95
:10E0A000FBFEFEFF0102040507090B0C0D0D0E0F10
:10E0B0000E10111114141415131415153617F9F93F
:10E0C000F9F8F9F9FCFCFE000203040608090A0C41
:10E0D0000C0D0E0C0F101012131313121214143512
:10E0E00016F8F8F8F7F8F8FBFCFE00010303050743
:10E0F00008090B0B0C0C0B0D0F0E12121212111241
:10E1000012133417F9F9F8F7F8F8FCFDFE000203D2
:10E1100004050708090B0C0C0D0C0E0F0F12121240
:10E1200012111213133513F8F7F6F6F8F9FBFCFD8C
:10E1300000010302040606070B0B0B0C0A0D0E0E62
:10E14000101111111010111231C8EEEEEDEEEEEEBD
:10E15000F1F2F4F4F5F7F7FAFBFEFF0907070806FA
:10E160000808080B0C0B0C0B0B0C0DE946544D3337
:10E1700001019D01E70402040202020202020604F8
:10E18000040808080C080201010001000201040251
:10E19000040400000000CE2B0C0A08080A02040642
:10E1A00004080606080A080C0808080A080A060CEB
:10E1B0000A0C0C0C0A0406060A2B2B0A0808040891
:10E1C000040406040604060808080C0806060808E5
:10E1D0000A060A0A0C0C0A0A0406040A302B08086C
:10E1E000080406040404040806060808060C0606CB
:10E1F0000608080A060A0A0C0C06080606040A3075
:10E200002B0A080604080404040406040608080887
:10E210000A060604080808040608080A0608040492
:10E22000040A2E2B060A080408040406040804063F
:10E230000808080C06060608080804060A0C0A0660
:10E24000080404060A302F080A08080A040606040F
:10E250000804060A08060C0606060A080A04060848
:10E260000C0A06080404060A3031080808040804E9
:10E270000406040806060808060806060608080834
:10E2800004040808080608040604041531060808F2
:10E29000040A040406040806060A08060A06060616
:10E2A0000806080406080808060804040404152DD6
:10E2B0000808080406040404040606060808060AFA
:10E2C00006060608060804040808060408040404F0
:10E2D0000A2E2B0A0A080808040404040806060883
:10E2E00008060A06060408060A040608080A0606BE
:10E2F000040402082E290A0A080408040404040875
:10E3000004040808060A06060408060804040808A7
:10E31000060608020402082E290A0A0A080804064A
:10E3200006040806060808080A06060608080A047D
:10E33000060A0C0A06080406060A302B0C0A08080E
:10E340000A040606060806060A08060C0608080A55
:10E35000080804060A0C0A080A0406060C32290CEE
:10E360000A0A0A0A040606060806080A0A080C062B
:10E3700008060A0A0A060A0A0C0A0A0A0406060C11
:10E380002EDA0204040002FE000202000202000271
:10E390000204020E0A0C0C0C080E0E12100E0E0EC9
:10E3A0000C0E12E3464D53430007160013060507F3
:10E3B00007050807070608070705060706080904F2
:10E3C000060607050606060605040605030A0014E8
:10E3D0000507070707080A070809070608080606C9
:10E3E0000A080607070506060606060405050405CD
:10E3F0000D00140707080708090A09070A08090990
:10E4000009060608080607070607060506070506A3
:10E410000504040F00110604080806070707080B87
:10E4200008080B070807080606050606080605077C
:10E430000506050505030F0014060507070907096A
:10E44000090909080909080706090809080707064C
:10E450000707090805040504040F00160706070747
:10E460000809070808080908070908070A0805062F
:10E470000707070706080605050605051000150924
:10E480000708080B0A090908070809080A08070904
:10E490000808070706060705060704060405050F12
:10E4A0000015060509070A0907080A090A090B09E0
:10E4B00009060908080808060706060506060705EE
:10E4C00006060F001307060706090709090B0608C9
:10E4D000070A0809070A07070808070608060606C4
:10E4E00006060504040C00110607040809090708BC
:10E4F000090806080A090508080A080807060704A3
:10E500000506060405050305100015090508090997
:10E51000070609090808080A070807080707070582
:10E5200006060605060405060504040F0012040588
:10E5300007070B080709090908080707070608085D
:10E5400005050406060506050605050403030F0078
:10E550000F0406050707070807060607060507084C
:10E560000809060606070505040306070505050351
:10E57000040E00120507070608080808070808091E
:10E5800008080807090706060904060A070607041B
:10E59000040405040F00110707070B060809080803
:10E5A0000707070709060709080605070307060402
:10E5B00004070404050505100013060705060807EF
:10E5C00006060808080708060806080607050606DE
:10E5D000050605050404040405050A000000000002
:10E5E000000000000000000000000000000000002B
:10E5F000000000000000000000000000000000001B
:10E60000000000000000000000000000000000000A
:10E6100000000000000000000000000000000000FA
:10E6200000000000000000000000000000000000EA
:10E6300000000000000000000000000000000000DA
:10E6400000000000000000000000000000000000CA
:10E6500000000000000000000000000000000000BA
:10E6600000000000000000000000000000000000AA
:10E67000000000000000000000000000000000009A
:10E68000000000000000000000000000000000008A
:10E69000000000000000000000000000000000007A
:10E6A000000000000000000000000000000000006A
:10E6B000000000000000000000000000000000005A
:10E6C000000000000000000000000000000000004A
:10E6D000000000000000000000000000000000003A
:10E6E000000000000000000000000000000000002A
:10E6F000000000000000000000000000FFFFFFFF1E
:10E70000FFFFFFFFFFFFFFFFFFFFFFFFFFFFFFFF19
:10E71000FFFFFFFFFFFFFFFFFFFFFFFFFFFFFFFF09
:10E72000FFFFFFFFFFFFFFFFFFFFFFFFFFFFFFFFF9
:10E73000FFFFFFFFFFFFFFFFFFFFFFFFFFFFFFFFE9
:10E74000FFFFFFFFFFFFFFFFFFFFFFFFFFFFFFFFD9
:10E75000FFFFFFFFFFFFFFFFFFFFFFFFFFFFFFFFC9
:10E76000FFFFFFFFFFFFFFFFFFFFFFFFFFFFFFFFB9
:10E77000FFFFFFFFFFFFFFFFFFFFFFFFFFFFFFFFA9
:10E78000FFFFFFFFFFFFFFFFFFFFFFFFFFFFFFFF99
:10E79000FFFFFFFFFFFFFFFFFFFFFFFFFFFFFFFF89
:10E7A000FFFFFFFFFFFFFFFFFFFFFFFFFFFFFFFF79
:10E7B000FFFFFFFFFFFFFFFFFFFFFFFFFFFFFFFF69
:10E7C000FFFFFFFFFFFFFFFFFFFFFFFFFFFFFFFF59
:10E7D000FFFFFFFFFFFFFFFFFFFFFFFFFFFFFFFF49
:10E7E000FFFFFFFFFFFFFFFFFFFFFFFFFFFFFFFF39
:10E7F000FFFFFFFFFFFFFFFFFFFFFFFFFFFFFFFF29
:10E80000FFFFFFFFFFFFFFFFFFFFFFFFFFFFFFFF18
:10E81000FFFFFFFFFFFFFFFFFFFFFFFF46012B850D
:10E82000F4000000000000000000000004000000F0
:10E830003BB4AD07EBB5ED0090013D1E3214250051
:10E84000C201431F37150600F401491F3B1616008D
:10E8500026024F243F180700580253254419170079
:10E860008A025A26491B0800BC025F284D1C18006A
:10E87000EE026628541C090020036A2A571E19005C
:10E880005203712C5D1F29008403762F622039000A
:10E89000B6037C2F66220A00E80382316B231A003C
:10E8A0001A0487336F252A004C048B3372263A00F2
:10E8B0007E04923678280B00B004993980291B0019
:10E8C000E2049E3A822A2B001405A33A872C3B00CF
:10E8D0004605A83C8C2D0C007805AC40902F1C0000
:10E8E000AA05B04194302C00DC05B54299323C00B9
:10E8F0005A0020141A0D0000640023171C0E10008B
:10E900006E0020161A0D200082001F141B0D01003E
:10E910008C0021161A101100960021151A0E2100E4
:10E92000AA0020141B0D0200B40024171E0F1200B1
:10E93000C8002816210F2200DC002816210F030032
:10E94000F0002C1824101300FA00301826112300B0
:10E950000E013018261104002C01321B291214005C
:10E960004A01381C2D12050068013B1C30131500AC
:10E970009001020C1000F401020E08005802030F6F
:10E980001000BC02030F08008403040F10004C04A5
:10E99000050F10001405060F0400DC05070F040026
:10E9A0006E00000B20029600000D1000C800000D44
:10E9B0000400FA00010D10002C01010D08000000F8
:10E9C0006572726F72205B25735D20282530346478
:10E9D00029206461746120747970652069732073E3
:10E9E000686F727420726573706F6E736521206337
:10E9F0006D645F636F756E745B25645D206F766513
:10EA0000722073697A650A005B25735D20282530C2
:10EA10003464292076696463206572726F722021E4
:10EA2000737461747573305B307825785D3B7374F3
:10EA300061747573315B307825785D3B73746174F4
:10EA40007573325B307825785D210A005B25735D34
:10EA500020282530346429207761726E696E672121
:10EA60002054455B25645D206673206C696E655B90
:10EA700025645D2064697370206C696E655B256434
:10EA80005D2073746F705B25645D2074785F6C69C2
:10EA90006E655F64656C61795B25645D0A000000EA
:10EAA0006572726F72205B25735D20282530346497
:10EAB0002920445343204552525B307825785D200D
:10EAC0004552525F5250545B307825785D20525841
:10EAD000425220737461747573305B307825785DB1
:10EAE00020737461747573315B307825785D0A002A
:10EAF0006572726F72205B25735D20282530346447
:10EB000029206572726F72212120707073206C65EC
:10EB10006E677468203A202564202C6D617820731C
:10EB2000697A6520697320313238202120666C753E
:10EB3000736820706B74206275660A006CEB0100CC
:10EB4000D00107002C090000880B01006CEB0100CC
:10EB500000010700C00000002C150100C0F00100FA
:10EB6000FC0A0700BC2F00002C150100116201599E
:10EB70000741021464360AEC29B00F2D03F04D90C2
:10EB8000082DFBF97168082DF4FB9948082DEDFD5F
:10EB9000C128082DE7FBED080836E0FD19E10E2D30
:10EBA000DBF945C1082DD6F375A1082DD1EBA9815C
:10EBB000082DCDE1D969082DC9D50D52082DC7C73B
:10EBC0003D3A082DC4B7712A082DC3A79D1A083DE8
:10EBD000C293CD12084B7DF9083C672513202C4FBA
:10EBE0004D1B083DC5396D23402C1F8D3B083DCA88
:10EBF00007A94B602CEDC06B082DD0D5D48B082D08
:10EC0000D4BBE4B3082DD8A3F0DB082DDC8DF803CA
:10EC1000A82DE177F43B082DE561F86B083DE94D3F
:10EC2000F4A3D02C39F0DB0845F227E01B2D0AECC9
:10EC300029B0102D03F04D90082DFBF97168083DA7
:10EC4000F4FB9948302CFDC128082DE7FBED08089E
:10EC50002DE0FD19E1682DDBF945C1082DD6F375CE
:10EC6000A1083DD1EBA981A02CE1D969083DC9D506
:10EC70000D52C02CC73D3A083DC4B7712AE03CA7ED
:10EC80009D1AF04B93CDF84B7DF9083C6725132076
:10EC90002C4F4D1B083DC5396D23402C1F8D3B0863
:10ECA0003DCA07A94B602CEDC06B082DD0D5D48B85
:10ECB000082DD4BBE4B3082DD8A3F0DB082DDC8DE0
:10ECC000F803A82DE177F43B082DE561F86B083DCA
:10ECD000E94DF4A3D02C39F0DB0895F227E01B12A4
:10ECE000FF2301A012A01401A20215C00701A41362
:10ECF00005A41303A41F02A40501A405061304A47C
:10ED00001501A4031314A4030C33A203120332014C
:10ED100024C0E1E42909011B1201EA0222828215C2
:10ED20001D03020202C20225080986A623FA201248
:10ED3000781C3E0507F42129D72908DA3F105A42EA
:10ED4000105A0810031B02030418B4C404363772A7
:10ED5000DDC80E2D3174F5C0082D2C720DC1083C94
:10ED6000267225083C21703D083C1B6E59083C1654
:10ED70006C71082D116889C9082D0C64A1D1082D6A
:10ED80000760B9D9082D0358D1E9082DFE53E9F9D8
:10ED90000836FA4B010A0F2DF645151A082DF23DDB
:10EDA0002D2A082DEF334142082DEB2B555A082D03
:10EDB000E821657A082DE5177992082DE30B89B2D1
:10EDC000082DE10195D2082DDFF5A4F20845DDE913
:10EDD000B01A45DBDDC03A45DAD1C86245D9C5D0A5
:10EDE0008A3DD8B9D8B2083CADDCDA082D9FE00ADC
:10EDF00001083C93E432083C87E462082C7BE88AF3
:10EE0000082D347ED1C8A82D2E80E9C0082D288079
:10EE100005B9083C22801D082D1D7E39B1083C171C
:10EE20007C55083C127A6D083C0C7889083C0772C6
:10EE3000A5283D026CC1C1F82C67D9C9082DF9611C
:10EE4000F5D1082DF5590DE2082DF15125F2082DC7
:10EE5000ED493D02C82DE93F551A083DE6356932B6
:10EE6000F02C2B7D4A082DE01F916A082DDE13A19E
:10EE70008A082DDC07B1AA082DDAFBC0CA082DD9F3
:10EE8000EDCCF20845D8E1D81245D7D3E43A3DD6C7
:10EE9000C5F062083CB7F492083CABF8BA083C9D58
:10EEA000FCEA28128F2A13F013D7832A430813D8B9
:10EEB000752A73084548DE20094545E0241145427E
:10EEC000DE2C214540DA3431453DDA3841453BD628
:10EED00040514538D644614535D44C714533D05402
:10EEE000814531CE5891452ECC60A1452CCA64B1E4
:10EEF0004529CA68C14527C670D14525C474E14576
:10EF000023C278F12D20C08001882D1EBC841908F1
:10EF10002D1CBA8829082D1AB88C39082D18B494DC
:10EF200049082D16B29461082D14B09871082D125D
:10EF3000AC9C89082D10AAA099082D0EA6A8A90896
:10EF40002D0CA2ACC1082D0AA0ACD9082D089CB488
:10EF5000E90836069AB401022D0496BC11082D0268
:10EF600092C029083647021D890F2D4302259908B2
:10EF70002D40FE30A9082D3DFC38B9082D39FA4442
:10EF8000C9082D36F84CD9082D33F458E9082D2F2F
:10EF9000F460F9083D2CF26809E844EE74193D2646
:10EFA000EA7C31E03CE88441E044E48C59451DE2D0
:10EFB0009469451ADE9C814518DAA4914515D6ACB2
:10EFC000A94512D2B4C14510CEBCD1450DCAC4E981
:10EFD0003D0BC6C801C83CC2D019C82CBED43108EC
:10EFE0002D03BADC49082D01B4E461082DFFB1E816
:10EFF00079082DFDADE899082DFBA7F0B1082DF992
:10F00000A3F4C9082DF79DF8E9082DF599FC01F83E
:10F010002DF393041A0810418710C5077E24C107F9
:10F02000743CB9076A52B5076166B107577CAD07F2
:10F030004D90AD0744A2AD073BB4AD0732C4B10754
:10F0400029D4B50721E2B90719ECC50712F4D10795
:10F050000BFCDD0705FEED0713FE0114FBFF151485
:10F06000F7FD2D14F4F54914F1ED6514EEE3851464
:10F07000EDD5A514ECC5C914EBB5ED101DEBA3112E
:10F0800001EB913501EB7D5D01EC678501ED53A945
:10F0900001EE3DD101F025F9012995C1091A10129F
:10F0A0005803104008125C0310400912600310401E
:10F0B0000A1264F3400BD4441A07F2FF022F060031
:04000005000100C135
:00000001FF
